:100000000C94C4090C94210A0C94210A0C94210A22
:100010000C94210A0C94210A0C94210A0C94210AB4
:100020000C94210A0C94631D0C94210A0C94210A4F
:100030000C94DE380C94210A0C94210A0C94210AA9
:100040000C94210A0C94210A0C9481190C94210A15
:100050000C9422100C94210A0C94EC0F0C94210A9D
:100060000C94A9200C94210A0C9403340C94210ABA
:100070000C94DD9C0C94210A0C942E920C94210A71
:100080000C94210A0C94210A0C94210AD220D72026
:10009000DC20E520FC201321232133216E21FF23C6
:1000A00013218A229B22CB22EA2207236123BC232D
:1000B0006F265027E62767289F284F29162A772A78
:1000C000E92A292B812BAF2BDC2B412C8C2CD72C14
:1000D0003B2D372E2234563497340935213561357E
:1000E00027362B372B372B372B372B372B372B3705
:1000F0002B372B372B372B37E036E236E736FF36F8
:100100000137A17295731A7441736E749D74E07215
:1001100070739F834384C8842A857E85E785658DB7
:1001200068869A869A869A869A869A869A869A8601
:100130009A869A86C8864387D487F9873C889488AC
:100140002A89358A9C8A9C8A9C8A9C8A9C8A9C8A59
:100150009C8A9C8A9C8AD48AF28A178B738BAF8B79
:10016000138C408CE08C658D408D408D408D408D92
:10017000408D408D408D408DEC9AEF9AEF9AEF9A2A
:10018000F89AFB9AFE9A109B0D9B0A0D3D3D3D3D52
:100190003D3D3D3D3D3D3D3D3D3D3D3D3D3D3D3D8F
:1001A0003D3D3D3D3D3D3D3D3D3D3D3D3D3D3D00BC
:1001B0000A0D426174743A002025642043656C6C1A
:1001C000732000204C6F77207761726E696E673AFA
:1001D0002025642E25640020204175746F6C616EAB
:1001E00064696E673A2025642E2564000A0D466F07
:1001F000756E6420424C2D4374726C3A2000256465
:10020000000A0D0A0D2121204D495353494E472024
:10021000424C2D4354524C3A202564202121000A9F
:100220000D43616C6962726174696E6720707265FA
:1002300073737572652073656E736F722E2E004F27
:100240004B0A0D000A0D466C696768742D74696D60
:1002500065202575206D696E20546F74616C3A2598
:1002600075206D696E00416E676C654E69636B2029
:10027000202020202020416E676C65526F6C6C201E
:100280002020202020204163634E69636B202020C2
:10029000202020202020416363526F6C6C2020209E
:1002A0002020202020205961774779726F2020205C
:1002B000202020202020416C746974756465205BC7
:1002C000302E316D5D204163635A20202020202094
:1002D0002020202020204761732020202020202063
:1002E000202020202020436F6D70617373205661A1
:1002F0006C7565202020566F6C74616765205B30DB
:100300002E31565D20205265636569766572204CFA
:100310006576656C20204779726F20436F6D706140
:100320007373202020204D6F746F722031202020A5
:100330002020202020204D6F746F7220322020203A
:100340002020202020204D6F746F72203320202029
:100350002020202020204D6F746F72203420202018
:100360002020202020203136202020202020202066
:100370002020202020203137202020202020202055
:100380002020202020203138202020202020202044
:100390002020202020203139202020202020202033
:1003A000202020202020536572766F2020202020DE
:1003B000202020202020486F7665726761732020FE
:1003C00020202020202043757272656E74205B30DF
:1003D0002E31415D20204361706163697479205B37
:1003E0006D41685D202048656967687420536574B5
:1003F000706F696E7420323520202020202020204C
:1004000020202020202032362020202020202020C4
:10041000202020202020436F6D706173732053656E
:1004200074706F696E744932432D4572726F722019
:10043000202020202020424C204C696D697420200F
:100440002020202020204750535F4E69636B2020DE
:100450002020202020204750535F526F6C6C2020BA
:1004600020202020202021212120494E434F4D5083
:10047000415449424C4520212121002E000A0D20E3
:10048000444143206F7220493243204552524F521B
:100490002120436865636B204932432C2033567218
:1004A00065662C2044414320616E6420424C2D43FC
:1004B00074726C005B25695D005B25695D002B2013
:1004C0004D696B726F4B6F70746572202B004857CB
:1004D0003A5625642E25642053573A25642E25303C
:1004E00032642563200053657474696E673A25642D
:1004F000202573004D69786572204572726F7221F4
:10050000004552522532643A004861726477617244
:1005100065204572726F7220313A256420212100D6
:100520004D697373696E6720424C2D4374726C3A47
:10053000256420212100493243204552524F522147
:10054000212100424C2D53656C66746573742045FF
:1005500072723A253264004865696768743A2020EF
:1005600025356900536574706F696E743A25356975
:100570000050726573737572653A253569004F6670
:10058000667365743A2020253569002841290025C5
:1005900069006163742E2062656172696E67004E46
:1005A00069636B3A20202020202025356900526F96
:1005B0006C6C3A20202020202025356900436F6D87
:1005C000706173733A202020253569004B25693A04
:1005D00025346920204B25693A25346920004E696D
:1005E0003A2534692020526F3A2534692000477338
:1005F0003A253469202047693A2534692000503172
:100600003A253469202050323A253469200050338D
:100610003A253469202050343A253469200047793E
:10062000726F202D2053656E736F72004E69636B7D
:100630002025346920282533692E25782900526F1A
:100640006C6C2025346920282533692E25782900F3
:1006500059617720202534692028253369290041F4
:100660004343202D2053656E736F72004E69636B98
:100670002025346920282533692900526F6C6C20AD
:10068000253469202825336929005A202020202577
:10069000346920282533692900566F6C74616765B9
:1006A0003A2020202533692E253169560043757282
:1006B00072656E743A2020202533692E25316941F8
:1006C00000506F7765723A2020202020253469572A
:1006D000004469736368617267653A202535696D06
:1006E00041680052656365697665720052432D5119
:1006F00075616C6974793A202534690052432D4341
:1007000068616E6E656C733A25346900436F6D7075
:10071000617373004D61676E65743A202020253542
:1007200069004779726F3A20202020202535690022
:10073000536574706F696E743A2025356900506F87
:10074000746925693A202025336900506F74692542
:10075000693A202025336900536572766F202000A6
:10076000536574706F696E74202025336900506F73
:10077000736974696F6E3A202533690052616E6740
:10078000653A2533692D25336900424C2D43747237
:100790006C204572726F72732000253364202533FC
:1007A0006420253364202533642000424C205465A6
:1007B0006D70657261747572650025336420253330
:1007C0006420253364202533642000424C20437587
:1007D0007272656E740028696E20302E31412900D6
:1007E0002533642025336420253364202533642099
:1007F00000424C2D4374726C20666F756E6420004D
:100800002025632020202563202020256320202010
:10081000256320002025632020202563202020251B
:1008200063202020256320002025632020202D2008
:1008300020202D2020202D200031300031310031AA
:100840003200466C696768742D54696D652020001C
:10085000546F74616C3A2535756D696E004163742F
:100860003A20202535756D696E00287265736574B0
:1008700029000A0D2D2D3E20486172647761726552
:100880002056657273696F6E2042797465204368E3
:10089000616E676564203C2D2D000A0D47656E650D
:1008A000726174696E672064656661756C7420504E
:1008B0006172616D657465722053657420256400F2
:1008C0000A0D5573696E6720506172616D657465BC
:1008D0007220536574202564000A0D47656E6572A9
:1008E0006174696E672064656661756C74204D691A
:1008F000786572205461626C65000A0D4D697865F7
:10090000722D436F6E6669673A202725732720286A
:100910002575204D6F746F727329000A0D41434392
:10092000206E6F742063616C69627261746564210A
:100930000D0A0000008F001E01AD013B02CA0258E3
:1009400003E603740402058F051B06A7063307BEE2
:10095000074808D2085B09E3096B0AF20A780BFD25
:100960000B810C040D860D070E870E060F840F00F9
:10097000107B10F5106E11E5115B12CF124213B30C
:100980001323149214FE146A15D3153B16A11605F1
:10099000176717C81727188318DE1837198E19E339
:1009A00019361A871AD61A231B6E1BB61BFD1B415C
:1009B0001C831CC31C001D3C1D751DAB1DE01D12BE
:1009C0001E421E6F1E9A1EC31EE91E0D1F2E1F4DB6
:1009D0001F691F841F9B1FB01FC31FD31FE11FEC84
:1009E0001FF51FFB1FFF1F002004010000FF7900FF
:1009F000020101457B01030202D97B02040303814A
:100A00007C03000404367C2532692E2531695600AA
:100A1000253364256320253033646D2563005374CA
:100A200061747573004552524F523A20253264204A
:100A30000053657425643A2573202000253469200D
:100A40002532693A25303269002534696D25630005
:100A50002533692025336920253369202533690032
:100A60002533692025336920253369202533690022
:100A700054656D70657261747572657320202020F5
:100A8000002563432020202020002532692E2531B7
:100A90006956202533692E2531694100253469576F
:100AA000202536696D4168004D61676E65743A2591
:100AB0003369252520253369256300496E636C69F8
:100AC0002E3A2533692563202825692920002532FF
:100AD000756D2F73205361743A25642000202033F4
:100AE00044004E6F4678004447505300486F6D6590
:100AF0003A2533646D202533642563202563004E39
:100B00006F204E6176694374726C2100000005000D
:100B100005000401060108000601020004000400AB
:100B20000700070007000700070007000700030190
:100B30000301050017010F01060009010A0119014F
:100B40000501050119011A010F01010009004E6F8D
:100B5000204572726F722020202020202020004E1D
:100B60006F7420636F6D70617469626C6520200022
:100B70004D4B334D6167206E6F7420636F6D7061F4
:100B8000004E6F20464320636F6D6D756E69636123
:100B90007400436F6D7061737320636F6D6D756E5C
:100BA00069630047505320636F6D6D756E696361B3
:100BB00074696F00636F6D706173732076616C751B
:100BC00065202020005243205369676E616C206CC1
:100BD0006F73742020004643207370692072782060
:100BE0006572726F7220004E6F204E4320636F6DEE
:100BF0006D756E69636174004643204E69636B20B6
:100C00004779726F2020202000464320526F6C6C81
:100C1000204779726F2020202000464320596177B9
:100C2000204779726F2020202020004643204E6903
:100C3000636B204143432020202020004643205264
:100C40006F6C6C204143432020202020004643202D
:100C50005A2D414343202020202020202000507284
:100C60006573737572652073656E736F72200049CA
:100C700032432046432D3E424C2D4374726C20007B
:100C8000426C204D697373696E67202020202020FC
:100C9000004D69786572204572726F7220202020A5
:100CA00020004361726566726565204572726F72DD
:100CB00020200047505320466978206C6F737420C1
:100CC000202020004D61676E6574204572726F723E
:100CD00020202020004D6F746F7220726573746144
:100CE000727420202000424C204C696D697461743C
:100CF000696F6E202020004750532052616E676557
:100D000020202020202020004E6F2053442D4361BE
:100D100072642020202020200053442D4C6F6767F0
:100D2000696E67206572726F7200466C79696E67D2
:100D30002072616E676521202020004D617820417E
:100D40006C74697475646521202020004E6F204703
:100D500050532066697820202020202000636F6D8A
:100D600070617373206E6F742063616C2E00424C4F
:100D70002D53656C66746573742020202020005309
:100D8000657420203A002021212020204C414E442F
:100D9000494E4720202020212120200020212120F1
:100DA0004C69506F20766F6C74616765202121203B
:100DB000200020202020204D696B726F4B6F7074D3
:100DC00065722020202020002020202020202020AC
:100DD0002020202020202020202020202000202033
:100DE0002532692E253169562020002020253269C0
:100DF0002E25316956202000414C543A2534696D26
:100E000020256300414C543A2534696D202000416F
:100E10004C543A2D2D2D2D200020202532693A25C5
:100E200030326920200020202532693A253032698D
:100E30002020004449523A202533642563004300B2
:100E4000200020202535692020002020253569201C
:100E50002000493A2532692E2531694120003A00A7
:100E60003A003A002D2D2D2D2D2D2D2D2D2B2D2DF4
:100E70002D2D2D2D2D2D2D2D2D002D2D2D2D2D2DCF
:100E80002D2D2D2D2D2D2D2D2D2D2D2D2D2D2D00BF
:100E90003A005341543A2532642000444953543AAD
:100EA0002533646D004420003344002121004D416E
:100EB000473A25337525252000484D3A25336425CA
:100EC0006320256300696E636C3A253264256328CC
:100ED0002532692900202020202532756D2F733A94
:100EE0002020484D3A253364256320256300455270
:100EF000523A202532642021004552523A200021E6
:100F000021204C69506F20766F6C746167652021D9
:100F10002100207777772E4D696B726F4B6F70745D
:100F200065722E6465202000202532693A25303212
:100F30006920202532692E25316956202534696DB6
:100F4000416800202532693A253032692020253257
:100F5000692E25316956202534696D416800444960
:100F6000523A253364256300414C543A2534696D67
:100F700000414C543A2534696D00414C543A2D2DB2
:100F80002D2D2000256300484D3A2533642563202C
:100F900020444953543A2533646D2025630050574B
:100FA000523A2532692E2531694120282569572971
:100FB00020004346002020004750533A2532756DEB
:100FC0002F73205341543A256420002020334420BD
:100FD000004E4F46495800444750532000202020DF
:100FE0004E6F204E6176694374726C202020202061
:100FF0002020002532692E2569202532692E256999
:10100000202532692E2569202532692E2569410067
:101010002533692025336920253369202533692547
:101020006343002532692E2569202532692E256902
:1010300041002532692E2569202532692E25692037
:101040002532692E2569202532692E256941002522
:101050003369202533692563432020202020202068
:101060002000253369202533692025336920253365
:1010700069256343004552523A20253264202100FD
:101080004552523A20002121204C69506F20766F42
:101090006C7461676520212100207777772E4D6978
:1010A0006B726F4B6F707465722E646520200053F5
:1010B000657474696E673A257520257320004D6943
:1010C0006E3A2532692E253169562025732000415C
:1010D0004C543A00504F54493A2533752000284F5C
:1010E0004E29202000284F46462920004C494D49D2
:1010F0005400564152494F0044495341424C4544E3
:101100000043463A0044495341424C45440020289C
:101110004F4E29200020284F4646290020544541A3
:101120004348004750533A0044495341424C4544D8
:10113000002846524545290028484F4D452900289A
:1011400041494429200028484F4C44290020465357
:101150003A257573656B2000484F4D4520414C542E
:101160003A0025756D00484F4C4420004E693A25E1
:10117000346920526F3A25346920433A2533690097
:1011800047733A2534692059613A25346920005063
:10119000313A2534692050323A25346920333A25D2
:1011A00033690050343A2534692050353A25346982
:1011B00020363A25336900434F55504C494E47205D
:1011C0004F46462120004C4F4F50494E47212000AA
:1011D0004848212000434F4D50415353204F46462D
:1011E000212000004F505152535453565748005835
:1011F00059005A5545464748410049424A4A00006D
:10120000000000000000000000444C4D0000000001
:10121000004E0000004B00430A0D7777772E4D6992
:101220006B726F4B6F707465722E64652028632932
:1012300020486953797374656D7320476D62480067
:101240000A0D74686520757365206F66207468697F
:101250007320736F667477617265206973206F6E97
:101260006C79207065726D6974746564200A0D6F05
:101270006E206F726967696E616C204D696B726F69
:101280004B6F707465722D4861726477617265008E
:101290005573657200486F545420563400414354CE
:1012A0002044534C004A657469005370656B747236
:1012B000756D0050504D000A0D5265636569766585
:1012C000723A2000532E42757300756E6B6E6F7705
:1012D0006E2E205573696E672050504D2E2E2E00B5
:1012E0006E6F7420737570706F72746564206279AC
:1012F00020686172647761726521000A0D202D20DB
:101300004C4942204E4F5420434F4D504154494286
:101310004C452021212121000A0D0A0D21212042C6
:101320006F6F746C6F61646572206E6F7420636F91
:101330006D70617469626C6520746F2048617264BD
:1013400077617265203E20322E322021210A0D0A5B
:101350000D000A0D466C69676874436F6E74726F96
:101360006C0A0D48617264776172653A25642E25B6
:10137000640A0D536F6674776172653A5625642E60
:10138000253032642563200011241FBECFEFD0E446
:10139000DEBFCDBF12E0A0E0B1E0ECE9F0E401E097
:1013A0000BBF02C007900D92A83EB107D9F71CE011
:1013B000A8EEB2E001C01D92A73BB107E1F77AEABF
:1013C000E2E0F0E081E280935700D4907E0108943F
:1013D000E11CF11C20EF37EF41E050E087016FE0A6
:1013E000DA01C9012F5F3F4F4F4F5F4FABBFFC0189
:1013F0008791F80181938F01615067FFF1CF84EEEF
:101400008ABD898580936D05893138F086E08093A7
:10141000140187E0809313017BEAF7016EE081916C
:1014200078277095615067FFFACF8889781729F07F
:10143000F7E9DF1611F40000FECF0E940A0B0C94AE
:101440004DA00C9400008AE891E09F938F9388E967
:1014500096E19F938F93E0919C05F0919D050995EE
:101460000F900F900F900F90089580914108E82FF2
:10147000FF27EE0FFF1FE858F64F808191818D5EA8
:101480009F4F14F010920401808191818A5B9F4FDD
:10149000CCF4809104018823A9F481E080930401B5
:1014A0008091D0058F5F8093D005853038F088EE2D
:1014B00093E090931E0380931D03089566E970E006
:1014C0000E94243C0895CF93DF93C82F882389F08E
:1014D00080EB91E09F938F9388E996E19F938F93A0
:1014E000E0919C05F0919D0509950F900F900F904C
:1014F0000F9080912601909127016BE270E00E948D
:10150000C09F962F9F5F9093000180916408823363
:1015100018F5989F802D112480930201CC23F1F0BF
:1015200068EC70E0892F0E94243C8091000199278B
:101530009F938F9388EB91E09F938F9388E996E137
:101540009F938F93E0919C05F0919D0509958DB730
:101550009EB706968DBF02C0809302019091AF089E
:10156000923338F480910001899F802D112480935B
:10157000AF088091AF0890910201981720F4915024
:101580009093AF089F5FCC2309F441C0892F6AE094
:101590000E94A09F892F99279F938F93809102018A
:1015A0000E94A09F99279F938F9383EC91E09F9334
:1015B0008F93C8E9D6E1DF93CF93E0919C05F0913A
:1015C0009D0509958DB79EB708968DBF8091AF0890
:1015D0008823E9F06AE00E94A09F892F99279F93B2
:1015E0008F938091AF080E94A09F99279F938F931C
:1015F00087ED91E09F938F93DF93CF93E0919C05CC
:10160000F0919D0509958DB79EB708968DBFDF9126
:10161000CF910895CFEFD0E4DEBFCDBF88249924C9
:10162000C1E07C2E14B815B88AE08AB98FE58BB971
:10163000B7EECB2EB3E0DB2E2EEC3FEFC20ED31E67
:10164000D7FEFACF6624199B08C04C9B04C085E1E5
:101650008093030108C086E101C089E18093030102
:1016600081E08093080481E887B93E9A8FEF88B9BA
:101670008BE184B981E085B9469A84B7877F84BFBE
:10168000809160008861809360001092600084EC1B
:1016900099E090931E0380931D03109256041092BC
:1016A000550410927D0910927C09109258041092F2
:1016B000570410925A0410925904209103012431C6
:1016C00028F084EC94E0A0E0B0E004C08BE095E06A
:1016D000A0E0B0E08093420190934301A0934401C5
:1016E000B09345012A3011F0243110F0289801C040
:1016F000289A2C3010F0293111F4299A01C0299828
:101700000E94D21A0E94A31A0E94A0160E94A53815
:101710000E94E41E81E00E94B7330E9447710E943C
:10172000797D85E00E94649B809103018C3010F0EC
:10173000893111F4299A01C0299878940E949E3227
:1017400080916A03826080936A0310926D030E9405
:10175000314884EF91E00E94691A6C0180916A031C
:1017600080FD05C0C6010E94721A8823B9F38CEE71
:1017700091E09F938F93A8E9AA2EA6E1BA2EBF927B
:10178000AF92E0919C05F0919D05099580EA9FE05C
:101790000E94691A6C01C0E0D0E00F900F900F908A
:1017A0000F900AE119E0FEECEF2EF8E0FF2E0E9408
:1017B000314880916A0380FD05C0C6010E94721AFB
:1017C0008823B9F3F70180811816ACF40BC00E948E
:1017D000314880916A0380FD05C0C6010E94721ADB
:1017E0008823B9F3C6010E94721A882321F4F801F4
:1017F0008081882364F7F801808187FF19C02196D2
:10180000DF93CF9321978EEF91E09F938F93BF92B9
:10181000AF92E0919C05F0919D0509958091E902B8
:101820008F5F8093E9022DB73EB72A5F3F4F2DBFF0
:10183000219684E090E0E80EF91E085F1F4FCC303F
:10184000D10508F4B4CFC0E0D0E007E119E0EEEC38
:10185000EE2EE8E0FE2EF801838187FD1DC0F70122
:1018600080811816CCF42196DF93CF93219781E0E5
:1018700092E09F938F9388E996E19F938F93E091F5
:101880009C05F0919D05099582E080931B032DB77F
:101890003EB72A5F3F4F2DBFF80183818078838355
:1018A000219624E030E0E20EF31E085F1F4FCC309B
:1018B000D10588F20E94230A90913F088091E902A5
:1018C000981728F48091B60580618093B6058FE162
:1018D00092E09F938F93C8E9D6E1DF93CF93E09195
:1018E0009C05F0919D05099588EE93E00E94691A88
:1018F0006C010E94221F0F900F900F900F90C60155
:101900000E94721A8823D9F38FE392E09F938F93FA
:10191000DF93CF93E0919C05F0919D05099580E0C0
:101920000E94083D809103010F900F900F900F903F
:101930008A3011F0843110F0289801C0289A80ED87
:1019400097E090931E0380931D0385E58093D20555
:101950008EE090E00E94BE309927182F00278FE07C
:1019600090E00E94BE30080F111D1093EF0200930B
:10197000EE028AE090E00E94BE309927182F0027DF
:101980008BE090E00E94BE30080F111D1093ED0215
:101990000093EC020F5F1F4F39F08091EE0290919F
:1019A000EF028F5F9F4F41F41092EF021092EE0210
:1019B0001092ED021092EC028091EC029091ED02F7
:1019C0009F938F938091EE029091EF029F938F935C
:1019D00084E492E09F938F93DF93CF93E0919C05F3
:1019E000F0919D0509950E94E72588E893E1909381
:1019F0003D0180933C01C1E0C093D1058C2F0E9432
:101A0000630A809167080E94B09A0E94230A80EDC1
:101A100097E00E94691A6C018AEF90E00E94691AAF
:101A200083E0809399071092E8028091B2082DB765
:101A30003EB7285F3F4F2DBF84FF02C0C093F00226
:101A400012BC11BC8091F202882311F04798FECF9E
:101A500080912103882309F4AEC280911801882364
:101A600009F4A9C2F8948091210381508093210345
:101A700078948091D005882319F00E94350A02C01D
:101A80000E94B84B0E943148209103012A3011F086
:101A9000243110F0289801C0289A809149048823A5
:101AA00031F0809149048150809349040EC08091A7
:101AB0006F00806280936F0010927909109278090C
:101AC0008091B60588608093B60580913C01909125
:101AD0003D01019790933D0180933C0180913C0131
:101AE00090913D01892B21F080916B038823C9F1EE
:101AF00080913C0190913D01892BD9F40E94E13302
:101B000085E090E090933D0180933C018091D30764
:101B10009091D40701969093D4078093D307809136
:101B2000B60581608093B60580919A0782608093A4
:101B30009A0780910B0190910C018F5F9F4FC1F428
:101B4000809148048823A1F088EA91E690931E03CF
:101B500080931D0380E890E090930C0180930B012B
:101B600007C02A3011F0243110F0289801C0289ABB
:101B70000E94609C80912103882309F01AC2809101
:101B80006805882319F00E94E58D13C28091110128
:101B9000882311F00E942C1B0E94E9160E947712E4
:101BA000C6010E94721A882309F4FFC184E190E003
:101BB000C80ED91E0E94EA1A80916708863019F46F
:101BC0000E94638304C0843011F40E94B58E80911A
:101BD0000804882331F18091E0079091E1078C524D
:101BE000914074F08091A9079091AA07805092408B
:101BF000C4F48091E0079091E107835593408CF005
:101C0000639432E3361570F480914804882331F0F0
:101C10008091B50580628093B50504C0809334043B
:101C200001C0662480916B03882329F48091F10A16
:101C30008E3150F405C08091B60582608093B60560
:101C400080919A0782600FC080911D0390911E03BE
:101C5000892B59F480913C0190913D01079728F020
:101C600080919A078D7F80939A078091F002882354
:101C700061F080914904873940F01092F00288E8C1
:101C800093E190931E0380931D03809106018823A6
:101C900021F08150809306012EC08093DC051092C4
:101CA0001C0410921B0410921A0410921904109232
:101CB000180410921704809149048823E1F480915C
:101CC0000B0190910C018F5F9F4FA9F42091F002BE
:101CD000223089F088E99AE390931E0380931D03D4
:101CE00080E09CE090930C0180930B01222319F07B
:101CF00082E08093F0028091A401893C70F08150D1
:101D00008093A4018091B6058B7F8093B605809166
:101D1000B90581608093B90551C080917E0A8823FE
:101D2000F9F08091B60584608093B60589E08093D0
:101D30002A0580910B0190910C018F5F9F4F81F4D8
:101D400080914804882361F088E99AE390931E0308
:101D500080931D0380E098EA90930C0180930B011F
:101D600010921C0510921B0510921A05109219056D
:101D7000109218051092710A8FEF8093E60A109264
:101D8000B00A1092AF0A1092B20A1092B10A8FEF05
:101D90009FEF9093AE0A8093AD0A10923804109290
:101DA000390410923A0410923B0410923C04809142
:101DB000B9058E7F8093B9051092A401609102014C
:101DC000262F332780912601909127012817390764
:101DD000F4F08091100480628093100480910B01D4
:101DE00090910C018F5F9F4F91F48091260190910B
:101DF00027010B9764F080E797E190931E0380938F
:101E00001D0380E093E090930C0180930B0112BCC2
:101E100011BC8091F1028F5F8093F102813309F050
:101E20007BC01092F10280915205882319F08150F5
:101E3000809352058091100481FF0AC08091EA02CC
:101E40009091EB0201969093EB028093EA0204C01A
:101E50005AEA852E55E0952E809111049091120436
:101E60008050944008F049C02091E2073091E30788
:101E70004091E4075091E50780911E0190911F0168
:101E8000A0912001B0912101281739074A075B076B
:101E900064F48091E2079091E307A091E407B09188
:101EA000E5070596A11DB11D20C02091E2073091E4
:101EB000E3074091E4075091E50780911E0190915E
:101EC0001F01A0912001B091210182179307A4075F
:101ED000B5079CF48091E2079091E307A091E40795
:101EE000B091E5070597A109B1098093E2079093A6
:101EF000E307A093E407B093E507862F992701969F
:101F00002091260130912701821793072CF48091AC
:101F100010048F7D809310040894811C911C82E72B
:101F200088168BE0980609F040C0882499242091F7
:101F3000EE023091EF022F5F3F4F3093EF0220937C
:101F4000EE028091EC029091ED0201969093ED02E9
:101F50008093EC02832F9927682F8EE090E00E94F7
:101F6000C6308091EE029091EF029070682F8FE062
:101F700090E00E94C6308091EC029091ED02892F92
:101F80009927682F8AE090E00E94C6308091EC0289
:101F90009091ED029070682F8BE090E00E94C63027
:101FA00084E190E00E94691A6C010E9494760E947C
:101FB000AC7D71107A94772039F40E94587688238A
:101FC00019F08CE0782E3ECD80911C03882309F017
:101FD00039CD0E94687136CD1F920F920FB60F92C5
:101FE00011248F939F93EF93FF938091080188238F
:101FF000E1F480910C0390910D03019690930D03F1
:1020000080930C03FC01E354F94FE081ED3019F0AB
:102010008C3D910539F410920D0310920C0381E070
:1020200080930801E093C60004C010920D03109243
:102030000C03FF91EF919F918F910F900FBE0F9026
:102040001F9018951F920F920FB60F9211242F9385
:102050003F934F935F936F937F938F939F93AF9330
:10206000BF93CF93EF93FF9390E08091F202813082
:1020700029F48091C6008093CE00D1C08091F202F5
:10208000823029F48091C6008093DF05C8C080911A
:10209000C60080930403509112035C3D10F09093AE
:1020A0001303809104038D3009F06AC080911303FB
:1020B000823009F065C090931303852F99278152D0
:1020C0009A4FFC013297408120910E0330910F030B
:1020D000241B3109DC0111978C91281B3109C9019E
:1020E0009F7090930F0380930E0346E0969587951B
:1020F0004A95E1F7982F935C909310032F733070FB
:10210000235C209311038081981729F48C91281760
:1021100011F491E006C090E0809101038F5F8093FD
:10212000010380910303882309F079C0992309F4FE
:1021300076C081E080930303580F50930003515001
:10214000E52FFF27E152FA4F8DE080838091E10572
:10215000823509F064C0C0914804CC2309F05FC007
:102160000E94E72588E190E02CE00FB6F894A8954E
:10217000809360000FBE20936000C0931B034FC08C
:1021800020911303822F992781309105F9F0823035
:1021900091051CF4892B21F040C0029711F13DC03C
:1021A00080910403833239F480910303882319F466
:1021B00081E080931303809104038093DF0581E025
:1021C0008093120380910403992722C02F5F2093EC
:1021D0001303E52FFF27E152FA4F80910403808318
:1021E00009C0E52FFF27E152FA4F80910403808355
:1021F0005C3D20F45F5F5093120302C01092130302
:102200002091040380910E0390910F03820F911D82
:1022100090930F0380930E0302C010921303FF915B
:10222000EF91CF91BF91AF919F918F917F916F91DE
:102230005F914F913F912F910F900FBE0F901F9084
:102240001895AC01A0E0B0E09D01A817B90748F4CB
:10225000EDEBF6E08191280F311D1196A417B5071B
:10226000C8F33F70FD01E354F94FC90156E096955C
:1022700087955A95E1F7835C80831196FD01E354BD
:10228000F94F2F733070822F835C8083A254B94F33
:102290008DE08C93109208018091BD068093C6005A
:1022A0000895A0E0B0E0E7E5F1E10C9419A02C85D9
:1022B0009D850E85BB2483E28093BD069F59909334
:1022C000BE062093BF0633E0E32EF12C002309F471
:1022D0009EC0CF84D888BE016D5E7F4FA989BA8920
:1022E0000150109709F493C01097B9F0F601EB0D67
:1022F000F11DB3949081119791F4002349F1FB01F2
:102300006E5F7F4FDB01C080D1806E5F7F4F0D908D
:10231000BC91A02DBB24015002C090E019C01097C1
:10232000B9F0F601EB0DF11DB3944081119791F4D2
:10233000002341F1FB016E5F7F4FDB01C080D18044
:102340006E5F7F4F0D90BC91A02DBB24015002C049
:1023500040E018C01097B1F0F601EB0DF11DB394F9
:102360001081119781F4002371F0FB013296DB019B
:10237000CD90DC90BF016E5F7F4FA081B181BB2407
:10238000015001C010E0F701E354F94F892F869501
:102390008695835C80830894E11CF11CF701E3546B
:1023A000F94F892F99278370907024E0880F991F27
:1023B0002A95E1F755279A0194E0369527959A9545
:1023C000E1F7822B835C80830894E11CF11CF70108
:1023D000E354F94F4F705070440F551F440F551F71
:1023E000812F992726E0969587952A95E1F7842BEA
:1023F000835C80830894E11CF11CF701E354F94FDE
:102400001F73135C10830894E11CF11C6ACFC70191
:102410000E942111E9E00C9435A0A3E07A2F4091AD
:1024200000034650442309F458C0E72FFF27E15228
:10243000FA4F80818D537F5FE72FFF27E152FA4FDC
:1024400020812D537F5FE72FFF27E152FA4F308124
:102450003D537F5FE72FFF27E152FA4F60816D53B5
:102460007F5F9927880F991F880F991F522F5295C8
:102470005F70582B822F99278F709070F4E0880F2F
:10248000991FFA95E1F7232F26952695282B832F60
:10249000992783709070E6E0880F991FEA95E1F71D
:1024A000682B41504F3FC9F0EA2FFF27E152FA4F06
:1024B0005083AF5F41504F3F81F0EA2FFF27E15239
:1024C000FA4F2083AF5F41504F3F39F0EA2FFF278B
:1024D000E152FA4F6083AF5FA5CF82EE95E0909313
:1024E000FF028093FE02A350A093FD020895A2E094
:1024F000B0E0EDE7F2E10C941FA080910303882384
:1025000009F412C40E940D128091E005823609F090
:10251000DEC28091E10599278037910509F4AFC0AB
:1025200081379105C4F48A36910509F43BC28B3694
:10253000910544F48B34910571F18636910509F4C7
:1025400064C1C5C28D36910509F469C08E36910506
:1025500009F44DC0BCC28437910541F1853791051E
:102560004CF48137910509F491C08337910509F442
:10257000E4C0ADC28737910509F4D6C1883791050B
:102580002CF48537910509F492C1A1C289379105D0
:1025900009F477C19CC2E091FE02F091FF028081B4
:1025A0009181909391018093900191C28091000359
:1025B000A091FE02B091FF02853140F080E1EAEB8C
:1025C000F5E00D9001928A95E1F70DC08D919D91F6
:1025D0000D90BC91A02D8093BA059093BB05A0935C
:1025E000BC05B093BD0580EF8093FB024BC080918A
:1025F00008018823E1F38DE490E09F938F9381ECB1
:1026000098E09F938F9381E08F938F938EE48F93C5
:102610000E9451118DB79EB707968DBF58C2A091E9
:10262000FE02B091FF021C91113081F48DE4E1ECC7
:10263000F8E00D9001928A95E1F70E94D931198353
:102640008091B6058F7E8093B60501C01982809176
:1026500008018823E1F381E090E09F938F93CE01FE
:1026600001969F938F9381E08F938F938DE48F9347
:102670000E945111ADB7BEB71796ADBF28C281E019
:10268000809306038FEF8093060121C28091480456
:10269000882309F01CC2E091FE02F091FF02E08164
:1026A0008E2F8A508A3058F48983882311F481E070
:1026B00003C0863010F085E0898361E00EC08E2F64
:1026C00084518A3070F48983882311F481E003C037
:1026D000863010F085E0898360E089810E945B325A
:1026E00012C0E983EF3F19F40E943C32898389814B
:1026F000882311F481E003C0863010F085E08983DF
:1027000089810E94DC30809108018823E1F380E810
:1027100090E09F938F9380E498E09F938F9381E064
:1027200090E09F938F93CE0101969F938F9382E0C9
:102730008F9381E08F9381E52DC12091FE0230912E
:10274000FF02D9018C918150853008F045C0F90114
:102750008181813609F040C0809148048823E1F5E9
:102760002F5F3F4F80E8E0E4F8E0D9010D9001923F
:102770008A95E1F7F90182910E944931809181089F
:102780009927AA27BB27BC01CD0124EC39E040E002
:1027900050E00E94819FDC01CB01809388019093DF
:1027A0008901A0938A01B0938B01809182089927B7
:1027B000AA27BB27BC01CD010E94819FDC01CB0170
:1027C0008093840190938501A0938601B093870143
:1027D0000E943C32898301C01982809108018823BC
:1027E000E1F381E090E09F938F93CE0101969F9358
:1027F0008F9381E08F938F9383E58F930E94511184
:102800008DB79EB707968DBF2BC080914804882353
:1028100009F05DC1E091FE02F091FF02E0818E2F90
:102820008150853018F48E2F0E94DC300E943C329B
:102830008983809108018823E1F381E090E09F93F0
:102840008F93CE0101969F938F9381E08F938F9307
:1028500086E48F930E945111ADB7BEB71796ADBFF6
:1028600010914804112341F46EE670E089810E94C2
:10287000243C812F0E94630A809167080E94B09ACD
:1028800026C119822981A091FE02B091FF02E8E7DA
:10289000F9E08D91992787FD909593A382A3822FCC
:1028A0008F5F8983282F32968C3098F310C1E09186
:1028B000FE02F091FF0280810E94FB378A83882309
:1028C00019F481E0898301C019828091080188236D
:1028D000E1F388E090E09F938F938FE099E09F93DE
:1028E0008F9321E030E03F932F938091FE029091EF
:1028F000FF029F938F933F932F93CE0102969F9356
:102900008F933F932F93CE01820F931F9F938F93AB
:1029100084E08F9381E08F9385E58F930E9451111E
:10292000EDB7FEB773963CC08091FD02893008F484
:10293000CEC02091FE023091FF022F5F3F4F88E012
:10294000AFE0B9E0F90101900D928A95E1F7D90164
:102950008E910E944E378A83882319F481E08983FF
:1029600001C01982809108018823E1F321E030E061
:102970003F932F93CE0102969F938F933F932F9374
:10298000CE01820F931F9F938F9382E08F9381E0FC
:102990008F9387E58F930E945111EDB7FEB73B9659
:1029A000EDBF95C080914804882309F090C00E9433
:1029B000679A8983823019F0843009F088C020E456
:1029C00030E0F8948091C1008F738093C1008091B2
:1029D000C9008F738093C9008091C100877E809366
:1029E000C1008091C900877E8093C9008091C80092
:1029F00087FF03C08091CE00F9CF8091C00087FF90
:102A000003C08091C600F9CFE091FE02F091FF0271
:102A1000E081E13021F482E08093F2022EC0E436BE
:102A200011F421E830E081E08093F202832F9927AE
:102A30008093CD002093CC008091CD008093C50081
:102A40008091CC008093C4008091CA008F7D8093D8
:102A5000CA008091CA008F7E8093CA008091C9000D
:102A60008B7F8093C9008091CA0084608093CA00E4
:102A70008091CA0082608093CA008091CA00877FDB
:102A80008093CA008091C200877F8093C2008091AA
:102A9000C9008E7F8093C9008091C10088618093B6
:102AA000C1008091C90088618093C9008091C100F4
:102AB00080688093C1008091C90080688093C900BC
:102AC00010926E0010926F001092700078948091B6
:102AD000E10599278436910509F4BBC08536910537
:102AE000ACF48136910509F46FC0823691052CF45F
:102AF0008B34910509F45DC00FC18236910509F44C
:102B000070C08336910509F47FC006C18C369105EB
:102B100009F4EDC08D3691054CF48736910509F422
:102B2000F8C08836910509F4B2C0F6C08437910523
:102B300029F08637910509F4E8C0EEC080910003C2
:102B4000A091FE02B091FF02803140F080E1EAEBFB
:102B5000F5E00D9001928A95E1F70DC08D919D9160
:102B60000D90BC91A02D8093BA059093BB05A093C6
:102B7000BC05B093BD05809108018823E1F31F9245
:102B8000809105018F9384E58F930E9451118AEF04
:102B90008093FB028FEF8093060180EA9FE00E9402
:102BA000691A9093F4028093F3020F900F900F90A4
:102BB000B3C0E091FE02F091FF0280819181909379
:102BC000910180939001A8C0E091FE02F091FF0274
:102BD000808180930701803298F08FE18093070114
:102BE0000FC0A091FE02B091FF028BE0E2EDF5E094
:102BF0000D9001928A95E1F78091DB058093DB07C8
:102C00008FEF8093060188C08091F7029091F802BF
:102C1000892B89F4E091FE02F091FF02E081EE231E
:102C200051F08AE0E89FC00111240E94691A909334
:102C3000AD058093AC05E091FE02F091FF0290811A
:102C40008AE0989FC00111249093F8028093F702C4
:102C500015C08FEF80930601E091FE02F091FF0214
:102C600090818AE0989FC00111249093FA0280938A
:102C7000F902892B19F081E08093080380EA9FE034
:102C80000E94691A9093F4028093F30245C08FEF7B
:102C900080930601E091FE02F091FF02908197FD82
:102CA00008C082E0809305031092F6021092F502AC
:102CB0001AC0909580916303892B8093630391815F
:102CC0008AE0989FC00111249093F6028093F50248
:102CD00084E08093050380EA9FE00E94691A909344
:102CE000F4028093F30281E08093090315C08FEF13
:102CF00080930601E091FE02F091FF0280818093B3
:102D0000640381E080930A0307C081E08093070396
:102D100003C081E080930B03109203031092FF0223
:102D20001092FE021092FD02E3E0CE5F0C943BA0F5
:102D3000982F8091C00085FFFCCF9093C600089526
:102D40000F931F9388E18093C1008091C00082603F
:102D50008093C0008091C10080688093C100809101
:102D6000C10080648093C10000E010E00093C500C2
:102D70008AE290E08093C4008091F9029091FA0277
:102D80000E94691A9093AF058093AE058CED90E098
:102D90000E94691A9093DE058093DD0582E080939E
:102DA000B0058093B1051092B4058BE08093B20515
:102DB0001092B3051092B805809103018093B70576
:102DC0001093FF020093FE021092FD021F910F91DB
:102DD0000895A0E1B0E0EFEEF6E10C941EA0809122
:102DE0000801882309F489C28091F3029091F402CA
:102DF0000E94721A882361F01092F6021092F50276
:102E00001092FA021092F9021092F8021092F70250
:102E10008091F5029091F602892B41F08091BB06DA
:102E20009091BC060E94721A882329F480910903AC
:102E3000882309F460C080910801882309F45BC0ED
:102E4000809105030FEE17E08430A8F00E94FD2565
:102E500080E590E09F938F931F930F9381E08F9372
:102E60008F9388E48F930E9451112DB73EB7295F4D
:102E70003F4F2DBF34C01092650386E694E09F93C8
:102E80008F9380EF95E29F938F93E0919C05F09153
:102E90009D05099584E190E09F938F931F930F9375
:102EA00081E090E09F938F9385E093E09F938F93D1
:102EB00082E08F9381E08F9388E48F930E94511179
:102EC00080910503982F8F5F809305032DB73EB740
:102ED000215F3F4F2DBF943010F010920503809179
:102EE000F5029091F6020E94691A9093BC068093B5
:102EF000BB061092090380910A03882351F1809147
:102F00000801882331F10E94FD2580E590E09F9320
:102F10008F938FEE97E09F938F9321E030E03F9364
:102F20002F9388E291E09F938F933F932F9384E6B2
:102F300093E09F938F9383E08F9381E08F938CE452
:102F40008F930E94511110920A038DB79EB70F966E
:102F50008DBF809107038823D1F0809108018823D9
:102F6000B1F08AE090E09F938F9380EB95E09F9380
:102F70008F9381E08F938F9386E58F930E945111F9
:102F8000109207032DB73EB7295F3F4F2DBF8091A9
:102F90000B038823D9F0809108018823B9F08BE0D6
:102FA00090E09F938F9382ED95E09F938F9381E0C4
:102FB0008F93809105018F9387E48F930E94511125
:102FC00010920B038DB79EB707968DBF8091F902C3
:102FD0009091FA02892B41F08091AE059091AF0556
:102FE0000E94721A882321F480910803882341F1FA
:102FF00080910801882321F10E942E3B82E490E019
:103000009F938F9389E997E09F938F9381E08F93AC
:103010008F9384E48F930E945111109208032DB76F
:103020003EB7295F3F4F2DBF8091F9029091FA0280
:10303000009731F00E94691A9093AF058093AE0516
:103040008091F7029091F802892B09F497C0809142
:10305000AC059091AD050E94721A882309F48EC0C8
:1030600080910801882309F489C08091840A909195
:10307000850A90939F0580939E058091860A909182
:10308000870A9093A1058093A0052091660A30914C
:10309000670A4091680A5091690ADA01C90163E040
:1030A000880F991FAA1FBB1F6A95D1F7820F931F24
:1030B000A41FB51F820F931FA41FB51F20914201AB
:1030C000309143014091440150914501BC01CD0133
:1030D0000E94F59F3093A3052093A20580916B0475
:1030E00090916C04A0916D04B0916E0449E0B59587
:1030F000A795979587954A95D1F78093A4058091D8
:10310000670490916804A0916904B0916A0439E061
:10311000B595A795979587953A95D1F78093A5058D
:103120008091730490917404A0917504B091760419
:1031300029E0B595A795979587952A95D1F780931E
:10314000A6058EE090E09F938F938EE995E09F9384
:103150008F9381E08F938F9383E48F930E9451111B
:103160008091F7029091F8020E94691A9093AD0540
:103170008093AC058DB79EB707968DBF80910701F0
:103180008F3F79F1992704E0880F991F0A95E1F79D
:103190008A599D4F40E150E0BC01CE0101960E944A
:1031A000CB9D80E190E09F938F93CE0101969F93FA
:1031B0008F9381E090E09F938F9387E091E09F93BE
:1031C0008F9382E08F9381E08F9381E48F930E94AD
:1031D00051118FEF809307012DB73EB7255F3F4F09
:1031E0002DBF8091DB078823C9F0809108018823D7
:1031F000A9F081E090E09F938F938BED97E09F93F0
:103200008F9381E08F938F9382E48F930E9451116B
:103210001092DB078DB79EB707968DBF809106038E
:103220008823D1F0809108018823B1F086E490E0F2
:103230009F938F9388E799E09F938F9381E08F937B
:103240008F9380E58F930E945111109206032DB742
:103250003EB7295F3F4F2DBF8091DD059091DE0580
:103260000E94721A882309F448C0809108018823BB
:1032700009F443C08091840A9091850A9093CB050C
:103280008093CA058091860A9091870A9093CD0514
:103290008093CC05809125048093CE0580912404F1
:1032A0008093CF0588E090E09F938F938AEC95E020
:1032B0009F938F9381E08F9383E08F938BE68F931F
:1032C0000E9451118091D0052DB73EB7295F3F4F25
:1032D0002DBF853018F086E08093D0058091A40141
:1032E000882319F483E690E002C087EE93E00E9401
:1032F000691A9093DE058093DD05E4E0C05F0C94CD
:103300003AA01F920F920FB60F9211242F933F9362
:103310005F936F937F938F939F93AF93BF93EF933D
:10332000FF9380911C03882329F080911C03815016
:1033300080931C0380913D05882319F08150809370
:103340003D05809124038150809324038F3F09F031
:1033500051C089E08093240380912203909123033C
:1033600001969093230380932203809112018F5F33
:10337000817080931201882349F480912103843065
:1033800028F4809121038F5F80932103349903C037
:1033900081E080931A0380911D0390911E03892B75
:1033A00011F180911D0390911E030B9750F08091B5
:1033B0001D0390911E030A9790931E0380931D0393
:1033C00004C010921E0310921D0380911D03909162
:1033D0001E0320910B0130910C0182239323892B32
:1033E00041F0479A07C08FEF9FEF90930C018093B5
:1033F0000B01479880911A03882309F45AC0209141
:10340000A401222309F055C08091560A83FF51C0C0
:1034100086B19927FC01E071F07084FF13C08091A0
:103420001F039091200301969093200380931F0324
:1034300080911F0390912003895E9340D0F12093E7
:103440001A0337C080911F0390912003892B69F1E3
:1034500080911F03909120038A56914030F580910E
:103460001F039091200369E270E00E94AC9F80915D
:103470001F0390912003860F971F90932003809342
:103480001F0380911F03909120030B9750F08091B0
:103490001F03909120030A979093910180939001CC
:1034A00004C0F0939101E0939001109220031092D8
:1034B0001F03FF91EF91BF91AF919F918F917F91EA
:1034C0006F915F913F912F910F900FBE0F901F90C2
:1034D00018952091220330912303280F391FC90129
:1034E000019608952091220330912303821B930BB0
:1034F000892F99278695807490700895CF93DF93D4
:103500000E94691AEC01CE010E94721A8823D9F335
:10351000DF91CF910895CF93DF930E94691AEC0158
:1035200009C080911801882329F0909318018FEC2D
:1035300080937A00CE010E94721A982F882389F313
:10354000DF91CF9108959FB7F8945F983E9A469A7D
:103550008091B0008F708093B0008091B000836044
:103560008093B0008091B1008B738093B100809103
:10357000B1008B608093B1001092B2008FEF809306
:10358000B3008091B00080688093B000809170009B
:103590008A7F8093700080917000826080937000B9
:1035A0009FBF08958AE090E00E94691A9093DD071A
:1035B0008093DC0782E085BD83EB84BD8FEF88BDFF
:1035C00084EB87BD86E086BD80916E00816080932C
:1035D0006E0008958091B10820916F0182FF30C084
:1035E000909170088CE3989FB001112490916F081E
:1035F00080E5989FA0011124922F905897FD9D5F20
:103600009595959586E09802C001112420910901B5
:1036100030910A01281B390B30930A0120930901CC
:10362000421753072CF050930A0140930901089563
:103630002617370784F070930A01609309010895F3
:10364000822F992736E0880F991F3A95E1F79093DA
:103650000A01809309010895EF92FF920F931F933F
:10366000CF93DF9380917708E82FFF27E85BFE4F29
:103670009681C08180911101813009F026C180912D
:10368000B30887FF05C0C0E0D0E0E0E0F0E046C04E
:10369000892F992787FD9095A92FB92F2091A304F1
:1036A0003091A4044091A5045091A604BC01CD0121
:1036B0000E94819F97FF04C061587F4F8F4F9F4F9B
:1036C0007B018C0187E015950795F794E7948A951F
:1036D000D1F78C2F992787FD9095A92FB92F20918D
:1036E0009B0430919C0440919D0450919E04BC0128
:1036F000CD010E94819F97FF04C061587F4F8F4F7B
:103700009F4FB7E09595879577956795BA95D1F7CF
:10371000F801E701C61BD70BE80BF90B2091230535
:1037200030912405C901A3E0880F991FAA95E1F7FC
:10373000821B930BAA2797FDA095BA2FC81BD90B04
:10374000EA0BFB0B80916D019927AA27BB27BC01CF
:10375000CD019E01AF010E94819F97FF04C061507F
:103760007E4F8F4F9F4FFC01EB0179E0F595E79578
:10377000D795C7957A95D1F71091B1086091090155
:1037800070910A0112FF05C07093100160930F0140
:1037900018C040910F015091100180917608282F98
:1037A0003327CB01841B950BB9010E94C09F8091E8
:1037B0000F0190911001860F971F90931001809335
:1037C0000F0110FF14C080910F019091100197FD1F
:1037D0000F9664E0959587956A95E1F7AA2797FD7E
:1037E000A095BA2FC80FD91FEA1FFB1F15C08091E3
:1037F0000F019091100197FD0F9654E095958795D4
:103800005A95E1F7AA2797FDA095BA2F8C1B9D0B1F
:10381000AE0BBF0BFD01EC012091AA08222321F180
:1038200033278091160390911703829FA001839FF5
:10383000500D929F500D1124CA01AA2797FDA09503
:10384000BA2F8C0F9D1FAE1FBF1F2F5F3F4F442706
:1038500037FD4095542FBC01CD010E94F59F309358
:1038600017032093160304C0D0931703C0931603C5
:1038700080916F08282F3327220F331F220F331F09
:103880008091160390911703821793077CF0809123
:103890007008282F3327220F331F220F331F8091E8
:1038A0001603909117032817390724F43093170350
:1038B0002093160380910301843108F4FDC08091A8
:1038C00011018F5F80931101F9C0892F992787FD1E
:1038D0009095A92FB92F20919B0430919C04409181
:1038E0009D0450919E04BC01CD010E94819F97FFD1
:1038F00004C061587F4F8F4F9F4F7B018C0187E041
:1039000015950795F794E7948A95D1F78C2F992709
:1039100087FD9095A92FB92F2091A3043091A4047D
:103920004091A5045091A604BC01CD010E94819F45
:103930009B01AC0197FF04C021583F4F4F4F5F4F91
:10394000C7E05595479537952795CA95D1F72E0D20
:103950003F1D401F511F80916C019927AA27BB274B
:10396000BC01CD010E94819F97FF04C061507E4F32
:103970008F4F9F4FFC01EB01B9E0F595E795D79587
:10398000C795BA95D1F780916E019927A6E0880F67
:10399000991FAA95E1F740910D0150910E012091D8
:1039A00076083327841B950BB9010E94C09F809134
:1039B0000D0190910E01860F971F90930E01809339
:1039C0000D018091B10881FF14C080910D0190918B
:1039D0000E0197FD0F9674E0959587957A95E1F71E
:1039E000AA2797FDA095BA2FC80FD91FEA1FFB1F62
:1039F00015C080910D0190910E0197FD0F9664E026
:103A0000959587956A95E1F7AA2797FDA095BA2F16
:103A10008C1B9D0BAE0BBF0BFD01EC012091AB0885
:103A2000222321F133278091140390911503829F63
:103A3000A001839F500D929F500D1124CA01AA2707
:103A400097FDA095BA2F8C0F9D1FAE1FBF1F2F5F34
:103A50003F4F442737FD4095542FBC01CD010E94B4
:103A6000F59F309315032093140304C0D0931503DE
:103A7000C093140380917308282F3327220F331F1C
:103A8000220F331F8091140390911503821793071F
:103A90007CF080917408282F3327220F331F220FC8
:103AA000331F80911403909115032817390724F4CC
:103AB000309315032093140310921101E6E0CDB763
:103AC000DEB70C9438A01F920F920FB60F921124FC
:103AD0002F933F934F935F938F939F93EF93FF9316
:103AE0008091030190912503843108F04CC0992303
:103AF00009F029C18091B00086FF24C08091B000F8
:103B00008F7B8093B00080911603909117038755A7
:103B10009E4F909319038093180325E08D3D9207E3
:103B200018F08CED95E005C08757914030F487E799
:103B300091E090931903809318038091180390915A
:103B40001903C2C08091B00080648093B00080915E
:103B50007508282F33278DED96E0289FA001299F17
:103B6000500D389F500D1124CA0120912603309129
:103B70002703821B930B909319038093180381E012
:103B800080931101DDC0992309F0DDC08091B00060
:103B900086FF9FC08091B0008F7B8093B000E09142
:103BA000280320917508EE23D9F433278DED96E094
:103BB000289FA001299F500D389F500D1124CA0144
:103BC0002091260330912703821B930B90931903B6
:103BD000809318031092270310922603469AB0C0D0
:103BE0002E1738F48AE090E090931903809318031D
:103BF000A7C089EA93E090931903809318038E2F4E
:103C0000992783309105D9F08430910534F48130BF
:103C1000910549F0029761F020C08430910591F040
:103C2000059799F01AC0809116039091170304C06C
:103C3000809114039091150387559E4F1DC080916C
:103C4000310A05C080910A0A02C080913A0A992778
:103C5000880F991F880F991FEFCFFF27EE0FFF1FC7
:103C6000E858F64F20813181220F331F80911803CD
:103C700090911903820F931F909319038093180357
:103C8000809118039091190355E08D3D950718F028
:103C90008CED95E005C08757914030F487E791E0BF
:103CA00090931903809318032091180330911903FE
:103CB0002C5B304030931903209318038091260326
:103CC00090912703820F931F9093270380932603DD
:103CD00037C08091B00080648093B0008CEB90E09E
:103CE00090931903809318038091260390912703E2
:103CF00084549F4F909327038093260380911B0346
:103D0000882321F080914904882321F480911B03AA
:103D1000823011F4469801C0469A809128038F5F43
:103D200080932803282F33278091750899270196BF
:103D3000821793072CF481E08093110110922803DD
:103D400081E080932503209118033091190341E00D
:103D50002F37340730F08FEF8093B3002F5F304060
:103D60000FC02F3F3105C9F0C0F0A9014F5F50408F
:103D70004F37510550F480E88093B300205830400D
:103D8000309319032093180312C08FEF8093B30070
:103D900050931903409318030AC08091180380932D
:103DA000B300109219031092180310922503FF918B
:103DB000EF919F918F915F914F913F912F910F9034
:103DC0000FBE0F901F90189510927C008FEC80937F
:103DD0007A0008958091080460911601709117018E
:103DE00020913503882379F0CB01AA27BB273327FD
:103DF00027FD3095432F532FBC01CD010E94819F99
:103E0000DC01CB0116C084E0660F771F8A95E1F7CD
:103E1000CB01AA27BB27332727FD3095432F532FEC
:103E2000BC01CD010E94819FDC01CB010497A10957
:103E3000B10980932D0390932E03A0932F03B09389
:103E400030030895CF93DF93109235030E94EA1E4A
:103E500083E090E00E94BE30C82FDD27C03FD1052F
:103E600008F42A96C7BD8C2F809588BD86E990E01E
:103E70000E948B1A80911C0190911D0181529340E8
:103E800010F0C0EFD0E0C630D10510F1C7BD8C2FC7
:103E9000809588BD84E690E00E948B1A8BE794E0C1
:103EA0009F938F9388E996E19F938F93E0919C0570
:103EB000F0919D05099580911C0190911D010F9035
:103EC0000F900F900F908152934010F42197DBCF09
:103ED000C093EC076C2F83E090E00E94C630809185
:103EE0004D0880FF0AC08091EC078A508C3D28F075
:103EF0008091B50580648093B50580E180931501BC
:103F0000809108048823E9F080910301873150F4FF
:103F1000CC38D105B0F480EA90E08C1B9D0B6AE1AF
:103F200070E009C0CA3AD10560F48CEB90E08C1BBC
:103F30009D0B63E170E00E94AC9FCB01805F80939A
:103F4000150180911501282F332780911C01909134
:103F50001D01829FA001839F500D929F500D11243F
:103F6000CA01AA27BB2780931E0190931F01A0932B
:103F70002001B09321018CE291E00E948B1ADF9125
:103F8000CF910895EF92FF921F93CF9310E080EDB1
:103F900097E00E94691A7C01CCE8133019F4CB3009
:103FA00008F0C9E010E080914403909145038C5FD4
:103FB000934024F480911B0181500AC080914403F6
:103FC000909145038750944034F080911B018F5F9E
:103FD00080931B0101C011E0809142039091430343
:103FE0008C5F934024F480911A0181500AC0809123
:103FF0004203909143038750944034F080911A011A
:104000008F5F80931A0101C01F5F809140039091E0
:1040100041038C5F934024F48091190181500AC0C0
:10402000809140039091410387509440C4F0809167
:1040300019018F5F8093190113C08DE794E09F935E
:104040008F9388E996E19F938F93E0919C05F0917F
:104050009D0509950F900F900F900F905FC01F5F07
:1040600082E18093700380916A038E7F80936A035C
:1040700085EA8093BC0080911B018A3040F48091D6
:10408000B50581608093B5058AE080931B0180911E
:104090001B01863F40F08091B50581608093B50596
:1040A00085EF80931B0180911A018A3040F4809142
:1040B000B50582608093B5058AE080931A018091EE
:1040C0001A01863F40F08091B50582608093B50566
:1040D00085EF80931A01809119018A3040F4809114
:1040E000B50584608093B5058AE0809319018091BD
:1040F0001901863F40F08091B50584608093B50535
:1041000085EF8093190180917003882339F0C701EE
:104110000E94721A882309F090CFF5CF10921801EF
:104120008FEC80937A00809118018823E1F3CA30E4
:1041300020F48AE090E00E948B1AC15009F02DCF44
:1041400086E490E00E948B1ACF911F91FF90EF9030
:1041500008951F920F920FB60F921124EF92FF92C3
:104160000F931F932F933F934F935F936F937F937F
:104170008F939F93AF93BF93CF93DF93EF93FF936F
:1041800080914D03282F3327442755278F5F809335
:104190004D03F9012231310508F0F2C4EA5BFF4F0B
:1041A0000C9447A0809178009091790046C080914E
:1041B000780090917900B8C1809178009091790051
:1041C0009093510380935003E3C18091AD0490918B
:1041D000AE042091780030917900821B930B90936C
:1041E000DF078093DE078091DE079091DF079093D1
:1041F0005B0380935A03EBC1809178009091790022
:104200002091AF043091B004821B930B9093EB0785
:104210008093EA078091EA079091EB0790935D0302
:1042200080935C03AFC48091540390915503209117
:10423000780030917900820F931F909355038093FB
:10424000540381E0A0C480915203909153032091C4
:10425000780030917900820F931F909353038093DD
:10426000520384E090C48091B20883FF1AC0809109
:104270002601909127019C01220F331F280F391F1F
:1042800040917800509179008BE090E0489FB00118
:10429000499F700D589F700D1124CB016EE170E0A5
:1042A0000FC080912601909127019C01220F331F9E
:1042B000280F391F809178009091790063E070E0B9
:1042C0000E94AC9F260F371F369527953695279568
:1042D000309327012093260185E055C48091780012
:1042E000909179009093E1078093E0078091E00737
:1042F0009091E1074091A9045091AA04841B950B69
:104300006091A804262F332727FD3095821B930B3D
:1043100090933B0380933A0380910804882309F02B
:1043200071C080913A0390913B0302977CF172E057
:104330004E3E57070CF0A7C020914E0330914F031B
:104340002B5F3F4F30934F0320934E032550304057
:104350008091110490911204845F914030F4215FA8
:104360003F4F30934F0320934E0380914E03909123
:104370004F03853691050CF486C04F5F5F4F509315
:10438000AA044093A9048456904037C080913A0310
:1043900090913B038F5F9F4F0CF075C082E04732D6
:1043A00058070CF470C020914E0330914F032550F4
:1043B000304030934F0320934E032B5F3F4F80914B
:1043C000110490911204845F914030F42F503040DA
:1043D00030934F0320934E0380914E0390914F03EF
:1043E0007FEF8C3997070CF04EC0415050405093EE
:1043F000AA044093A9048C599F4F90934F03809334
:104400004E0341C08091260A9091270A8F5C9F41FC
:10441000D4F180913A0390913B030297ACF0209144
:104420004E0330914F03C901019690934F0380933F
:104430004E03895893413CF166301CF46F5F6093E2
:10444000A804275833411BC080913A0390913B0345
:104450008F5F9F4FC4F420914E0330914F03C901E9
:10446000019790934F0380934E0388579C4E5CF4C2
:104470006B3F1CF061506093A80429573C4E309369
:104480004F0320934E0380913A0390913B039C018C
:10449000442737FD4095542F809163049091640424
:1044A000A0916504B0916604820F931FA41FB51FED
:1044B0008093630490936404A0936504B0936604AE
:1044C0002091630430916404409165045091660426
:1044D00057FF04C021503C4F4F4F5F4F6AE0559546
:1044E0004795379527956A95D1F780916304909108
:1044F0006404A0916504B0916604821B930BA40B25
:10450000B50B8093630490936404A0936504B09307
:10451000660430C18091520390915303209178003A
:1045200030917900820F931F90935303809352032D
:1045300010924C032AC3809103018A3071F4809158
:104540007800909179002091500330915103820FAF
:10455000931F01969695879517C0409150035091EF
:104560005103843158F02091780030917900240F64
:10457000351F8FEF97E0821B930B06C08091780068
:1045800090917900840F951F90934103809340038D
:1045900080911401F8C28091AD049091AE042091F5
:1045A000780030917900821B930B9093DF07809302
:1045B000DE078091DE079091DF0720915A0330914A
:1045C0005B03820F931F90933F0380933E03809180
:1045D0001301D9C280917800909179002091AF04A5
:1045E0003091B004821B930B9093EB078093EA0702
:1045F0008091EA079091EB0720915C0330915D0375
:10460000820F931F90933D0380933C03BBC2209184
:104610005403309155038091780090917900280FD0
:10462000391F3093550320935403809103018A303E
:1046300019F4220F331F04C0220F331F220F331F20
:104640003093550320935403209154033091550324
:10465000C90137FD079603E0959587950A95E1F71F
:1046600090934503809344038091560390915703A0
:10467000820F931F97FD0196959587959093570309
:10468000809356032091B9043091BA04821B930B96
:10469000909325018093240120914A0330914B038C
:1046A0008091240190912501280F391F37FF02C006
:1046B0002F5F3F4F3595279530934B0320934A0347
:1046C000C0CD209152033091530380917800909196
:1046D0007900280F391F30935303209352038091A0
:1046E00003018A3019F4220F331F04C0220F331F35
:1046F000220F331F30935303209352032091520310
:1047000030915303C90137FD0796A3E0959587952E
:10471000AA95E1F790934303809342038091580355
:1047200090915903820F931F97FD01969595879558
:1047300090935903809358032091B7043091B804A3
:10474000821B930B909323018093220120914803B5
:10475000309149038091220190912301280F391F44
:1047600037FF02C02F5F3F4F3595279530934903A0
:104770002093480383E007C280910804882309F14D
:1047800080E00E94E8989B01AC0120503F4F4F4FC2
:104790005F4F57FF06C09B01AC0121503D4F4F4F6B
:1047A0005F4F79E055954795379527957A95D1F7DD
:1047B0002093290330932A0340932B0350932C0317
:1047C00010C08091430490914404A0914504B0919D
:1047D00046048093290390932A03A0932B03B0935C
:1047E0002C0310924D0381E08093180180913103D6
:1047F000909132030196909332038093310380911C
:1048000078009091790090931D0180931C01809114
:104810000804882309F472C080911C0190911D0145
:104820007C010027112780912D0390912E03A091E8
:104830002F03B0913003E81AF90A0A0B1B0BE09220
:104840005E03F0925F030093600310936103809115
:104850001501282F33274427552780911E01909159
:104860001F01A0912001B0912101BC01CD010E9446
:10487000F59F80911E0190911F01A0912001B091A0
:104880002101821B930BA40BB50B80931E01909307
:104890001F01A0932001B093210180911E019091EE
:1048A0001F01A0912001B09121018E0D9F1DA01F1D
:1048B000B11F80931E0190931F01A0932001B0931C
:1048C00021018091E2079091E307A091E407B09164
:1048D000E50720911E0130911F0140912001509168
:1048E0002101821B930BA40BB50B8093430490937F
:1048F0004404A0934504B093460444C180911C0134
:1049000090911D01AA27BB27C0915E03D0915F0340
:10491000E0916003F0916103C80FD91FEA1FFB1FEC
:10492000C0935E03D0935F03E0936003F093610351
:10493000809162038F5F80936203803108F422C10B
:1049400080911E0190911F01A0912001B091210141
:104950009C01AD0163E0220F331F441F551F6A9570
:10496000D1F7281B390B4A0B5B0B2C0F3D1F4E1F39
:104970005F1F80912D0390912E03A0912F03B09182
:104980003003281B390B4A0B5B0B57FF04C0295F10
:104990003F4F4F4F5F4F03E055954795379527950C
:1049A0000A95D1F720931E0130931F0140932001F7
:1049B00050932101C091E207D091E307E091E40711
:1049C000F091E50780911E0190911F01A0912001B7
:1049D000B0912101C81BD90BEA0BFB0BC093430418
:1049E000D0934404E0934504F093460420913603A9
:1049F00030913703409138035091390357FF04C079
:104A0000215F3F4F4F4F5F4F14E0559547953795C6
:104A100027951A95D1F78091360390913703A0918D
:104A20003803B0913903821B930BA40BB50B809311
:104A3000360390933703A0933803B09339038091E2
:104A4000360390913703A0913803B09139038C0F4E
:104A50009D1FAE1FBF1F8093360390933703A09313
:104A60003803B09339038091360390913703A091B6
:104A70003803B0913903B7FF03C00F96A11DB11DD4
:104A8000C4E0B595A79597958795CA95D1F72091DC
:104A9000430430914404281B390B64E0213036076D
:104AA0001CF020E034E006C07CEF2030370714F41F
:104AB00020E03CEF809133039091340380913303E5
:104AC0009091340397FF03C0909581959F4FA90162
:104AD000F3E0440F551FFA95E1F78D5B9240C4F067
:104AE00080913303909134039C01E4E0220F331F43
:104AF000EA95E1F7281B390B240F351F37FF02C059
:104B0000215F3F4F74E0359527957A95E1F717C0FF
:104B100080913303909134039C0165E0220F331F91
:104B20006A95E1F7281B390B240F351F37FF02C0A8
:104B3000215E3F4F45E0359527954A95E1F7309343
:104B400034032093330380915E0390915F03A0911F
:104B50006003B0916103B7FF03C00196A11DB11DB1
:104B6000B595A7959795879580935E0390935F037E
:104B7000A0936003B093610388E08093620302C056
:104B800010924D0382E080934C0380914C038093FC
:104B90007C0080914D03882319F08FEC80937A007C
:104BA000FF91EF91DF91CF91BF91AF919F918F9145
:104BB0007F916F915F914F913F912F911F910F9135
:104BC000FF90EF900F900FBE0F901F90189590E2FE
:104BD000EFEEF7E08FE49193815087FFFCCF0895CB
:104BE00090916503903540F4E92FFF27E151F84F8C
:104BF00080839F5F909365030895A0E0B0E0E3E0B9
:104C0000F6E20C941AA02091630320FF0AC0809161
:104C10006403882311F0815002C0809128018093A1
:104C2000640321FF0CC090916403809128019817C0
:104C300019F41092640303C09F5F90936403822F62
:104C4000992780FF04C081FF02C0109264030E9474
:104C5000E72580916403282F332700EF15E2C091E8
:104C60009C05D0919D058A3098F481E1809365037D
:104C70003F932F9384EB94E09F938F931F930F9315
:104C8000FE0109952DB73EB72A5F3F4F2DBF12C0D9
:104C900080E1809365033F932F9389EB94E09F938A
:104CA0008F931F930F93FE0109954DB75EB74A5F2F
:104CB0005F4F4DBF20916403822F9927AA27BB27FE
:104CC000FC01429710F00C94982EE85AFF4F00EF29
:104CD00015E2C0919C05D0919D050C9447A01092BF
:104CE00065038EEB94E09F938F9350EFE52E55E292
:104CF000F52E1F930F93FE01099584E180936503C0
:104D00000F900F900F900F9081E690E09F938F93FC
:104D100082E090E09F938F939F938F938091030104
:104D20006AE00E94A09F892F99279F938F9380917B
:104D300003010E94A09F99279F938F938EEC94E08C
:104D40009F938F931F930F93E0919C05F0919D0586
:104D5000099588E2809365038DB79EB70E968DBF47
:104D600082EC98E09F938F938091010199279F9304
:104D70008F9386EE94E09F938F931F930F93E09110
:104D80009C05F0919D0509958091B6059927EDB791
:104D9000FEB73896EDBFEC01C071D07084FF0AC039
:104DA0008CE38093650384EF94E09F938F931F932C
:104DB0000F9353C790912A05992351F18CE3809367
:104DC0006503892F99279F938F9381E095E09F93A7
:104DD0008F93FF92EF92E0919C05F0919D050995CC
:104DE000DF93CF9390912A0581E1989FC001112410
:104DF000825B944F9F938F93FF92EF92E0919C057B
:104E0000F0919D0509952DB73EB7245F3F4F77C4BC
:104E10009091B505992371F08CE380936503892FF8
:104E200099279F938F9389E095E09F938F93FF92AB
:104E3000EF9204C490916B039923B9F08CE38093B3
:104E40006503892F99279F938F9380E295E09F9325
:104E50008F93FF92EF92E0919C05F0919D0509954B
:104E60008DB79EB706968DBF6CC780913C0190911F
:104E70003D01069730F48CE38093650386E395E06B
:104E8000E8C69091F10A9E3108F05BC78CE38093ED
:104E90006503892F99279F938F9383E495E00AC137
:104EA000109265038091430490914404A0914504BD
:104EB000B0914604BC01CD0125E030E040E050E077
:104EC0000E94F59F3F932F9387E595E09F938F93E3
:104ED0001F930F93FE01099584E1809365032DB71D
:104EE0003EB72A5F3F4F2DBF80913F049091400411
:104EF000A0914104B0914204BC01CD0125E030E015
:104F000040E050E00E94F59F3F932F9384E695E0A8
:104F10009F938F931F930F93E0919C05F0919D05B4
:104F2000099588E2809365034DB75EB74A5F5F4F8E
:104F30004DBF80911C0190911D019F938F9381E73C
:104F400095E09F938F931F930F93E0919C05F091B1
:104F50009D0509958CE3809365038DB79EB70696F2
:104F60008DBF87B599279F938F938EE795E09F9389
:104F70008F931F930F93E0919C05F0919D050995E8
:104F8000EDB7FEB73696EDBF80910804882309F48B
:104F9000D8C689E3809365038BE895E09F938F9350
:104FA0001F930F93E0919C05F0919D0509958DE469
:104FB000809365030F900F900F900F9080911501D3
:104FC00099279F938F938FE895E08CC31092650388
:104FD00082E995E09F938F9340EFE42E45E2F42E13
:104FE0001F930F93FE01099584E1809365030F9051
:104FF0000F900F900F908091A3049091A404A09122
:10500000A504B091A604B7FF04C081509C4FAF4FD8
:10501000BF4F3AE0B595A795979587953A95D1F703
:10502000BF93AF939F938F938FE995E09F938F9357
:10503000FF92EF92E0919C05F0919D05099588E221
:10504000809365034DB75EB7485F5F4F4DBF80915A
:105050009B0490919C04A0919D04B0919E04B7FF85
:1050600004C081509C4FAF4FBF4F2AE0B595A79524
:10507000979587952A95D1F7BF93AF939F938F9379
:105080008EEA95E09F938F93FF92EF92E0919C05BB
:10509000F0919D0509958CE3809365038DB79EB7CC
:1050A00008968DBF8091120A9091130A9F938F9357
:1050B0008DEB95E09F938F93FF92EF92E0919C058B
:1050C000F0919D050995EDB7FEB73696D8C391E0EE
:1050D000F92EC1E0D0E00AE719E09F2D969584E112
:1050E000989FC001112480936503F8018281938108
:1050F0009F938F932196DF93CF9321978081918106
:105100009F938F93DF93CF938CEC95E09F938F9336
:1051100080EF95E29F938F93E0919C05F0919D0520
:1051200009952DB73EB7245F3F4F2DBF32E0F30EF8
:1051300022960C5F1F4F48E04F1578F602C610927A
:10514000650380914208E82FFF27EE0FFF1FE85804
:10515000F64F808191819F938F9380914108E82F32
:10516000FF27EE0FFF1FE858F64F808191819F9334
:105170008F938EED95E09F938F931F930F93FE0176
:10518000099584E1809365038DB79EB708968DBF1E
:1051900080914408E82FFF27EE0FFF1FE858F64FD5
:1051A000808191819F938F9380914308E82FFF27FF
:1051B000EE0FFF1FE858F64F8081918181589F4F75
:1051C0009F938F938EEE95E09F938F931F930F93F2
:1051D000E0919C05F0919D05099588E28093650317
:1051E000EDB7FEB73896EDBF80914608E82FFF2750
:1051F000EE0FFF1FE858F64F8081918181589F4F35
:105200009F938F9380914508E82FFF27EE0FFF1F94
:10521000E858F64F8081918181589F4F9F938F93DB
:105220008EEF95E09F938F931F930F93E0919C05D2
:10523000F0919D0509958CE3809365032DB73EB7EA
:10524000285F3F4F2DBF80914808E82FFF27EE0FC2
:10525000FF1FE858F64F8081918181589F4F9F939F
:105260008F9380914708E82FFF27EE0FFF1FE85824
:10527000F64F8081918181589F4F9F938F938EE04D
:1052800096E09F938F931F930F93E0919C05F0916D
:105290009D0509954DB75EB7485F5F4FD8C1109225
:1052A00065038EE196E09F938F9380EFE82E85E271
:1052B000F82E1F930F93FE01099584E180936503F7
:1052C0000F900F900F900F908091B9049091BA04B5
:1052D0009C0197FF02C0215F3F4F207F821B930BF1
:1052E00097FD0196959587959F938F938091B9042B
:1052F0009091BA0497FD0F96B4E095958795BA956D
:10530000E1F79F938F932091B9043091BA0437FF4E
:1053100002C0295F3F4FA3E035952795AA95E1F795
:105320008091440390914503821B930B9F938F932D
:105330008CE296E09F938F93FF92EF92E0919C0511
:10534000F0919D05099588E2809365038DB79EB71E
:105350000A968DBF8091B7049091B8049C0197FF85
:1053600002C0215F3F4F207F821B930B97FD019668
:10537000959587959F938F938091B7049091B804EA
:1053800097FD0F96E4E095958795EA95E1F79F9351
:105390008F932091B7043091B80437FF02C0295F82
:1053A0003F4F73E0359527957A95E1F78091420359
:1053B00090914303821B930B9F938F938EE396E010
:1053C0009F938F93FF92EF92E0919C05F0919D0542
:1053D00009958CE380936503EDB7FEB73A96EDBF70
:1053E0008091B5049091B60497FD019695958795A7
:1053F0009F938F938091B5049091B60420914003C0
:1054000030914103821B930B9F938F9380E596E02D
:105410009F938F93FF92EF92E0919C05F0919D05F1
:1054200009952DB73EB7285F3F4F69C110926503BC
:105430008FE596E09F938F931F930F93FE0109953D
:1054400084E1809365030F900F900F900F908091EF
:10545000AF049091B0049F938F9380913C039091FF
:105460003D039F938F938CE696E09F938F931F93BA
:105470000F93E0919C05F0919D05099588E280933A
:1054800065034DB75EB7485F5F4F4DBF8091AD0478
:105490009091AE049F938F9380913E0390913F0330
:1054A0009F938F938BE796E09F938F931F930F9318
:1054B000E0919C05F0919D0509958CE3809365032F
:1054C0008DB79EB708968DBF8091A9049091AA04CC
:1054D0009F938F9380913A0390913B039F938F9377
:1054E0008AE896E09F938F931F930F93C0C1109209
:1054F000650380912601909127016AE070E00E9487
:10550000C09F9F938F9380912601909127016AE01D
:1055100070E00E94C09F7F936F9389E996E09F930C
:105520008F931F930F93FE01099584E18093650388
:105530002DB73EB7285F3F4F2DBF8091EB0A90916A
:10554000EC0A6AE070E00E94AC9F9F938F93809179
:10555000EB0A9091EC0A6AE070E00E94AC9F7F93A6
:105560006F938DEA96E09F938F931F930F93E09133
:105570009C05F0919D05099588E2809365034DB7E0
:105580005EB7485F5F4F4DBF8091ED0A9091EE0A84
:105590009F938F9381EC96E09F938F931F930F932C
:1055A000E0919C05F0919D0509958CE3809365033E
:1055B0008DB79EB706968DBF8091EF0A9091F00A45
:1055C0009F938F9381ED96E09F938F931F930F93FB
:1055D00075CD1092650383EE96E09F938F931F9392
:1055E0000F93FE01099588E2809365030F900F9059
:1055F0000F900F908091490499279F938F938CEE81
:1056000096E09F938F931F930F93E0919C05F091E9
:105610009D0509958CE3809365032DB73EB72A5FFE
:105620003F4F2DBF80917709992701979F938F93C3
:105630008CEF96E09F938F931F930F93E0919C05BF
:10564000F0919D0509954DB75EB74A5F5F4F4DBF1D
:1056500078C3109265038CE097E09F938F931F931C
:105660000F93FE01099584E1809365030F900F90DD
:105670000F900F9080919001909191019F938F9343
:1056800084E197E09F938F931F930F93E0919C0584
:10569000F0919D05099588E2809365038DB79EB7CB
:1056A00006968DBF8091120A9091130A9F938F9353
:1056B00082E297E09F938F931F930F93E0919C0555
:1056C000F0919D0509958CE380936503EDB7FEB7D6
:1056D0003696EDBF80916104909162049F938F9301
:1056E00080E397E09F938F931F930F93E0919C0526
:1056F000F0919D0509952DB73EB72A5F3F4F2DBF0D
:1057000020C35AE4C52E54E0D52E20E030E0E90154
:1057100043E0F42EC0936503F60181916F01992750
:105720009F938F9389010F5F1F4F1F930F938EE3FA
:1057300097E09F938F9380EF95E29F938F93E091F3
:105740009C05F0919D0509952DB73EB7285F3F4F09
:105750002DBFFA9464969801F7FEDCCFF2C29EE466
:10576000C92E94E0D92EC0E0D0E08E0183E0F82E5F
:1057700000936503F60181916F0199279F938F93A1
:105780002596DF93CF938BE497E09F938F9380EFE1
:1057900095E29F938F93E0919C05F0919D0509956B
:1057A0002DB73EB7285F3F4F2DBFFA940C5E1F4FB9
:1057B0002497F7FEDDCFC5C21092650388E597E018
:1057C0009F938F93B0EFEB2EB5E2FB2E1F930F93B9
:1057D000FE01099584E1809365030F900F900F906F
:1057E0000F9080916F0199279F938F9380E697E0A8
:1057F0009F938F931F930F93E0919C05F0919D05CC
:10580000099588E2809365034DB75EB74A5F5F4FA5
:105810004DBF809116039091170397FD03969595C0
:105820008795959587959F938F938EE697E09F93A5
:105830008F93FF92EF92E0919C05F0919D05099561
:105840008CE3809365038DB79EB706968DBF8091DC
:10585000700899279F938F9380916F0899279F9342
:105860008F938CE797E09F938F93FF92EF92E09155
:105870009C05F0919D050995EDB7FEB73896EDBFF3
:1058800060C2109265038AE897E09F938F93F0EFD0
:10589000CF2EF5E2DF2E1F930F93FE0109950F9097
:1058A0000F900F900F90C7E1D9E000E010E0E2E028
:1058B000FE2E802F8C5E809365038B8D99278F77CA
:1058C00090709F938F938B8999278F7790709F9378
:1058D0008F938B8599278F7790709F938F938B8170
:1058E00099278F7790709F938F938AE997E09F9382
:1058F0008F93DF92CF92E0919C05F0919D050995E1
:105900002DB73EB7245F3F4F2DBFFA940C5E1F4F5B
:10591000A096F7FECECF15C2109265038BEA97E0F2
:105920009F938F9370EFC72E75E2D72E1F930F931F
:10593000FE0109950F900F900F900F90C7E1D9E0ED
:1059400000E010E062E0F62E802F8C5E809365030D
:105950008F8D992787FD90959F938F938F89992796
:1059600087FD90959F938F938F85992787FD9095BD
:105970009F938F938F81992787FD90959F938F9306
:105980008AEB97E09F938F93DF92CF92E0919C05F3
:10599000F0919D0509954DB75EB7445F5F4F4DBFD0
:1059A000FA940C5E1F4FA096F7FECECFCAC110929C
:1059B00065038BEC97E09F938F9350EFC52E55E2D4
:1059C000D52E1F930F93FE01099587E480936503FD
:1059D0000F900F900F900F9086ED97E09F938F930D
:1059E0001F930F93E0919C05F0919D050995FF246D
:1059F0000F900F900F900F90C0E0D0E08E01802F9D
:105A00008C5E809365038C2F8D5F0E94907D9F93A9
:105A10008F938C2F8E5F0E94907D9F938F938C2FFE
:105A20008F5F0E94907D9F938F938C2F0E94907D1B
:105A30009F938F9380EE97E09F938F93DF92CF9207
:105A4000E0919C05F0919D0509959E012C5F3F4FCB
:105A500080913F089927EDB7FEB73C96EDBF281718
:105A600039070CF06EC1F3940C5E1F4FE901F2E0B0
:105A7000FF1528F666C11092650381EF97E09F93AA
:105A80008F9340EFE42E45E2F42E1F930F93FE0117
:105A9000099584E1809365030F900F900F900F900C
:105AA00080913209881F8827881F97E0899FC0014D
:105AB00011248D969F938F9380912A09881F8827A0
:105AC000881F96E0899FC00111248D969F938F9324
:105AD00080912209881F8827881F95E0899FC0012F
:105AE00011248D969F938F9380911A09881F882780
:105AF000881F9927880F991F880F991F8D969F934C
:105B00008F9380E098E09F938F931F930F93E09182
:105B10009C05F0919D05099588E2809365032DB75A
:105B20003EB7245F3F4F2DBF80915209881F8827C1
:105B3000881F9BE0899FC00111248D969F938F93AE
:105B400080914A09881F8827881F9AE0899FC00191
:105B500011248D969F938F9380914209881F8827E7
:105B6000881F99E0899FC00111248D969F938F9380
:105B700080913A09881F8827881F992723E0880F7A
:105B8000991F2A95E1F78D969F938F9384E198E072
:105B90009F938F931F930F93E0919C05F0919D0528
:105BA00009958CE3809365034DB75EB7445F5F4F03
:105BB0004DBF80915A09881F8827881F9CE0899FC4
:105BC000C00111248D969F938F9388E298E09F9354
:105BD0008F931F930F93E0919C05F0919D0509957C
:105BE00080916209EDB7FEB73696EDBF87FF12C010
:105BF00080E48093650389E398E09F938F931F93DC
:105C00000F93E0919C05F0919D0509950F900F90E1
:105C10000F900F9080916A0987FF12C084E48093EF
:105C200065038CE398E09F938F93FF92EF92E0914E
:105C30009C05F0919D0509950F900F900F900F9086
:105C40008091720987FF7DC088E4809365038FE3AC
:105C500098E09F938F93FF92EF92E0919C05F091D3
:105C60009D0509950F900F900F900F906AC01092AC
:105C7000650382E498E09F938F931F930F93FE0137
:105C8000099584E1809365030F900F900F900F901A
:105C90008091EC029091ED029F938F9380E598E0C4
:105CA0009F938F931F930F93E0919C05F0919D0517
:105CB000099588E2809365032DB73EB72A5F3F4F71
:105CC0002DBF8091EE029091EF029F938F938DE50F
:105CD00098E09F938F931F930F93E0919C05F09111
:105CE0009D05099589E4809365034DB75EB74A5FCA
:105CF0005F4F4DBF8AE698E09F938F931F930F935A
:105D0000E0919C05F0919D050995809163030F90AA
:105D10000F900F900F9083FF14C01092EF0210921B
:105D2000EE0260E070E08EE090E00E94D73009C0A3
:105D300080912801281719F42150209328011092EE
:105D4000640310926303E8E0CDB7DEB70C9436A08D
:105D5000F999FECF92BD81BDF89A80B59927089533
:105D6000F999FECF1FBA92BD81BD60BD0FB6F89400
:105D7000FA9AF99A0FBE08954AEA20E030E0261711
:105D8000370740F4FC018191480F2F5F3F4F2617E2
:105D90003707C8F3842F99270895EAEA40E050E0D6
:105DA0004617570778F49C01F999FECF32BD21BD03
:105DB000F89A80B5E80F4F5F5F4F2F5F3F4F461750
:105DC000570790F38E2F9927089581E08093430819
:105DD00082E08093420883E08093410884E08093CE
:105DE000440885E08093450886E08093460887E074
:105DF0008093470888E08093480889E080934908A9
:105E00008AE080934A088BE080934B088CE0809373
:105E10004C08089581E6809340088CE0E4EBF8E0BC
:105E200011928A95E9F780910301843150F08AE05C
:105E300080936008109284088BE180935C088EE464
:105E40000AC083E08093600880E2809384088EE13A
:105E500080935C0885E5809381088093820880E2C6
:105E6000809383081092B0088AE680934D0882E7F9
:105E70008093B20880E58093B30886E0809367083A
:105E80001092A4081092A10838E030935A0886EEC8
:105E900080935B0880E480935D0885E080935008E0
:105EA0002EE120934E0890910804992399F084E103
:105EB0008093510888E280934F082093530881E033
:105EC00080935408109255088FE7809356082093CA
:105ED000A70810C08FE08093510820934F0890933B
:105EE00053083093540884E18093550890935608E2
:105EF0009093A7088FE0809352081092AC088CE032
:105F00008093AD081092690810926A0810926B088D
:105F100010926C08109286081092870810928808D8
:105F20001092890890E890936D0842E340936E08C0
:105F300072E07093B10888E180936F0886EE8093D9
:105F4000700883E0809375085DE75093780850935C
:105F5000790850937A089093710865E56093720808
:105F600086E4809373088CED809374088CE38093AF
:105F70007608109277089AEA90938A088CEC8093BE
:105F80008C0810928E0890938F0898E290938B085B
:105F900090938D081092900840937B082AE52093F7
:105FA0007C0840937D0836E03093910884E6809326
:105FB0009208809393082093940888E7809395082B
:105FC000909399088BE48093960860939708809348
:105FD000980830939A0888E080939B0840939C0827
:105FE0008AE280939D0885EF80939E088CE88093D9
:105FF0009F087093A0081092A2081092A30881E253
:106000008093640881E48093650820936608109269
:10601000A5081092A60886E98093A80850937E08E8
:1060200084E380937F081092A9081092AA08109226
:10603000AB081092AE088FE18093AF0808950E94DC
:106040000A2F8AE08093570880E18093580826E061
:10605000209359089AE590935E0888E780935F083B
:1060600090936108809362082093630880E2809394
:1060700068088CE3809380088BE48093850886E42D
:1060800091E6A3E7B4E78093B4089093B508A09392
:10609000B608B093B70860E870E080E498E00E942A
:1060A000BC2E8093C0080895CF93DF930E940A2FDF
:1060B00088E08093570830E13093580826E0209319
:1060C000590894E690935E0888E780935F08909360
:1060D000610880936208209363083093680886E41F
:1060E0008093800880938508A4EBB8E085E0E9E21E
:1060F000F1E0ED01019009928A95E1F760E870E026
:10610000CD01845790400E94BC2E8093C008DF913F
:10611000CF9108950E940A2F26E0209357088AE025
:106120008093580884E08093590894E690935E0821
:1061300088E780935F0890936108809362082093BA
:10614000630880E18093680886E4809380088093E8
:10615000850885E491E6A3E7B9E78093B4089093B6
:10616000B508A093B608B093B70860E870E080E483
:1061700098E00E94BC2E8093C0080895F999FECF44
:1061800092BD81BDF89A80B599270895F999FECFFF
:106190001FBA92BD81BD60BD0FB6F894FA9AF99A04
:1061A0000FBE089568EA7EE20E940F9E089540EBBC
:1061B0005EE20E94499E0895EF92FF920F931F9313
:1061C000CF93C82F8150853008F0C3E081E8C89F85
:1061D0008001112483EEE82E8FEFF82EE00EF11EE1
:1061E00060E870E0C7010E94CD2E682F98012D59FC
:1061F0003F4F8FB39927AC014270507081FDF9CFAA
:1062000032BD21BDF89A80B5861711F0CA0123C0AE
:106210008FB399279C012270307081FDF9CFF2BCB9
:10622000E1BCF89A80B5813611F0C90114C081E84B
:10623000C89FC00111244D9728EA3EE241E850E092
:10624000BC0180E498E00E94EA9D0E9485760E944D
:10625000839781E090E0CF911F910F91FF90EF9095
:106260000895282F863010F025E003C0882309F414
:1062700021E020930101F999FECF1FBA82E090E05E
:1062800092BD81BD20BD0FB6F894FA9AF99A0FBE5F
:106290000895CF93C82F80914008813609F051C0EE
:1062A000C63010F0C5E003C0CC2309F44AC00E94F8
:1062B0004A9C8091B30882FF07C0809165088436AC
:1062C00018F080E58093650860E870E080E498E06D
:1062D0000E94BC2E8093C00881E8C89FC001112491
:1062E00020EB3EE241E850E060E478E04D970E9408
:1062F000279E20EB3EE24CE050E061E478E080E550
:1063000090E00E94279E6CE070E081E498E00E949B
:10631000BC2E282FF999FECF1FBA8CE590E092BDD4
:1063200081BD20BD0FB6F894FA9AF99A0FBE8C2F52
:106330000E9431310E9485760E94839781E090E02F
:1063400002C080E090E0CF9108956DE470E088EEA7
:1063500093E00E94CD2E482F8FB399279C01227085
:10636000307081FDF9CF85E394E092BD81BDF89A4C
:1063700080B5841779F48FB399279C01227030700F
:1063800081FDF9CF88EE93E092BD81BDF89A80B58A
:10639000813011F0C901089528EA3EE24EE450E050
:1063A00068EE73E081EC98E00E94EA9D81E090E065
:1063B00008958091C1088130A9F46DE470E081EC0A
:1063C00098E00E94BC2E80930E0920EB3EE24EE442
:1063D00050E061EC78E088EE93E00E94279E81E037
:1063E00090E0089580E090E00895CF93DF9381E0FE
:1063F0008093C108E1ECF8E08FE0158616861786D9
:10640000108A8150349687FFF8CF80E48093CE08BD
:106410008093CF081092D0088093D1088093D2083F
:1064200090EC9093D3081092D4088093D508809371
:10643000D6081092D7089093D8089093D9088093E3
:10644000DA081092DB088093DC089093DD08A2EC58
:10645000B8E08CE0EFE2F1E0ED01019009928A955D
:10646000E1F76DE470E0CD0101970E94BC2E8093AE
:106470000E09DF91CF910895F999FECF82E090E067
:1064800092BD81BDF89A80B5282F863078F023E040
:10649000322FF999FECF1FBA82E090E092BD81BD04
:1064A00030BD0FB6F894FA9AF99A0FBE2093010105
:1064B000822F992708951F93CF93C82F162F8630C8
:1064C00010F0C5E003C0882309F4C1E08C2F9927A0
:1064D0008230910541F08330910544F4019731F405
:1064E0000E941F3005C00E94543002C00E948A30B2
:1064F0001123E1F06CE070E080E590E00E94CD2E89
:10650000282FF999FECF8CE590E092BD81BDF89AD5
:1065100080B5821759F428EA3EE24CE050E060E58D
:1065200070E081E498E00E94EA9D02C00E94E52E9E
:106530008C2F0E944931CF911F910895DF92EF92E5
:10654000FF920F931F93CF93FF24DF2CEF2C81E159
:1065500090E00E94BE3090910301981791F196311E
:1065600069F481E190E00E94BE30853139F44C99A4
:1065700005C06F2D81E090E00E94C630609103015C
:1065800081E190E00E94C63088E190E028E00FB6FB
:10659000F894A895809360000FBE2093600082E776
:1065A00098E09F938F9388E996E19F938F93E09172
:1065B0009C05F0919D0509950F900F900F900F90FD
:1065C000FFCF81E090E00E94BE30813611F031E0D3
:1065D000E32E6CE070E080E590E00E94CD2EC82FA5
:1065E000F999FECF8CE590E092BD81BDF89A80B517
:1065F0008C1711F421E0D22EC1E001E010E0EE2072
:1066000029F48C2F0E94DC308823B9F591E0F92E13
:106610001F930F938AE998E09F938F9388E996E1FF
:106620009F938F93E0919C05F0919D0509952DB75F
:106630003EB72A5F3F4F2DBF0130110521F00230D8
:10664000110521F006C00E941F3005C00E94543081
:1066500002C00E948A30DD2059F028EA3EE24CE078
:1066600050E060E570E081E498E00E94EA9D02C09D
:106670000E94E52E8C2F0E944931CF5F0F5F1F4F84
:10668000C63008F4BCCFFF2019F083E00E943131FE
:106690000E943C32C82F0E94DC308C2F99279F9398
:1066A0008F9380EC98E09F938F9308E916E11F93F6
:1066B0000F93E0919C05F0919D05099581E090E094
:1066C0000E94BE302DB73EB72A5F3F4F2DBF8F3F90
:1066D00021F00E94A531882399F489ED98E09F93D9
:1066E0008F931F930F93E0919C05F0919D05099561
:1066F0000E94F5310E94D9310F900F900F900F90AA
:10670000EE2029F061E681E090E00E94C630109210
:106710003F0890E0EEECF8E0CFE080813496181668
:106720000CF49F5FC150C7FFF8CF90933F08892FAB
:1067300099279F938F9382EC98E09F938F938AEF92
:1067400098E09F938F931F930F93E0919C05F09196
:106750009D0509950E94230A8DB79EB708968DBFA7
:10676000CF911F910F91FF90EF90DF900895982F98
:106770002FB7F8943998389A88B1836088B9809196
:10678000B9008C7F8093B9008AE28093B8001092A0
:10679000700310926E0310926D03992379F0E7E174
:1067A000F9E08BE01082118212821382148215822A
:1067B000168217828150389687FFF4CF78942FBFC6
:1067C00008951092700384E98093BC0080E8809360
:1067D000BC001092BD001092BA001092BB00109243
:1067E000B9001092B80010926C0380E00E94B73399
:1067F0001092BB0085E88093BC0080916A038260A0
:1068000080936A0308951F920F920FB60F9211247E
:106810002F933F934F935F938F939F93EF93FF93A8
:1068200080917003282F3327442755278F5F80934B
:106830007003F9012731310508F00DC3E659FF4F08
:106840000C9447A081E080936C0309C080916E0393
:106850008C3090F480916E038F5F80936E038091F3
:106860006E03E82FFF27EE0FFF1FEE0FFF1FEF5302
:10687000F74F8585181654F780916E038C3070F0B1
:10688000109269031092680310926E0385E0809362
:10689000700380916D03880F8D5A04C080916E0340
:1068A000880F8E5A8093BB0085E8CAC280916E0320
:1068B000E82FFF2723E0EE0FFF1F2A95E1F7E95E9F
:1068C000F64F81818093BB0085E88093BC00809166
:1068D0006E03E82FFF2793E0EE0FFF1F9A95E1F775
:1068E000E95EF64F808180FF92C080916E03E82FB1
:1068F000FF2783E0EE0FFF1F8A95E1F7E95EF64F71
:106900008281882329F080913F08873008F4B9C23A
:106910008091680390916903892B09F0B2C280913C
:10692000660390916703892B09F0ABC270C0809118
:106930006E0321E030E002C0220F331F8A95E2F798
:10694000809166039091670328233923232B79F0E4
:1069500080916E03E82FFF27EE0FFF1FEE0FFF1F42
:10696000EE0FFF1FE95EF64F80E184830DC080913A
:106970006E03E82FFF27EE0FFF1FEE0FFF1FEE0F36
:10698000FF1FE95EF64F148280916E03E82FFF2708
:10699000EE0FFF1FEE0FFF1FEE0FFF1FE95EF64F1A
:1069A0008481282F3327220F331F220F331F220FFA
:1069B000331F80916E03E82FFF2753E0EE0FFF1F78
:1069C0005A95E1F7E95EF64F82818770822B8093BA
:1069D000BB0085E88093BC0020916E0381E090E0CD
:1069E00002C0880F991F2A95E2F720916803309121
:1069F000690382239323892B51F08FE099E09093D0
:106A000074038093730388E0809375033AC284E033
:106A1000D4C1E0917303F091740381918093BB0022
:106A200085E88093BC00F0937403E0937303809136
:106A30007503815080937503882309F422C283E093
:106A4000BCC18091B900803349F5809171038823DE
:106A500029F480916E038F5F8093710380916E03A0
:106A6000E82FFF2743E0EE0FFF1F4A95E1F7E95EAD
:106A7000F64F838199278F7790708F37910574F443
:106A800080916E03E82FFF2733E0EE0FFF1F3A954A
:106A9000E1F7E95EF64F83818F5F83831092700385
:106AA00084E98093BC008AE090E090933D0180935C
:106AB0003C0180916E038F5F80936E031092700390
:106AC000B9C18091B9008034C1F180916D03E82F84
:106AD000FF2723E0EE0FFF1F2A95E1F7E95EF64F4F
:106AE00083818F77838380916D038F5F80936D03A4
:106AF00080916D038C30A0F010926D0310926703AB
:106B000010926603809172038F5F809372038C30C2
:106B100038F01092720380916A038D7F80936A032C
:106B200080916A03816080936A031092700384E904
:106B30008093BC0010926C0383C080916D03E82F9A
:106B4000FF2793E0EE0FFF1F9A95E1F7E95EF64FFE
:106B500083818068838380916D03E82FFF2783E022
:106B6000EE0FFF1F8A95E1F7E95EF64F808180FF07
:106B700040C080916D03E82FFF27EE0FFF1FEE0F3F
:106B8000FF1FEE0FFF1FE95EF64F848199270097E4
:106B9000D1F0409709F04BC08FE099E090937403D7
:106BA0008093730388E08093750380916D03E82FD1
:106BB000FF27EE0FFF1FEE0FFF1FEE0FFF1FE95E17
:106BC000F64F148234C080916D039927E3E0880F5B
:106BD000991FEA95E1F7845E964F90937403809332
:106BE000730390916D03809172039817E9F483E029
:106BF0001CC080916D039927880F991F880F991FDA
:106C0000880F991F845E964F90937403809373034B
:106C100080916A0381FD06C090916D03809172039B
:106C2000981711F482E001C081E080937503809190
:106C30007503813011F485E801C085EC8093BC00B8
:106C40008091710380936B03109271031AC1E091DC
:106C50007303F09174038091BB0080838091730370
:106C600090917403019690937403809373038091C1
:106C70007503815080937503823010F085EC9AC0C3
:106C8000813011F485E896C080916A0381FF6AC063
:106C90008091100480FD66C080916D03E82FFF276E
:106CA000EE0FFF1FEE0FFF1FEE0FFF1FE95EF64F07
:106CB000868199278C7F9070883F910579F4809127
:106CC0006D03E82FFF2753E0EE0FFF1F5A95E1F702
:106CD000E95EF64F8081816080830CC080916D03F6
:106CE000E82FFF2743E0EE0FFF1F4A95E1F7E95E2B
:106CF000F64F108280916D03E82FFF2733E0EE0FEF
:106D0000FF1F3A95E1F7E95EF64F8681883F71F4FF
:106D100080916D03E82FFF2723E0EE0FFF1F2A95D8
:106D2000E1F7E95EF64F808186601BC080916D03BC
:106D3000E82FFF2793E0EE0FFF1F9A95E1F7E95E3A
:106D4000F64F8681893F71F480916D03E82FFF270C
:106D500083E0EE0FFF1F8A95E1F7E95EF64F808131
:106D60008460808380916D038F5F80936D03809139
:106D70006D038C30A0F010926D0310926703109297
:106D80006603809172038F5F809372038C3038F0BA
:106D90001092720380916A038D7F80936A03109230
:106DA000700384E98093BC0080916A0381608093C2
:106DB0006A0365C08093BC0086E08093700361C065
:106DC00088E970CD80916F03880F805F6BCD8091D3
:106DD0006F0399278130910561F0823091051CF491
:106DE000892B21F04EC0029739F04BC080911B01D6
:106DF00059CD80911A0156CD8091190153CD80E86B
:106E000051CD1092700384E98093BC0010926C0302
:106E10008AE090E090933D0180933C0180916F0364
:106E2000823088F480916F038F5F80936F0382E1DB
:106E30008093700380916A038E7F80936A0385EA52
:106E40008093BC001EC010926F0380916A03816022
:106E500080936A0316C01092700384E98093BC008B
:106E600080916A03816080936A038AE090E0909346
:106E70003D0180933C0110926E0310926D031092BD
:106E80006C03FF91EF919F918F915F914F913F9193
:106E90002F910F900FBE0F901F9018951F93CF93B7
:106EA000DF93182F80914804882321F48091FB02FE
:106EB000882319F081E090E09AC01D3008F095C059
:106EC0001123B1F0E12FFF2743E0EE0FFF1F4A959A
:106ED000E1F7E95EF64F35978081359688230CF00F
:106EE00084C03897808180FD03C083E090E07FC03C
:106EF00080910F0999278B709070029719F084E0A8
:106F000090E075C067E070E08FE099E00E94BC2ED1
:106F100090911609891719F085E090E068C080ED1E
:106F200097E00E94691AEC0180916A0380FD05C018
:106F3000CE010E94721A8823B9F3112319F48FEF3E
:106F400090E00BC0212F33272150304081E090E0AA
:106F500002C0880F991F2A95E2F7909369038093E6
:106F60006803A1E0B0E0E7E1F9E040E050E06BE069
:106F7000CD01042E02C0880F991F0A94E2F72091D8
:106F800068033091690382239323892B11F01182C6
:106F9000128261504F5F5F4F389667FFE9CF1092C2
:106FA0006E031092700380916A038E7F80936A0350
:106FB00085EA8093BC0080916A0380FD05C0CE0104
:106FC0000E94721A8823B9F3809168039091690333
:106FD000892B29F0CE010E94721A882311F3809127
:106FE000680390916903009711F082E090E0DF91CF
:106FF000CF911F9108950F931F93CF93DF93982FF5
:1070000080914804882321F48091FB02882319F0A1
:1070100081E090E095C09D30A0F4992319F486E0BA
:1070200090E08EC0C92FDD27FE0153E0EE0FFF1F59
:107030005A95E1F7E95EF64F35978081359687FDE1
:1070400003C082E090E07CC03897808180FD03C05F
:1070500083E090E075C080ED97E00E94691A8C0192
:1070600080916A0380FD05C0C8010E94721A8823BE
:10707000B9F3219721E030E0C90102C0880F991FC0
:10708000CA95E2F79093670380936603D901E7E11D
:10709000F9E040E050E06BE0CD01042E02C0880F23
:1070A000991F0A94E2F720916603309167038223C7
:1070B0009323892B11F01182128261504F5F5F4F31
:1070C000389667FFE9CF10926D0310920F09109266
:1070D00016091092700380916A038E7F80936A0371
:1070E00085EA8093BC0080916A0380FD05C0C801D9
:1070F0000E94721A8823B9F3809166039091670306
:10710000892B29F0C8010E94721A882311F38091FB
:107110000F0999278B709070029719F084E090E026
:107120000FC067E070E08FE099E00E94BC2E909164
:107130001609891719F085E090E002C080E090E020
:10714000DF91CF911F910F910895CF93DF9380E04E
:1071500021E83FEFCEEBD9E0E8E7F9E0DF01853049
:1071600020F411961C921E9202C031832083198252
:10717000188222968F5F12963296833280F38FE7C1
:1071800090E09093B7098093B60981E89FEF9093C0
:10719000B5098093B4091092B9091092B8091092F8
:1071A000B6041092B5041092B8041092B70410926D
:1071B000BA041092B904DF91CF9108951F920F92F3
:1071C0000FB60F9211240F931F932F933F934F935A
:1071D0005F936F937F938F939F93AF93BF93CF935F
:1071E000DF93EF93FF938091B20882FDC2C040917C
:1071F0008600509187008091770390917803481B17
:10720000590B80918600909187009093780380932A
:107210007703CA018D549440A0917903B0917A0309
:10722000835F9A4158F4809179038093770914978A
:1072300014F01092400181E090E096C0A131B105B8
:107240000CF0F7C1CA018B5F9040845B914008F05D
:1072500086C080913E0190913F01481B590BE091FF
:10726000A908EE2351F0FF27EE0FFF1FE858F64F55
:107270008081918184369105ECF4FD01EA0FFB1FBA
:10728000E858F64F80819181FA01E81BF90BCF0194
:10729000F7FF03C0909581959F4F06975CF480910E
:1072A0004904883C20F480914904865F01C088EC41
:1072B00080934904FD01EA0FFB1FE858F64F8081D7
:1072C00091819C01220F331F280F391F240F351F76
:1072D00037FF02C02D5F3F4FE901D595C795D59582
:1072E000C795CA0101968C179D0714F4219706C013
:1072F00041505040C417D5070CF4219680914904A1
:10730000833CE0F08D010A0F1B1FF801E858F64F8F
:10731000808191819E01281B390BC90163E070E0D7
:107320000E94C09FCB01880F991F860F971F0254A0
:10733000164FD80111969C938E9307C0AA0FBB1FBE
:10734000A254B64F11961C921E92E0917903F091CF
:107350007A03EE0FFF1FE858F64FD183C083809168
:10736000790390917A03019690937A03809379033D
:1073700060C1409186005091870080917B0390917D
:107380007C03481B590B8091860090918700909355
:107390007C0380937B03CA018D5494406091050463
:1073A000835F9A4108F07AC06093760380917603F8
:1073B000843008F453C09091770980917603981730
:1073C00009F04CC0509106045B3008F43FC01092A5
:1073D00040011092050440E05F31C0F0E42FFF2728
:1073E000EE0FFF1F9F012F533C4FDF01A858B64FF0
:1073F0008D919C91D9018D939C93DF01A254B64F3E
:107400008D919C91ED51FC4F91838083E42FFF2758
:10741000EE0FFF1F9F012858364FDF01A358BC4FC6
:107420008D919C91D90111969C938E93DF01A15669
:10743000BC4F8D919C91E254F64F91838083842FB1
:107440008F5F482F813140F28093050480910604BC
:107450008F3FB9F08F5F8093060413C080910604BC
:10746000853620F08AE08093060402C0109206045C
:10747000809103018A3011F0843110F0289A01C004
:10748000289881E08093050480914804882309F0BE
:10749000D0C08091760380937709CBC0613108F02A
:1074A000A0C0CA018B5F9040845B914008F090C0FF
:1074B00080913E0190913F01481B590BE62FFF2719
:1074C000EE0FFF1FE358FC4F80819181FA01E81B0A
:1074D000F90BCF0105960B9720F5E091A908EE2353
:1074E00051F0FF27EE0FFF1FE858F64F8081918182
:1074F00084369105B4F4809106048A3120F080919D
:107500004904865F05C08B3028F0809149048E5F66
:107510008093490480914904893C18F088EC809359
:107520004904E62FFF27EE0FFF1FE358FC4F808131
:1075300091819C01220F331F280F391F240F351F03
:1075400037FF02C02D5F3F4FE901D595C795D5950F
:10755000C795CA0101968C179D0714F4219706C0A0
:1075600041505040C417D5070CF42196809149042E
:107570008E3BD8F0E62FFF27EE0FFF1FDF01A35849
:10758000BC4F8D919C919E01281B390BC90163E072
:1075900070E00E94C09FCB01880F991F860F971F34
:1075A000E156FC4F9183808308C0E62FFF27EE0F42
:1075B000FF1FE156FC4F1182108280910504E82FD5
:1075C000FF27EE0FFF1FE358FC4FD183C08309C094
:1075D000809103018A3011F0843110F0289A01C0A3
:1075E000289880910504843120F48F5F80930504EE
:1075F00020C08431F1F4809103018A3011F084318C
:1076000010F0289A01C028988EE18093050420E1AB
:10761000CEEBD9E0A1ECB3E0E8E7F9E08D919D91E4
:10762000918380833296198218822296215027FFF7
:10763000F5CFFF91EF91DF91CF91BF91AF919F91E6
:107640008F917F916F915F914F913F912F911F91FA
:107650000F910F900FBE0F901F9018958091840A84
:107660009091850A90939C0780939B078091860A4E
:107670009091870A90939E0780939D0780915A0A64
:1076800090915B0A97FD03969595879595958795BB
:107690009093A00780939F0780916A0A90916B0A4C
:1076A00097FD039695958795959587959093A20755
:1076B0008093A1078091B5049091B6042091400376
:1076C00030914103821B930B9093A4078093A307EF
:1076D0008091430490914404A0914504B0914604E4
:1076E000BC01CD012AE030E040E050E00E94F59F6F
:1076F0003093A6072093A5078091E0079091E107BA
:107700009093A8078093A707809190019091910191
:107710009093AC078093AB0780912601909127014D
:107720009093AE078093AD07809149049927909379
:10773000B0078093AF078091120A9091130A90933B
:10774000B2078093B1078091180999279093B407E5
:107750008093B3078091200999279093B60780936F
:10776000B5078091280999279093B8078093B707A8
:107770008091300999279093BA078093B907809137
:107780001603909117039093C4078093C3078091C9
:107790002D0490912E049093C6078093C507809185
:1077A000EB0A9091EC0A9093C8078093C7078091E9
:1077B000EF0A9091F00A9093CA078093C9078091CD
:1077C0003F0490914004A0914104B0914204BC0157
:1077D000CD012AE030E040E050E00E94F59F309378
:1077E000CC072093CB078091610490916204909321
:1077F000D2078093D1078091F10A99279093D607F9
:107800008093D50780911B0590911C059093D80714
:107810008093D7078091190590911A059093DA0704
:107820008093D9078091B505882321F48091B6050E
:10783000882321F080919A07816003C080919A0784
:107840008E7F80939A070895EF92FF921F93CF93B4
:10785000DF93182F7B0180914804882391F5809154
:1078600003018C3010F0893111F4299801C0299A54
:1078700011501F3FE9F0F0921E03E0921D03E70153
:1078800080911D0390911E03892B11F4209781F3A1
:10789000809121038823A1F31092210380911D037D
:1078A00090911E03892B09F421970E94609CE8CFD8
:1078B000809103018C3010F0893111F4299A01C0B4
:1078C0002998DF91CF911F91FF90EF900895CF936A
:1078D000DF93809103018D3011F40E94C21F10923A
:1078E0007A00809144039091450390931D0A809300
:1078F0001C0A809142039091430390930E0A809357
:107900000D0A80914003909141039093600A809307
:107910005F0A20913C0330913D03C901880F991FF4
:10792000880F991F820F931F820F931F90935B0AFA
:1079300080935A0A20913E0330913F03C901880F7A
:10794000991F880F991F820F931F820F931F909387
:107950006B0A80936A0A8FEC80937A00AAE4B4E001
:10796000C5E4D8E097E08991E82FFF27EE0FFF1FCD
:10797000E858F64F0190F081E02DE158FF4F1E16B8
:107980001F061CF0E0E0F0E005C0EF3FF10514F049
:10799000EFEFF0E08C91282F3327E217F30714F470
:1079A000815004C02E173F0714F48F5F8C939150C1
:1079B000119697FFD8CF809181089927AA27BB27D6
:1079C000BC01CD0124EC39E040E050E00E94819FF1
:1079D000DC01CB018093880190938901A0938A01F7
:1079E000B0938B01809182089927AA27BB27BC01FD
:1079F000CD010E94819FDC01CB0180938401909393
:107A00008501A0938601B0938701DF91CF910895FE
:107A1000A0E0B0E0EEE0FDE30C9414A0782E91E03D
:107A2000692ECC24DD2456014601E6011092B505ED
:107A3000D092B004C092AF04D092AE04C092AD0414
:107A4000D092AA04C092A9041092A804D092BA04B9
:107A5000C092B904D092B804C092B704D092B604D0
:107A6000C092B50410926A01109269011092350318
:107A70000E94673C84E690E00E948B1A0E94673C5B
:107A800080914D0880FF14C080911C0190911D01D0
:107A9000875B934058F480911C0190911D018E5E8C
:107AA000924020F080913503882311F00E94221F1C
:107AB00000911C0110911D0187B58B5F87BD87B5B3
:107AC000809588BD8FE1E82E8AE090E00E948B1AB5
:107AD0008091400390914103C80ED91E80914403C8
:107AE00090914503A80EB91E8091420390914303E3
:107AF000880E991E8091E0079091E107C80FD91F69
:107B0000EA94E7FEE1CF80911C0190911D01825F14
:107B1000934080F480911C0190911D01459750F095
:107B200080911C0190911D01081B190B10931701E6
:107B30000093160187B5855087BD87B5809588BDB0
:107B40009501205F3F4F36952795369527953093C1
:107B5000BA042093B904C4014096969587959695EA
:107B600087959093B8048093B70440E150E0C40E29
:107B7000D51EB5E0D694C794BA95E1F7D092B60475
:107B8000C092B504C40FD51FA5E0D695C795AA9598
:107B9000E1F7D093AA04C093A9049093B40480930E
:107BA000B3043093B2042093B10452E07516C9F5C2
:107BB00080915A0A90915B0A97FF03C09095819536
:107BC0009F4F6CE070E00E94C09F9B017093B004D7
:107BD0006093AF0480916A0A90916B0A97FF03C08B
:107BE000909581959F4F6CE070E00E94C09F7093CC
:107BF000AE046093AD04B90184E090E00E94D730F8
:107C00006091AD047091AE0486E090E00E94D730A0
:107C10006091A9047091AA0488E090E00E94D73096
:107C20004FC084E090E00E94D2309093B0048093E3
:107C3000AF0486E090E00E94D2309C019093AE04A5
:107C40008093AD048091AF049091B004815098402E
:107C500018F421503840A0F18BE199E09F938F9365
:107C600088E996E19F938F93E0919C05F0919D05A3
:107C7000099580915A0A90915B0A97FF03C09095ED
:107C800081959F4F6CE070E00E94C09F7093B0049C
:107C90006093AF0480916A0A90916B0A97FF03C0CA
:107CA000909581959F4F6CE070E00E94C09F70930B
:107CB000AE046093AD0466240F900F900F900F9068
:107CC00012BC11BC10921D0A10921C0A10920E0ACE
:107CD00010920D0A1092600A10925F0A88EC90E0F0
:107CE0000E948B1A80913C0390913D039C01220FCE
:107CF000331F220F331F280F391F280F391F3093CE
:107D00005B0A20935A0A80913E0390913F038C01B5
:107D1000000F111F000F111F080F191F080F191F47
:107D200010936B0A00936A0A80915C08C82EDD24C8
:107D3000EE24FF24442737FD4095542FC701B60198
:107D40000E94819F4B015C016093A3047093A40483
:107D50008093A5049093A6049801442737FD40958D
:107D6000542FC701B6010E94819FDC01CB01809393
:107D70009B0490939C04A0939D04B0939E048092D6
:107D8000830490928404A0928504B0928604809328
:107D90007B0490937C04A0937D04B0937E041092A6
:107DA000730410927404109275041092760400917A
:107DB000900110919101109362040093610484E694
:107DC00090E090938D0180938C0182E390E09093FA
:107DD0001E0380931D03809181089927AA27BB2742
:107DE000BC01CD0124EC39E040E050E00E94819FCD
:107DF000DC01CB018856954CAF4FBF4F8093880173
:107E000090938901A0938A01B0938B01809182089D
:107E10009927AA27BB27BC01CD010E94819FDC01C5
:107E2000CB018856954CAF4FBF4F80938401909300
:107E30008501A0938601B0938701109247011092AB
:107E40004601C801AA2797FDA095BA2F20914201AB
:107E5000309143014091440150914501BC01CD0155
:107E60000E94819FDC01CB018093660A9093670A90
:107E7000A093680AB093690A10925E0410925D04A0
:107E80000E948576772029F0809110048460809389
:107E900010048FEF8093E60A1092E70A80E2809345
:107EA000E80ACAE4D4E0A5E4B8E077E0E72E8D91D3
:107EB000E82FFF27EE0FFF1FE858F64F80819181D2
:107EC00081588993EA94E7FEF2CF84E680934904CF
:107ED00080911B03882311F0579A17C08091B10835
:107EE000992780FF05C082FF03C080EE9EE202C09A
:107EF00080E091E190930A018093090181E08093F1
:107F000011010E942C1B0E942C1B8091A3049091B4
:107F1000A404A091A504B091A604E0904201F090C1
:107F200043010091440110914501BC01CD01A8011C
:107F300097010E94F59F59016A0180919B049091DD
:107F40009C04A0919D04B0919E04BC01CD01A801A8
:107F500097010E94F59FB901C5010E94A19D8C0166
:107F60000E94F7799C019093270A8093260A8091BA
:107F7000A9049091AA04AA2797FDA095BA2F6DE0B5
:107F8000880F991FAA1FBB1F6A95D1F78050904F89
:107F9000AF43B040442737FD4095542FBC01CD017D
:107FA0000E94F59FC90180509E4F9093AA04809330
:107FB000A904053111050CF06624772079F0809131
:107FC0000804882359F0C90181599040C39730F0C3
:107FD0008091B50580628093B50566248091B904CF
:107FE0009091BA0480569940815C9B4228F0809120
:107FF000B50581608093B5058091B7049091B80470
:1080000080569940815C9B4228F08091B505826042
:108010008093B5058091B5049091B6048C5291403F
:108020008957954028F08091B50584608093B50507
:108030008091AF049091B0048C529140835C914048
:1080400028F08091B50588608093B5058091AD04D6
:108050009091AE048C529140835C914028F08091C5
:10806000B50580618093B5058091A9049091AA041B
:10807000805092408355914028F08091B5058062F0
:108080008093B5058091B5058111662486E48093BF
:108090007F010E94839782E00E94E89880911E01F0
:1080A00090911F01A0912001B09121018093E207DE
:1080B0009093E307A093E407B093E507109234038D
:1080C0001092330310923603109237031092380344
:1080D00010923903109263041092640410926504A4
:1080E000109266041092D4071092D3070E94EA1EE1
:1080F000862D9927EEE0CDB7DEB70C9430A0A3E132
:10810000B0E0E5E8F0E40C9410A08091B504909103
:10811000B6042091400330914103821B930B90934E
:10812000600A80935F0A80914A0390914B0397FD08
:1081300007969C0153E0359527955A95E1F73093C2
:108140001D0A20931C0A809148039091490397FDD2
:10815000079643E0959587954A95E1F790930E0A27
:1081600080930D0A3093290A2093280A9093200ABD
:1081700080931F0A80915A0A90915B0AAC01440FC8
:10818000551F480F591F20913C0330913D03C901F1
:10819000880F991F880F991F820F931F820F931FBB
:1081A000480F591F57FF02C04D5F5F4F55954795C8
:1081B0005595479550935B0A40935A0A80916A0AF5
:1081C00090916B0AAC01440F551F480F591F209125
:1081D0003E0330913F03C901880F991F880F991FF3
:1081E000820F931F820F931F480F591F57FF02C022
:1081F0004D5F5F4F559547955595479550936B0A41
:1082000040936A0A20913C0330913D03C901880FD5
:10821000991F880F991F820F931F820F931F9C0134
:10822000442737FD4095542F8091930490919404F6
:10823000A0919504B0919604820F931FA41FB51FBF
:108240008093930490939404A0939504B093960420
:1082500020913E0330913F03C901880F991F880F79
:10826000991F820F931F820F931F9C01442737FD94
:108270004095542F80918F0490919004A091910487
:10828000B0919204820F931FA41FB51F80938F0497
:1082900090939004A0939104B09392048091320A39
:1082A0009091330A20913C0330913D03820F931F3C
:1082B0009093330A8093320A8091620A9091630A04
:1082C00020913E0330913F03820F931F9093630AE6
:1082D0008093620A8091AB049091AC0401969093D4
:1082E000AC048093AB048091E0079091E10720916A
:1082F000A9043091AA04821B930B9C01442737FDEB
:108300004095542F80918B0490918C04A0918D0402
:10831000B0918E04820F931FA41FB51F80938B040E
:1083200090938C04A0938D04B0938E048FEC809373
:108330007A001092180120917B0430917C044091C6
:108340007D0450917E0429873A874B875C872954A6
:108350003B46414050402CF028E43BE641E050E0F1
:108360000DC089859A85AB85BC85885B9449AE4FE5
:10837000BF4F4CF428EB34E94EEF5FEF2D833E8383
:108380004F83588708C089859A85AB85BC858D83C6
:108390009E83AF83B88720918304309184044091F9
:1083A0008504509186042D873E874F87588B29542A
:1083B0003B46414050402CF028E43BE641E050E091
:1083C0000DC08D859E85AF85B889885B9449AE4F79
:1083D000BF4F4CF428EB34E94EEF5FEF29833A832B
:1083E0004B835C8308C08D859E85AF85B889898362
:1083F0009A83AB83BC83A0915F0AB091600ABB8B68
:10840000AA8BFD01CF01AA2797FDA095BA2FA090B6
:108410007304B0907404C0907504D0907604A80ED4
:10842000B91ECA1EDB1EA0927304B0927404C092DF
:108430007504D0927604E090660AF090670A009185
:10844000680A1091690AE80EF91E0A1F1B1FE092C4
:10845000660AF092670A0093680A1093690AF0911D
:108460002C04F98BFF2309F098C180912B048823F9
:1084700009F093C18091560A86FF8FC180910D0A41
:1084800090910E0AAA2797FDA095BA2FBC01CD01A5
:1084900029813A814B815C810E94819F9B01AC01C3
:1084A00097FF04C02150384F4F4F5F4F6BE05595F9
:1084B0004795379527956A95D1F780916901682E80
:1084C000772488249924CA01B901A40193010E9448
:1084D000819FDC01CB018093C5049093C604A093D7
:1084E000C704B093C804B7FF04C08150904FAF4F8A
:1084F000BF4F1C012D013CE05594479437942794BD
:108500003A95D1F72092C5043092C6044092C70430
:108510005092C80480911C0A90911D0AAA2797FDC9
:10852000A095BA2FBC01CD012D813E814F81588588
:108530000E94819F97FF04C06150784F8F4F9F4FDB
:108540002BE095958795779567952A95D1F7A401A6
:1085500093010E94819FDC01CB018093C904909319
:10856000CA04A093CB04B093CC04B7FF04C08150DD
:10857000904FAF4FBF4F9C01AD018CE05595479593
:10858000379527958A95D1F72093C9043093CA046B
:108590004093CB045093CC048091C5049091C604C1
:1085A0009093050A8093040A8091C9049091CA04AB
:1085B0009093090A8093080A22193309440955093E
:1085C0002093C9043093CA044093CB045093CC0445
:1085D000E20EF31E041F151FE092660AF092670A6E
:1085E0000093680A1093690A809168018823B1F4A6
:1085F00057FF04C02F5F3F4F4F4F5F4F5595479533
:1086000037952795A21AB30AC40AD50AA092730413
:10861000B0927404C0927504D09276042A893B8982
:1086200079010027F7FC0095102F8091C9049091E3
:10863000CA04A091CB04B091CC04E80EF91E0A1F25
:108640001B1FC801B70129813A814B815C810E94BF
:10865000819F9B01AC0197FF04C02150384F4F4FC1
:108660005F4FBBE05595479537952795BA95D1F75C
:1086700080916A01A82EBB24CC24DD24CA01B90153
:10868000A60195010E94819FDC01CB018093BD046E
:108690009093BE04A093BF04B093C004B7FF04C07E
:1086A0008150904FAF4FBF4F3C014D01ACE09594CE
:1086B000879477946794AA95D1F76092BD047092DD
:1086C000BE048092BF049092C004C801B7012D81FE
:1086D0003E814F8158850E94819F97FF04C0615061
:1086E000784F8F4F9F4FFBE09595879577956795CE
:1086F000FA95D1F7A60195010E94819FDC01CB017B
:108700008093C1049093C204A093C304B093C404A3
:10871000B7FF04C08150904FAF4FBF4FAC01BD01B8
:10872000ECE07595679557954795EA95D1F7409395
:10873000C1045093C2046093C3047093C4042A8993
:108740003B8937FF03C0309521953F4F21343105D8
:10875000E4F1D401C30197FE07C0B095A0959095B0
:1087600081959F4FAF4FBF4F81389105A105B1054E
:1087700084F4DB01CA0177FF07C0B095A0959095FE
:1087800081959F4FAF4FBF4F81389105A105B1052E
:10879000E4F081E080935F0418C01092090A1092FF
:1087A000080A1092050A1092040A1092C10410924D
:1087B000C2041092C3041092C4041092BD0410921B
:1087C000BE041092BF041092C0048091C104909125
:1087D000C204A091C304B091C404BC01CD0124E63D
:1087E00030E040E050E00E94F59FE090BD04F09042
:1087F000BE04E21AF30AF0921B0AE0921A0A809170
:10880000BD049091BE04A091BF04B091C004BC010E
:10881000CD0124E630E040E050E00E94F59FDA010F
:10882000C9012091C1043091C2048C01021B130BB9
:108830001093100A00930F0A809142019091430116
:10884000A0914401B0914501BC01CD0128E631E081
:1088500040E050E00E94819F2091660A3091670AB3
:108860004091680A5091690A261737074807590747
:1088700064F0261B370B480B590B2093660A309384
:10888000670A4093680A5093690A2091660A3091FA
:10889000670A4091680A5091690A57FF0CC0260F79
:1088A000371F481F591F2093660A3093670A409369
:1088B000680A5093690A60910D0A70910E0A6E0D54
:1088C0007F1D9B01442737FD4095542F80917704ED
:1088D00090917804A0917904B0917A04820F931F4B
:1088E000A41FB51F8093770490937804A093790414
:1088F000B0937A048091310490913204681B790B13
:10890000CB01AA2797FDA095BA2F29853A854B85DB
:108910005C85820F931FA41FB51F80937B049093E7
:108920007C04A0937D04B0937E04C0908401D09019
:108930008501E0908601F0908701C816D906EA0605
:10894000FB06C4F488EA91E6A0E0B0E08C199D092A
:10895000AE09BF0980937B0490937C04A0937D04AF
:10896000B0937E048093770490937804A093790465
:10897000B0937A0422273327A9012C193D094E0907
:108980005F0980917B0490917C04A0917D04B0915B
:108990007E0482179307A407B507B4F4D701C60174
:1089A000885A9146A040B04080937B0490937C0409
:1089B000A0937D04B0937E04809377049093780411
:1089C000A0937904B0937A0460911C0A70911D0AF7
:1089D000600F711F9B01442737FD4095542F8091F4
:1089E0007F0490918004A0918104B0918204820F51
:1089F000931FA41FB51F80937F0490938004A093BE
:108A00008104B093820480912F0490913004681BFC
:108A1000790BCB01AA2797FDA095BA2F2D853E850E
:108A20004F855889820F931FA41FB51F809383041D
:108A300090938404A0938504B0938604E090880109
:108A4000F090890100918A0110918B01E816F906D6
:108A50000A071B07C4F488EA91E6A0E0B0E08E198B
:108A60009F09A00BB10B8093830490938404A0937F
:108A70008504B093860480937F0490938004A09330
:108A80008104B093820422273327A9012E193F09BC
:108A9000400B510B8091830490918404A091850434
:108AA000B091860482179307A407B507B4F4D801E0
:108AB000C701885A9146A040B040809383049093A8
:108AC0008404A0938504B093860480937F049093DC
:108AD0008004A0938104B0938204809173049091E8
:108AE0007404A0917504B0917604809387049093E8
:108AF0008804A0938904B0938A04809183049091A0
:108B00008404A0918504B09186048093A30490937B
:108B1000A404A093A504B093A60480917B04909133
:108B20007C04A0917D04B0917E0480939B0490937B
:108B30009C04A0939D04B0939E0480917F04909127
:108B40008004A0918104B091820480939F0490934B
:108B5000A004A093A104B093A20480917704909103
:108B60007804A0917904B0917A048093970490934B
:108B70009804A0939904B0939A0480912401909151
:108B8000250197FD079633E0959587953A95E1F78E
:108B900090931D0A80931C0A8091220190912301D9
:108BA00097FD079623E0959587952A95E1F7909391
:108BB0000E0A80930D0A80914403909145030F970C
:108BC00034F488E19CEF90931D0A80931C0A8091F5
:108BD000440390914503079734F480E398EF909312
:108BE0001D0A80931C0A209103012A30A9F4809168
:108BF000440390914503835F934034F088EE93E003
:108C000090931D0A80931C0A809144039091450320
:108C10008A5F9340DCF014C0809144039091450337
:108C2000815D974034F088EE93E090931D0A809325
:108C30001C0A8091440390914503805E974034F074
:108C400080ED97E090931D0A80931C0A8091420367
:108C5000909143030F9734F488E19CEF90930E0AB0
:108C600080930D0A8091420390914303079734F457
:108C700080E398EF90930E0A80930D0A2A30A9F4AE
:108C80008091420390914303835F934034F088EED8
:108C900093E090930E0A80930D0A80914203909185
:108CA00043038A5F9340DCF014C0809142039091AB
:108CB0004303815D974034F088EE93E090930E0A71
:108CC00080930D0A8091420390914303805E974008
:108CD00034F080ED97E090930E0A80930D0A609136
:108CE0007701662309F4AFC040912401509125011A
:108CF0008091CD049091CE04481B590B5093D4041D
:108D00004093D3042091240130912501280F391F6D
:108D100037FF02C02F5F3F4F359527953093CE0424
:108D20002093CD04413851051CF080E890E005C047
:108D300040585F4F34F480E89FEF9093D4048093C1
:108D4000D30440912201509123018091CF0490914E
:108D5000D004481B590B5093D2044093D104209166
:108D6000220130912301280F391F37FF02C02F5FE6
:108D70003F4F359527953093D0042093CF04413849
:108D800051051CF080E890E005C040585F4F34F476
:108D900080E89FEF9093D2048093D104462F55270B
:108DA0008091D3049091D404849FB001859F700D6D
:108DB000949F700D11249B0177FF02C0215F3F4FEC
:108DC000B4E035952795BA95E1F780911C0A90910A
:108DD0001D0A820F931F90931D0A80931C0A809195
:108DE000D1049091D204849FD001859FB00D949FAF
:108DF000B00D1124AD019D01B7FF02C0215F3F4FAF
:108E0000A4E035952795AA95E1F780910D0A9091F8
:108E10000E0A820F931F90930E0A80930D0A809181
:108E2000240190912501860F971F9093250180932F
:108E300024018091220190912301840F951F90932A
:108E400023018093220100911F0A1091200A809132
:108E5000040A9091050A101611065CF59C0197FF13
:108E600004C022273327281B390BC901AA2797FDE5
:108E7000A095BA2F20916801332744275527BC01BC
:108E8000CD010E94819F9B01AC0197FF04C0215C32
:108E90003F4F4F4F5F4FF6E05595479537952795D4
:108EA000FA95D1F780911A0A90911B0A820F931FAD
:108EB00027C097FF03C0909581959F4FAA2797FDE4
:108EC000A095BA2F20916801332744275527BC016C
:108ED000CD010E94819F9B01AC0197FF04C0215CE2
:108EE0003F4F4F4F5F4FE6E0559547953795279594
:108EF000EA95D1F780911A0A90911B0A821B930B75
:108F000090931B0A80931A0AE090280AF090290A8D
:108F10008091080A9091090A1E141F045CF59C01B7
:108F200097FF04C022273327281B390BC901AA2722
:108F300097FDA095BA2F2091680133274427552724
:108F4000BC01CD010E94819F9B01AC0197FF04C031
:108F5000215C3F4F4F4F5F4F76E0559547953795D2
:108F600027957A95D1F780910F0A9091100A820F78
:108F7000931F27C097FF03C0909581959F4FAA2705
:108F800097FDA095BA2F20916801332744275527D4
:108F9000BC01CD010E94819F9B01AC0197FF04C0E1
:108FA000215C3F4F4F4F5F4F66E055954795379592
:108FB00027956A95D1F780910F0A9091100A821B2C
:108FC000930B9093100A80930F0A8091560A87FFA3
:108FD00044C0B989BB2309F040C080912B04882389
:108FE000E1F5E1E0EE16E1E0FE064CF080911C0AAE
:108FF00090911D0A8E0D9F1D805091400DC0F0E094
:10900000EF16FFEFFF0664F480911C0A90911D0A91
:109010008E0D9F1D80509F4F90931D0A80931C0AB8
:1090200021E0013012074CF080910D0A90910E0A58
:10903000800F911F805091400CC03FEF003013070C
:1090400064F480910D0A90910E0A800F911F805058
:109050009F4F90930E0A80930D0AE2E1CD5E0C942F
:109060002CA080914804882329F5809110048C7FDE
:109070008093100480910F048F7D80930F04AAEBDE
:10908000B5E0E7E1F9E09BE08091FB02882309F479
:109090008C938D91818312829150389697FFF4CFF3
:1090A0008091FB02882359F08091FB0281508093CC
:1090B000FB0205C0809110048160809310048091B0
:1090C0006C03882319F010926C03089580936E034B
:1090D0008093700380916A038E7F80936A0385EA90
:1090E0008093BC000895882319F480E090E00895EF
:1090F000E82FFF27EE0FFF1FE858F64F8081918180
:1091000081589F4F8F3F910521F01CF08FEF90E029
:1091100004C097FF02C080E090E099270895CF93A4
:10912000DF93AAE4B4E0C5E4D8E057E08991E82FE2
:10913000FF27EE0FFF1FE858F64F0190F081E02D5A
:10914000E158FF4FEF3FF10521F01CF0EFEFF0E0A9
:1091500004C0F7FF02C0E0E0F0E0893111F4EC93C5
:109160001BC04C91242F3327E217F307A9F0CF013E
:10917000821B930B97FD03969595879595958795FB
:10918000242F280F2C93822F9927E817F90714F41E
:10919000215001C02F5F2C935150119657FFC6CF1D
:1091A00080914F08883F38F0EFEFF0E0E81BF109BD
:1091B000E65BFB4F808180937C0180917C0188235A
:1091C00029F0843618F084E680937C018091510860
:1091D000883F38F0EFEFF0E0E81BF109E65BFB4F6A
:1091E000808180937B0180917B01882329F08436E4
:1091F00018F084E680937B0180915E08883F38F008
:10920000EFEFF0E0E81BF109E65BFB4F8081809314
:109210007601809176018B3010F48AE002C08F3F96
:1092200011F48093760180918B08883F38F0EFEF3E
:10923000F0E0E81BF109E65BFB4F80818093340A84
:109240008091340A863010F485E002C08F3F11F41B
:109250008093340A80918D08883F38F0EFEFF0E07A
:10926000E81BF109E65BFB4F808180935D0A8091EA
:109270005D0A863010F485E002C08F3F11F48093C0
:109280005D0A80917808873F19F4429905C006C0AD
:10929000863F31F4439B02C08CE815C086E413C0BE
:1092A000883F38F0EFEFF0E0E81BF109E65BFB4F99
:1092B00080818093310A8091310A893110F488E1EC
:1092C00002C08F3F11F48093310A80917908873F63
:1092D00019F4429905C006C0863F31F4439B02C091
:1092E0008CE815C086E413C0883F38F0EFEFF0E05B
:1092F000E81BF109E65BFB4F808180930A0A8091AD
:109300000A0A893110F488E102C08F3F11F480937A
:109310000A0A80917A08883F38F0EFEFF0E0E81B06
:10932000F109E65BFB4F808180933A0A80913A0A0B
:10933000893110F488E102C08F3F11F480933A0A1A
:10934000809150080E9473488093260480915308AE
:10935000883F38F0EFEFF0E0E81BF109E65BFB4FE8
:10936000808180937A0180915508883F38F0EFEF33
:10937000F0E0E81BF109E65BFB4F80818093780108
:1093800080915D08883F38F0EFEFF0E0E81BF109CD
:10939000E65BFB4F80818093790180915F08883F75
:1093A00038F0EFEFF0E0E81BF109E65BFB4F80815E
:1093B0008093750180916008883F38F0EFEFF0E00E
:1093C000E81BF109E65BFB4F808180937701809178
:1093D0006108883F38F0EFEFF0E0E81BF109E65B49
:1093E000FB4F80818093740180916208883F38F040
:1093F000EFEFF0E0E81BF109E65BFB4F8081809323
:10940000730180916808883F38F0EFEFF0E0E81BC7
:10941000F109E65BFB4F80818093710180916908BF
:10942000883F38F0EFEFF0E0E81BF109E65BFB4F17
:1094300080818093250480916A08883F38F0EFEF9F
:10944000F0E0E81BF109E65BFB4F80818093240488
:1094500080916B08883F38F0EFEFF0E0E81BF109EE
:10946000E65BFB4F80818093230480916C08883FEA
:1094700038F0EFEFF0E0E81BF109E65BFB4F80818D
:109480008093220480918608883F38F0EFEFF0E067
:10949000E81BF109E65BFB4F8081809321048091FA
:1094A0008708883F38F0EFEFF0E0E81BF109E65B52
:1094B000FB4F80818093200480918808883F38F09A
:1094C000EFEFF0E0E81BF109E65BFB4F8081809352
:1094D0001F0480918908883F38F0EFEFF0E0E81B27
:1094E000F109E65BFB4F808180931E0480916D083B
:1094F000883F38F0EFEFF0E0E81BF109E65BFB4F47
:10950000808180936F0180917108883F38F0EFEF80
:10951000F0E0E81BF109E65BFB4F808180936E0170
:1095200080916E08883F38F0EFEFF0E0E81BF1091A
:10953000E65BFB4F808180936D0180917208883FCC
:1095400038F0EFEFF0E0E81BF109E65BFB4F8081BC
:1095500080936C0180917B08883F38F0EFEFF0E05A
:10956000E81BF109E65BFB4F808180936B018091E2
:109570007E08883F38F0EFEFF0E0E81BF109E65B8A
:10958000FB4F808180936A0180917F08883F38F08B
:10959000EFEFF0E0E81BF109E65BFB4F8081809381
:1095A000690180918008883F38F0EFEFF0E0E81B18
:1095B000F109E65BFB4F8081809368018091A808E8
:1095C000883F38F0EFEFF0E0E81BF109E65BFB4F76
:1095D00080818093190A90912505992321F080912B
:1095E000190A981720F08091190A882311F4909392
:1095F000190A80914D088093560A8091B208809391
:10960000390A80918508883F38F0EFEFF0E0E81BD9
:10961000F109E65BFB4F8081809367018091A1088F
:10962000883F38F0EFEFF0E0E81BF109E65BFB4F15
:10963000808180936D0A80917101282F33272F5FDD
:109640003F4F8CE398E2B9010E94C09F70937E0166
:1096500060937D0180915B0880935E0A80915A0837
:109660008093210AE091A308EE2309F449C081E028
:1096700080931D04FF27EE0FFF1FE858F64F8081EF
:109680009181805C9F4F14F410921D0480917F01A2
:1096900020911D04821721F18330F8F43091AC0140
:1096A000222351F08CED95E090931E0380931D03CF
:1096B000332369F48EE209C088EC90E090931E0396
:1096C00080931D03332319F487E18093AC0185E077
:1096D0008093330420937F0103C0815080937F01E6
:1096E0008091AD0A9091AE0A97FF0FC080911D0442
:1096F000882359F08091B50580688093B50505C031
:10970000E0931D048AE080937F018091AD0A9091DF
:10971000AE0A97FF1DC0809148048823C9F080914C
:109720001D048823A9F080910B0190910C018F5F9B
:109730009F4F71F488E99AE390931E0380931D0371
:1097400080E094EA90930C0180930B0110921D0429
:1097500080911D04882321F080910F04816003C053
:1097600080910F048E7F80930F04DF91CF91089535
:10977000A7E1B0E0EEEBFBE40C9410A00E947F4068
:1097800080911004992784719070892B91F58091B4
:10979000B30882FF27C080912D0490912E0400977A
:1097A000F1F002E088359007D4F49C0197FF02C0E5
:1097B0002D5F3F4F35952795359527958091650805
:1097C0009927289FA001299F500D389F500D1124E3
:1097D000CA0164E670E00E94C09FCB0106C08DE222
:1097E00090E003C080916508992790930E048093C0
:1097F0000D0420910B0430910C0455E720333507FC
:1098000059F410925404109253048091210A99271C
:1098100090930E0480930D0460915304709154044E
:109820007A8369838091210A99270A9668177907B4
:1098300014F49A83898380914904843608F06AC0BD
:1098400080910F0482FD66C08091E9049091EA0442
:10985000009731F001979093EA048093E9040BC0DC
:109860001092480490931204809311048091100484
:109870008D7E80931004809103018A3011F0843131
:1098800010F0289A01C02898809111049091120438
:10989000895E9340E0F18091F10A8536C0F18091B4
:1098A0000D0490910E049A83898380911004806145
:1098B0008093100480914108A82FBB27AA0FBB1FDB
:1098C000FD01E254F64F1182108280914208282F48
:1098D0003327220F331FC9018254964FFC01118296
:1098E0001082A858B64F11961C921E922858364FD7
:1098F000D90111961C921E9280914408E82FFF27EF
:10990000EE0FFF1FE858F64F11821082B4C5109277
:109910004804B1C5809149048D3808F482C59091FE
:10992000AC08992309F445C08091AD08882309F457
:1099300040C0E92FFF27EE0FFF1FE858F64F808148
:109940009181C397BCF080919401823361F480913E
:109950000F0485FF08C080910F04806480930F047A
:1099600080E38093AC0180910F048F7780930F0484
:1099700086E917C0808191818E5C9F4FACF4809105
:109980009401863941F480910F04806880930F041C
:109990008FE28093AC0180910F048F7B80930F0442
:1099A00082E38093940105C080910F048F738093AC
:1099B0000F04809110048F7E8093100490916608AC
:1099C00082E3989FC00111249093EA048093E904F4
:1099D000E981FA81B9978CF080914804882369F075
:1099E0008091110490911204FFEF8F3F9F0729F09F
:1099F00001969093120480931104409111045091A8
:109A000012044F3F510509F048F510926B04109273
:109A10006C0410926D0410926E0410926704109200
:109A200068041092690410926A041092D50410928E
:109A3000D6041092D7041092D80410927304109296
:109A40007404109275041092760480910F04806261
:109A500080930F0484E68093940135C180911004B3
:109A600082608093100480910F0485FF98C08091DC
:109A7000260599279C012470307082FD04C08091D6
:109A80000F0486FF2AC0809141018D3331F580910A
:109A90000804882311F180E58093380484EF91E075
:109AA000A0E0B0E08093390490933A04A0933B0483
:109AB000B0933C0480933F0490934004A0934104EE
:109AC000B093420488EE93E09093930180939201C7
:109AD000232B19F08DE08093AC01809129039091A4
:109AE0002A03A0912B03B0912C0387399105A1057E
:109AF000B1058CF48091430490914404A0914504F5
:109B0000B0914604825A9E4FAF4FBF4F24F08091D0
:109B1000560A80FD21C088EE93E0909393018093D4
:109B2000920180910F0486FF0FC0109238048CE2DE
:109B300091E0A0E0B0E080933F0490934004A093B4
:109B40004104B093420403C080E38093AC01809150
:109B50000F048F7180930F0410926B0410926C04A9
:109B600010926D0410926E041092670410926804B3
:109B70001092690410926A04109273041092740493
:109B80001092750410927604495E534008F49BC00D
:109B900088EE93E0909312048093110494C0809116
:109BA0000F0487FF1AC080914101863711F08D3371
:109BB000A1F480910804882381F08091AD088093FE
:109BC000380480EE91EBAFEFBFEF809339049093B0
:109BD0003A04A0933B04B0933C042091920130914D
:109BE000930143E0283E340708F048C02F5F3F4F01
:109BF000309393012093920110926B0410926C04A5
:109C000010926D0410926E04109267041092680412
:109C10001092690410926A041092730410927404F2
:109C200010927504109276048091290390912A0372
:109C3000A0912B03B0912C038C529140A040B040D6
:109C400080933F0490934004A0934104B093420456
:109C5000285E3340C1F580910F0487FF34C08091A6
:109C600041018B3281F180910F048F7780930F0433
:109C700080910F04806280930F0425C080910804B6
:109C8000882309F180914101863711F08D32D9F492
:109C90008091430490914404A0914504B0914604FE
:109CA000885E9340A040B04074F48091E0079091AA
:109CB000E1078D5A93403CF010929301109292016B
:109CC0008EE08093AC0180914308E82FFF27EE0FD0
:109CD000FF1FE858F64F80819181813591050CF482
:109CE00054C120914804222309F04FC180914408B7
:109CF000E82FFF27EE0FFF1FE858F64F8081918174
:109D00008C3491050CF411C18091EB048F5F80932A
:109D1000EB04893C08F439C12093EB04109212043F
:109D20001092110430914108E32FFF27EE0FFF1F1F
:109D3000E858F64F8081918187349105B4F4809181
:109D40004208E82FFF27EE0FFF1FE858F64F8081EB
:109D500091810190F081E02DF7FF03C0F095E1952E
:109D6000FF4FE734F1050CF478C041E02091420840
:109D7000A22FBB27AA0FBB1FA858B64F8D919C914D
:109D800011978734910544F0E32FFF27EE0FFF1F53
:109D9000E858F64F808191818D919C91873491058F
:109DA00074F080914108E82FFF27EE0FFF1FE8585D
:109DB000F64F80819181873491050CF042E0E22FCB
:109DC000FF27EE0FFF1FE858F64F80819181863400
:109DD000910574F480914108E82FFF27EE0FFF1FD3
:109DE000E858F64F80819181873491050CF043E06B
:109DF000E22FFF27EE0FFF1FE858F64F8081918179
:109E00008A5B9F4F74F480914108E82FFF27EE0F83
:109E1000FF1FE858F64F80819181873491050CF03F
:109E200044E0E22FFF27EE0FFF1FE858F64F808136
:109E300091818A5B9F4F74F480914108E82FFF273E
:109E4000EE0FFF1FE858F64F80819181863491050F
:109E50000CF445E0842F0E94313180914208E82FB4
:109E6000FF27EE0FFF1FE858F64F80819181019088
:109E7000F081E02DF7FF03C0F095E195FF4F7E974D
:109E8000CCF480914108E82FFF27EE0FFF1FE85820
:109E9000F64F808191818A5B9F4F64F481E08093CB
:109EA000D0051092340488EE93E090931E038093C3
:109EB0001D036BC0809101010E94DC3080E00E9494
:109EC000630A809167080E94B09A8091560A80FFC9
:109ED00010C080911C0190911D01875B934038F464
:109EE00080911C0190911D018E5E924010F40E94A1
:109EF000221F81E00E94083D982F8093340421E0C6
:109F000020931B03579A8091B505882311F087E0B1
:109F100006C0992319F42093AC0103C088E1809313
:109F2000AC0185E08093520527C080819181855BDB
:109F30009F4F4CF58091EB048F5F8093EB04893C3D
:109F400020F1209348042093EB0410921204109205
:109F5000110482E00E94083D982F80933404809180
:109F6000B505882311F087E005C0992311F481E03D
:109F700001C088E18093AC0168E770E08091010145
:109F80000E94243C02C02093EB0480914308E82FF8
:109F9000FF27EE0FFF1FE858F64F808191818C5903
:109FA0009F4F0CF037C22091A408E22FFF27EF77D4
:109FB000F070EE0FFF1FE254F64F808191810697FB
:109FC00014F084E606C0808191818B5F9F4F1CF462
:109FD0008CE98093EE0480914804E0914408882342
:109FE00009F063C1FF27EE0FFF1FE858F64F80818D
:109FF00091818C599F4F9CF48091B30883FD0BC0D5
:10A00000E22FFF27EE0FFF1FE858F64F8081918166
:10A01000855B9F4FDCF08091A4088823B9F0809184
:10A02000B30883FF3FC18091A408E82FFF27EE0FFC
:10A03000FF1FE858F64F80819181875F9F4F0CF496
:10A0400031C18091EE04843609F02CC18091340432
:10A05000882329F0809110048860809310048091F7
:10A060001E0190911F01A0912001B09121018093C8
:10A07000E2079093E307A093E407B093E5071092FB
:10A08000290310922A0310922B0310922C03109292
:10A090004304109244041092450410924604109216
:10A0A00036031092370310923803109239038091CF
:10A0B0004108E82FFF27EE0FFF1FE858F64F808179
:10A0C00091818D599F4FACF480914208E82FFF2772
:10A0D000EE0FFF1FE858F64F808191810190F081CB
:10A0E000E02DF7FF03C0F095E195FF4FE436F10551
:10A0F00034F48091A408882311F48093EC048091B7
:10A10000EC048F5F8093EC048E3F08F466C180916D
:10A110005F0A9091600A97FF03C0909581959F4FC9
:10A120008197B4F480911C0A90911D0A97FF03C097
:10A13000909581959F4F45975CF480910D0A909181
:10A140000E0A97FF03C0909581959F4F459714F095
:10A15000109234041092EC048091B505882309F024
:10A1600094C080913404882309F48FC080912A051B
:10A17000882309F08AC081E090E0909312048093D4
:10A18000110481E0809348041092D5041092D60403
:10A190001092D7041092D804109273041092740491
:10A1A000109275041092760410926F04109270044D
:10A1B000109271041092720480915C08E82EFF24C2
:10A1C0000027112780915A0A90915B0A9C0144272D
:10A1D00037FD4095542FC801B7010E94819FDC01D3
:10A1E000CB018093830490938404A0938504B0935F
:10A1F000860480916A0A90916B0A9C01442737FD7E
:10A200004095542FC801B7010E94819FDC01CB010A
:10A2100080937B0490937C04A0937D04B0937E0490
:10A220008091A3049091A404A091A504B091A604E8
:10A2300080937F0490938004A0938104B093820460
:10A2400080919B0490919C04A0919D04B0919E04E8
:10A250008093770490937804A0937904B0937A0460
:10A2600010926B0410926C0410926D0410926E04A4
:10A2700010926704109268041092690410926A04A4
:10A2800084E68093330484E39AC08CED95E0909348
:10A290001E0380931D0380913404882309F09DC020
:10A2A00081E08DC01092EC0498C0FF27EE0FFF1FD5
:10A2B000E858F64F80819181853691059CF0809118
:10A2C000B30883FD0BC0E22FFF27EE0FFF1FE858F6
:10A2D000F64F80819181855B9F4FDCF08091A408CF
:10A2E0008823B9F08091B30883FF75C08091A408DA
:10A2F000E82FFF27EE0FFF1FE858F64F808191816E
:10A300008E5C9F4F0CF067C08091EE048C3909F091
:10A3100062C080914108E82FFF27EE0FFF1FE85829
:10A32000F64F808191818D599F4FACF48091420806
:10A33000E82FFF27EE0FFF1FE858F64F808191812D
:10A340000190F081E02DF7FF03C0F095E195FF4FFC
:10A35000E436F1053CF48091A408882319F4809335
:10A36000ED0418C010926B0410926C0410926D04EE
:10A3700010926E041092670410926804109269049F
:10A3800010926A0410925A041092590410925804C0
:10A39000109257048091ED048F5F8093ED048B3F02
:10A3A00088F0109248041092ED041092120410925A
:10A3B000110480910F048F7180930F0486E28093C3
:10A3C000AC010BC0843649F48CEA9DE090931E03E7
:10A3D00080931D0302C01092ED0420910B04309174
:10A3E0000C04F3E0283E3F0708F045C0809133039A
:10A3F000909134038B569F4F1CF02F5F3F4F05C049
:10A4000021153105C1F12150304030930C042093C7
:10A410000B0431C01092EE0410920C0410920B0445
:10A420002AC02E5E324038F18091750A9091760AEA
:10A430008059914000F58091430490914404A0918B
:10A440004504B09146048C5D9540A040B0409CF41A
:10A4500080E395E790930C0480930B0480911104A2
:10A46000909112048A5E934030F089EE93E09093CD
:10A470001204809311048091400181508093400127
:10A48000809140018F3F21F08091100484FFDFC351
:10A490000E948F48B09057088091F7049091F8047B
:10A4A0009C01220F331F280F391FC0904108AC2D8B
:10A4B000BB27AA0FBB1FFD01E858F64F4B2D5527B0
:10A4C00080819181849FB001859F700D949F700D54
:10A4D0001124260F371F37FF02C02D5F3F4FB901F0
:10A4E0007595679575956795A254B64F80915808F4
:10A4F000082F11278D919C91809FD001819FB00DD5
:10A50000909FB00D11246A0F7B1F7093F804609325
:10A51000F7048091F9049091FA049C01220F331FF3
:10A52000280F391FD0904208AD2DBB27AA0FBB1FA3
:10A53000FD01E858F64F80819181849FF001859F4D
:10A54000F00D949FF00D11242E0F3F1F37FF02C016
:10A550002D5F3F4FA9015595479555954795A254B5
:10A56000B64F8D919C91809F7001819FF00C909FC0
:10A57000F00C11244E0D5F1D5093FA044093F90422
:10A5800080911D04882309F448C0CB0177FD039610
:10A59000DC01B595A795B595A795CA0157FD03961A
:10A5A000FC01F595E795F595E7958091A501682F54
:10A5B000772767FD70956A9F90016B9F300D7A9F9A
:10A5C000300D112480912C05482F552747FD5095BB
:10A5D0004E9FC0014F9F900D5E9F900D1124280F3C
:10A5E000391F37FF02C0295F3F4F03E0359527959C
:10A5F0000A95E1F730935A04209359046E9F900115
:10A600006F9F300D7E9F300D11244A9FC0014B9FDC
:10A61000900D5A9F900D11243FC08091A208E82F01
:10A62000FF27E85BFE4F86818093A5019081909380
:10A630002C05A82FBB27A7FDB095A69F9001A79F2B
:10A64000300DB69F300D1124E92FFF27E7FDF0955F
:10A65000E49FC001E59F900DF49F900D1124280FF9
:10A66000391F37FF02C0295F3F4F13E0359527950B
:10A670001A95E1F730935A0420935904A49F90014E
:10A68000A59F300DB49F300D1124E69FC001E79FB8
:10A69000900DF69F900D1124281B390B37FF02C037
:10A6A000295F3F4F43E0359527954A95E1F7309371
:10A6B00058042093570480914408E82FFF27EE0F99
:10A6C000FF1FE858F64F80819181909581959F4FAB
:10A6D00090935604809355048530910514F00497A7
:10A6E00005C00FEF8C3F900734F404969093560406
:10A6F0008093550404C01092560410925504809122
:10A700000B0490910C048150924078F1809159048F
:10A7100090915A0497FD079623E0959587952A9581
:10A72000E1F790935A0480935904809157049091D3
:10A73000580497FD079603E0959587950A95E1F7EC
:10A74000909358048093570410926B0410926C04F9
:10A7500010926D0410926E041092670410926804B7
:10A760001092690410926A0443C0809118058823EE
:10A7700009F43EC0282F33278091590490915A0440
:10A7800097FD079613E0959587951A95E1F7289F11
:10A79000A001299F500D389F500D1124CA0157FD6B
:10A7A0000F96B4E095958795BA95E1F790935A0482
:10A7B00080935904809157049091580497FD07960F
:10A7C000A3E095958795AA95E1F7289FB001299F69
:10A7D000700D389F700D1124CB0177FD0F96F4E0BA
:10A7E00095958795FA95E1F79093580480935704CF
:10A7F0008090590490905A0480911B0590911C05FB
:10A80000881A990A90925A04809259040091570428
:10A81000109158048091190590911A05081B190B85
:10A82000109358040093570480914308E82FFF27A2
:10A83000EE0FFF1FE858F64FE080F1808FE790E0C1
:10A84000E80EF91EF0925404E092530480917601D0
:10A850009927AA2797FDA095BA2FBC01CD010E9488
:10A86000F59EDC01CB0120E030E040E251E4BC0188
:10A87000CD010E94639EDC01CB01BC01CD010E9491
:10A88000C79EDC01CB018093640A8091750180939F
:10A890003B0A809174019927AA2797FDA095BA2FAA
:10A8A000BC01CD010E94F59EDC01CB0120E030E02F
:10A8B00040E251E4BC01CD010E94639EDC01CB016A
:10A8C000BC01CD010E94C79EDC01CB018093140A1C
:10A8D0008091730180932A0A8091DC0580FF59C022
:10A8E00080916D0A813808F454C08091D50599276C
:10A8F00087FD90952B2D3327829FD001839FB00D2C
:10A90000929FB00D11248A0E9B1E90925A04809241
:10A9100059048091D605992787FD9095829FF00173
:10A92000839FF00D929FF00D11240E0F1F1F1093A7
:10A930005804009357048091D705282F332727FD0B
:10A9400030958091550490915604820F931F9093F7
:10A950005604809355048091D905282F332727FD6D
:10A960003095809152089927289F8001299F100DCA
:10A97000389F100D112410934701009346018091D8
:10A98000D80599278E159F0524F49093540480933D
:10A990005304809153049091540497FF04C0109283
:10A9A0005404109253048091560A82FF02C0109200
:10A9B0003B0A4091590450915A04CA0157FD03962D
:10A9C0009C01359527953595279537FF03C0309520
:10A9D00021953F4F8091150490911604821793079B
:10A9E000B4F4CA0157FF03C0909581959F4F97FD1E
:10A9F00003969595879595958795909316048093E2
:10AA000015048536910544F084E690E001C0019775
:10AA10009093160480931504409157045091580464
:10AA2000CA0157FD03969C013595279535952795C5
:10AA300037FF03C0309521953F4F809113049091CB
:10AA4000140482179307B4F4CA0157FF03C090950A
:10AA500081959F4F97FD0396959587959595879539
:10AA600090931404809313048536910544F084E692
:10AA700090E001C001979093140480931304809197
:10AA8000100484FF08C0109216041092150410924E
:10AA9000140410921304ED2DFF27EE0FFF1FE8584A
:10AAA000F64F40917C08242F33278081918128170D
:10AAB000390744F48091B00882FF04C081E080939C
:10AAC0002A0413C0ED2DFF27EE0FFF1FE858F64FA5
:10AAD000842F992720917D08821B91092081318143
:10AAE0002817390714F410922A0440914208E42FE1
:10AAF000FF27EE0FFF1FE858F64F50917C08852F77
:10AB0000992722273327281B390B808191818217AF
:10AB1000930744F48091B00883FF04C081E08093E0
:10AB2000290416C080912904882391F0E42FFF277F
:10AB3000EE0FFF1FE858F64F80917D089927851B7F
:10AB40009109208131818217930714F4109229040E
:10AB5000EC2DFF27EE0FFF1FE858F64F40917C08C1
:10AB6000242F3327808191812817390744F480915D
:10AB7000B00880FF04C081E08093270417C0809153
:10AB80002704882399F0EC2DFF27EE0FFF1FE858CC
:10AB9000F64F842F992720917D08821B91092081EF
:10ABA00031812817390714F4109227044091410885
:10ABB000E42FFF27EE0FFF1FE858F64F50917C0857
:10ABC000852F992722273327281B390B80819181D4
:10ABD0008217930744F48091B00881FF04C081E09C
:10ABE0008093280416C080912804882391F0E42FD4
:10ABF000FF27EE0FFF1FE858F64F80917D08992739
:10AC0000851B9109208131818217930714F41092DA
:10AC1000280480912A04882319F480912904811141
:10AC200081E080932B0480912704882321F4809174
:10AC30002804882351F081E080932C0410922B0487
:10AC400010922A041092290402C080932C0480914F
:10AC50002B04882321F480912C04882369F08091AF
:10AC60007B08992729813A818217930714F49A83E4
:10AC7000898381E080935F0480910F0499279C0170
:10AC80002470307082FF2DC080911B0590911C05AF
:10AC9000909581959F4F90935A0480935904809189
:10ACA000190590911A05909581959F4F909358049E
:10ACB0008093570480918201909183019093540472
:10ACC000809353048091560A8B778B668093560A43
:10ACD0008091390A8C7B8093390A88EC8093260412
:10ACE0001EC08091100484FF1AC030935604209334
:10ACF000550430935A0420935904309358042093F8
:10AD000057049AE59093640A88E780933B0A9093EE
:10AD1000140A80932A0A10922B0410922C0480911A
:10AD20002D0A90912E0AA0912F0AB091300A2091FD
:10AD3000A3043091A4044091A5045091A604820F6D
:10AD4000931FA41FB51F80932D0A90932E0AA093E2
:10AD50002F0AB093300A8091350A9091360AA0915B
:10AD6000370AB091380AE0909B04F0909C0400915F
:10AD70009D0410919E04EB82FC820D831E838E0D38
:10AD80009F1DA01FB11F8093350A9093360AA09390
:10AD9000370AB093380A8091220A9091230AA09131
:10ADA000240AB091250AE0909F04F090A00400913D
:10ADB000A1041091A204EF82F88609871A878E0DEC
:10ADC0009F1DA01FB11F8093220A9093230AA09376
:10ADD000240AB093250A8091150A9091160AA09131
:10ADE000170AB091180AE0909704F0909804009127
:10ADF000990410919A04EB86FC860D871E878E0DB0
:10AE00009F1DA01FB11F8093150A9093160AA0934F
:10AE1000170AB093180AF0902C04FF86FF2029F43B
:10AE200080912B04882309F460C01092930410923F
:10AE30009404109295041092960410928F0410922C
:10AE40009004109291041092920410922D0A109284
:10AE50002E0A10922F0A1092300A1092350A109280
:10AE6000360A1092370A1092380A1092220A10926B
:10AE7000230A1092240A1092250A1092150A1092A1
:10AE8000160A1092170A1092180A80918304909162
:10AE90008404A0918504B091860480937F049093EC
:10AEA0008004A0938104B093820480917B049091EC
:10AEB0007C04A0917D04B0917E04809377049093EC
:10AEC0007804A0937904B0937A041092320310921C
:10AED00031031092300410922F0410923204109219
:10AEE00031040F85002309F0D0C180912B04882301
:10AEF00009F0CBC18091E0079091E1078150924029
:10AF00002CF480914804882309F4BFC19090E60A8C
:10AF1000A0905C0820905A0A30905B0A40906A0A20
:10AF200050906B0A19140CF0BBC0BB24CC24DD2458
:10AF3000CA01B901A60195010E94F59F79018A0114
:10AF40008091AF0A9091B00A281A390AC101AA2744
:10AF500097FDA095BA2FE81AF90A0A0B1B0B6B8113
:10AF60007C818D819E81A60195010E94F59F5901EA
:10AF70006A018091B10A9091B20A481A590AC20135
:10AF8000AA2797FDA095BA2FA81AB90ACA0ADB0A00
:10AF9000292C332427FC3094432C532CC801B701AF
:10AFA000A20191010E94819F97FF04C061507E4FD2
:10AFB0008F4F9F4F3B014C0109E095948794779404
:10AFC00067940A95D1F7C601B501A20191010E94CB
:10AFD000819F97FF04C061507E4F8F4F9F4F5B0151
:10AFE0006C0119E0D594C794B794A7941A95D1F73A
:10AFF0008091150490911604813491053CF4809160
:10B0000013049091140481349105D4F0D401C30148
:10B0100097FE03C00196A11DB11D3C014D01959401
:10B02000879477946794D601C501D7FE03C0019633
:10B03000A11DB11D5C016D01D594C794B794A7946F
:10B040008091E80A282F332727FD3095432F532F6F
:10B05000261537054805590514F439014A01992781
:10B0600087FD9095909581959F4FAA2797FDA09574
:10B07000BA2F681679068A069B0614F43C014D0126
:10B080002A153B054C055D0514F459016A01A81603
:10B09000B906CA06DB060CF0D0C05C016D01CDC05C
:10B0A000EA2CFF2400271127CA01B901A801970142
:10B0B0000E94F59F39014A01C101AA2797FDA09579
:10B0C000BA2F681A790A8A0A9B0A6B817C818D8162
:10B0D0009E81A80197010E94F59F59016A01C20152
:10B0E000AA2797FDA095BA2FA81AB90ACA0ADB0A9F
:10B0F000D401C30197FE03C00F96A11DB11D3C01F1
:10B100004D01F4E09594879477946794FA95D1F77C
:10B11000D601C501D7FE03C00F96A11DB11D5C016C
:10B120006D01E4E0D594C794B794A794EA95D1F75C
:10B130008091150490911604813491053CF480911E
:10B1400013049091140481349105A4F0C401B30157
:10B1500023E030E040E050E00E94F59F39014A01D1
:10B16000C601B50123E030E040E050E00E94F59FC9
:10B1700059016A0180914408E82FFF27EE0FFF1F55
:10B18000E858F64F808191810190F081E02DF7FF22
:10B1900003C0F095E195FF4F7A97A4F0C401B30185
:10B1A00023E030E040E050E00E94F59F39014A0181
:10B1B000C601B50123E030E040E050E00E94F59F79
:10B1C00059016A0189E180938E0121E262167104BE
:10B1D000810491042CF070E2672E712C812C912C4B
:10B1E00030EE63163FEF73063FEF83063FEF9306A3
:10B1F00044F460EE662E6FEF762E6FEF862E6FEFC3
:10B20000962E41E2A416B104C104D1042CF050E200
:10B21000A52EB12CC12CD12C50EEA5165FEFB50692
:10B220005FEFC5065FEFD50644F440EEA42E4FEF66
:10B23000B42E4FEFC42E4FEFD42E80918304909103
:10B240008404A0918504B091860486199709A80901
:10B25000B9098093830490938404A0938504B093E8
:10B26000860480917B0490917C04A0917D04B09130
:10B270007E048A199B09AC09BD0980937B049093D5
:10B280007C04A0937D04B0937E048091310390915F
:10B2900032038F3F910509F008F4C4C56F8566231A
:10B2A00009F04EC580912B04882309F049C580918F
:10B2B0005F04882309F044C570918408788B772354
:10B2C00009F43EC580912D0A90912E0AA0912F0A73
:10B2D000B091300AB7FF04C081509F4FAF4FBF4FAE
:10B2E000E92EFA2E0B2F112707FD1A95E0922D0A51
:10B2F000F0922E0A00932F0A1093300A8091350A9B
:10B300009091360AA091370AB091380AB7FF04C06D
:10B3100081509F4FAF4FBF4F892F9A2FAB2FBB2725
:10B32000A7FDBA95898B9A8BAB8BBC8B8093350A22
:10B330009093360AA093370AB093380A80915C083C
:10B34000A82EBB24CC24DD242091930430919404B6
:10B350004091950450919604C601B5010E94819FC9
:10B3600097FF04C061507F4F8F4F9F4F672E782EFD
:10B37000892E992487FC9A94609293047092940485
:10B38000809295049092960420918F0430919004BD
:10B390004091910450919204C601B5010E94819F91
:10B3A00097FF04C061507F4F8F4F9F4F272E382E3D
:10B3B000492E552447FC5A9420928F0430929004D1
:10B3C000409291045092920480918B0490918C044D
:10B3D000A0918D04B0918E04B7FF04C081509F4F9F
:10B3E000AF4FBF4F892F9A2FAB2FBB27A7FDBA9521
:10B3F00080938B0490938C04A0938D04B0938E045F
:10B40000D801C70186199709A809B9098093E104F1
:10B410009093E204A093E304B093E40420918308A2
:10B42000E22EFF2400271127BC01CD01A8019701BE
:10B430000E94F59F59016A012093EF043093F004B4
:10B440004093F1045093F20489899A89AB89BC89AD
:10B4500082199309A409B5098093E5049093E60441
:10B46000A093E704B093E804BC01CD01A8019701C3
:10B470000E94F59F2093F3043093F4044093F50465
:10B480005093F604D601C501D7FE04C081509F4FEA
:10B49000AF4FBF4F892F9A2FAB2FBB27A7FDBA9570
:10B4A0009093300480932F0457FF04C021503F4FE6
:10B4B0004F4F5F4FBB2757FDBA95A52F942F832F72
:10B4C0009093320480933104809115049091160476
:10B4D00081349105DCF4809113049091140481343B
:10B4E0009105A4F480914408E82FFF27EE0FFF1F79
:10B4F000E858F64F808191810190F081E02DF7FFAF
:10B5000003C0F095E195FF4F7A97E4F08091E60A49
:10B510008F3FC1F480912F049091300497FD0196E4
:10B52000959587959093300480932F0480913104F2
:10B530009091320497FD01969595879590933204EA
:10B54000809331048091220A9091230AA091240AC9
:10B55000B091250AB7FF04C081509F4FAF4FBF4F36
:10B56000892F9A2FAB2FBB27A7FDBA958093220A6C
:10B570009093230AA093240AB093250A8091150A78
:10B580009091160AA091170AB091180AB7FF04C04B
:10B5900081509F4FAF4FBF4F892F9A2FAB2FBB27A3
:10B5A000A7FDBA958093150A9093160AA093170ADF
:10B5B000B093180A8091A3049091A404A091A504CB
:10B5C000B091A6042F81388549855A85281B390BEF
:10B5D0004A0B5B0B2093D9043093DA044093DB04CD
:10B5E0005093DC0480919B0490919C04A0919D0455
:10B5F000B0919E04EB84FC840D851E85E81AF90A3F
:10B600000A0B1B0BE092DD04F092DE040093DF04D2
:10B610001093E0042093E1043093E2044093E304A8
:10B620005093E404E092E504F092E6040093E7040A
:10B630001093E80480917F0490918004A09181048C
:10B64000B0918204821B930BA40BB50B80937F04F3
:10B6500090938004A0938104B09382048091770436
:10B6600090917804A0917904B0917A048E199F0981
:10B67000A00BB10B8093770490937804A093790486
:10B68000B0937A0488898823E1F020915D04309199
:10B690005E04213831054CF08091B5049091B604D8
:10B6A00001969093B6048093B50420583F4F4CF414
:10B6B0008091B5049091B60401979093B60480935D
:10B6C000B50410925E0410925D0481E090E09093C6
:10B6D000FC048093FB04E090E104F090E20400910C
:10B6E000E3041091E404D801C70117FF07C08827BD
:10B6F0009927DC018E199F09A00BB10B8150924054
:10B70000A040B04034F084E090E09093FC0480933B
:10B71000FB048091010590910205A0910305B09171
:10B72000040520912D0A30912E0A40912F0A509144
:10B73000300A821B930BA40BB50B815E914BAF4F6C
:10B74000BF4F8F539C49A040B04028F08091E70A3A
:10B7500089310CF4FFC021E0E21620E1F20620E07E
:10B76000020720E012070CF473C08091FD048823C7
:10B7700009F46AC0D801C70117FF07C088279927B5
:10B78000DC018E199F09A00BB10B9C01AD01B7FF25
:10B7900004C021503E4F4F4F5F4FF9E055954795FC
:10B7A00037952795FA95D1F78091FB049091FC0489
:10B7B000820F931F9093FC048093FB04D801C70170
:10B7C00017FF03C00796A11DB11DE3E0B595A7952E
:10B7D00097958795EA95D1F78093EF049093F004BD
:10B7E000A093F104B093F20489589341A040B04073
:10B7F00064F088E893E1A0E0B0E08093EF049093D8
:10B80000F004A093F104B093F2042091EF0430917E
:10B81000F0044091F1045091F20457FF04C021500C
:10B820003F4F4F4F5F4F232F342F452F552747FD55
:10B830005A9580912F0490913004820F931F90931A
:10B84000300480932F0406C081E08093FD0402C081
:10B850001092FD0440E0E41640EFF4064FEF0407B9
:10B860004FEF14070CF073C08091FE04882309F495
:10B870006AC0D801C70117FF07C088279927DC01D4
:10B880008E199F09A00BB10B9C01AD01B7FF04C03D
:10B8900021503E4F4F4F5F4F69E055954795379583
:10B8A00027956A95D1F78091FB049091FC04820F53
:10B8B000931F9093FC048093FB04D801C70117FFEA
:10B8C00003C00796A11DB11D23E0B595A7959795D7
:10B8D00087952A95D1F78093EF049093F004A09375
:10B8E000F104B093F20488579C4EAF4FBF4F64F4FD
:10B8F00088E79CEEAFEFBFEF8093EF049093F004E6
:10B90000A093F104B093F2042091EF043091F0047D
:10B910004091F1045091F20457FF04C021503F4F71
:10B920004F4F5F4F232F342F452F552747FD5A95F3
:10B9300080912F0490913004820F931F90933004D4
:10B9400080932F0411C081E08093FE040DC01092FB
:10B95000FE040AC01092FC041092FB0484E690E0FE
:10B9600090938D0180938C016889262F33278091D5
:10B97000FB049091FC042817390724F43093FC044D
:10B980002093FB041091E70A112379F0212F33272C
:10B9900027FD30958091FB049091FC04281739070E
:10B9A00024F43093FC042093FB044091E104509173
:10B9B000E2046091E3047091E404413851056105AB
:10B9C000710574F08091B9049091BA042091FB0440
:10B9D0003091FC04820F931F9093BA048093B904B2
:10B9E00040585F4F6F4F7F4F74F48091B90490912E
:10B9F000BA042091FB043091FC04821B930B9093BA
:10BA0000BA048093B90481E090E09093FC048093A1
:10BA1000FB04C090E504D090E604E090E704F090C9
:10BA2000E804D701C601F7FE07C088279927DC0183
:10BA30008C199D09AE09BF0981509240A040B040C9
:10BA400034F084E090E09093FC048093FB048091B8
:10BA5000050590910605A0910705B0910805209174
:10BA6000350A3091360A4091370A5091380A821BC4
:10BA7000930BA40BB50B815E914BAF4FBF4F8F5310
:10BA80009C49A040B04018F019310CF4FFC001E00F
:10BA9000C01600E1D00600E0E00600E0F0060CF47D
:10BAA00073C08091FF04882309F46AC0D701C601DE
:10BAB000F7FE07C088279927DC018C199D09AE097C
:10BAC000BF099C01AD01B7FF04C021503E4F4F4F4D
:10BAD0005F4F09E055954795379527950A95D1F71A
:10BAE0008091FB049091FC04820F931F9093FC04BF
:10BAF0008093FB04D701C601F7FE03C00796A11D82
:10BB0000B11D13E0B595A795979587951A95D1F72F
:10BB10008093F3049093F404A093F504B093F60497
:10BB200089589341A040B04064F088E893E1A0E0D8
:10BB3000B0E08093F3049093F404A093F504B093E1
:10BB4000F6042091F3043091F4044091F5045091EF
:10BB5000F60457FF04C021503F4F4F4F5F4F232F34
:10BB6000342F452F552747FD5A95809131049091E8
:10BB70003204820F931F909332048093310406C0E5
:10BB800081E08093FF0402C01092FF0420E0C216FF
:10BB900020EFD2062FEFE2062FEFF2060CF073C073
:10BBA00080910005882309F46AC0D701C601F7FE19
:10BBB00007C088279927DC018C199D09AE09BF09A8
:10BBC0009C01AD01B7FF04C021503E4F4F4F5F4F66
:10BBD000E9E05595479537952795EA95D1F78091F6
:10BBE000FB049091FC04820F931F9093FC048093BC
:10BBF000FB04D701C601F7FE03C00796A11DB11DC6
:10BC000073E0B595A795979587957A95D1F7809329
:10BC1000F3049093F404A093F504B093F6048857CA
:10BC20009C4EAF4FBF4F64F488E79CEEAFEFBFEF81
:10BC30008093F3049093F404A093F504B093F60476
:10BC40002091F3043091F4044091F5045091F604EE
:10BC500057FF04C021503F4F4F4F5F4F232F342FCA
:10BC6000452F552747FD5A95809131049091320414
:10BC7000820F931F909332048093310411C081E0AE
:10BC8000809300050DC0109200050AC01092FC04BC
:10BC90001092FB0484E690E090938D0180938C01D8
:10BCA0004889242F33278091FB049091FC042817A6
:10BCB000390724F43093FC042093FB048091E70AB5
:10BCC000882379F0282F332727FD30958091FB04B6
:10BCD0009091FC042817390724F43093FC04209336
:10BCE000FB044091E5045091E6046091E7047091F3
:10BCF000E804413851056105710574F08091B7047D
:10BD00009091B8042091FB043091FC04820F931FA2
:10BD10009093B8048093B70440585F4F6F4F7F4FA4
:10BD2000CCF48091B7049091B8042091FB04309139
:10BD3000FC04821B930B9093B8048093B7040AC051
:10BD400010923204109231041092300410922F0499
:10BD500010925F0480913B0A882341F410923204D0
:10BD6000109231041092300410922F0480912D0A09
:10BD700090912E0AA0912F0AB091300A809301056C
:10BD800090930205A0930305B09304058091350AB2
:10BD90009091360AA091370AB091380A8093050530
:10BDA00090930605A0930705B0930805109293049D
:10BDB00010929404109295041092960410928F049D
:10BDC00010929004109291041092920410928B049D
:10BDD00010928C0410928D0410928E0410922D0AF1
:10BDE00010922E0A10922F0A1092300A1092350AE1
:10BDF0001092360A1092370A1092380A1092220ACC
:10BE00001092230A1092240A1092250A1092150A01
:10BE10001092160A1092170A1092180A1092320302
:10BE200010923103E0905504F0905604C701F7FEDC
:10BE300004C0882799278E199F0904973CF08091A8
:10BE4000560A84FD03C082E380933304109159089D
:10BE5000A12EBB24CC24DD24B701882777FD809553
:10BE6000982F9701F7FE04C0222733272E193F0988
:10BE7000442737FD4095542F0E94819F9B01AC01C0
:10BE8000C601B5010E94819F97FF04C061507E4F9B
:10BE90008F4F9F4F59E095958795779567955A9560
:10BEA000D1F79B01812F99278E9DD0018F9DB00DD9
:10BEB0009E9DB00D1124CD01B7FD039695958795F4
:10BEC00095958795280F391F80910B0490910C044C
:10BED0008150924010F020E030E080913504909144
:10BEE0003604280F391F442737FD4095542F2093DF
:10BEF000D5043093D6044093D7045093D80480914E
:10BF0000730490917404A0917504B0917604821B1F
:10BF1000930BA40BB50B8093730490937404A093BC
:10BF20007504B09376048155934CA040B04064F002
:10BF300080E593ECA0E0B0E08093730490937404E8
:10BF4000A0937504B0937604809173049091740467
:10BF5000A0917504B0917604805B9C43AF4FBF4FB6
:10BF600064F480EB9CE3AFEFBFEF80937304909396
:10BF70007404A0937504B09376040091900110911D
:10BF8000910117FDFCC08091560A83FFF8C0809193
:10BF90008F01815080938F01882309F0F4C08DE0D8
:10BFA00080938F018091A3049091A404A091A50493
:10BFB000B091A604B7FF04C081509E4FAF4FBF4F52
:10BFC00039E0B595A795979587953A95D1F77C0176
:10BFD00097FF04C0F094E194F108F39480919B04DE
:10BFE00090919C04A0919D04B0919E04B7FF04C061
:10BFF00081509E4FAF4FBF4F29E0B595A7959795BC
:10C0000087952A95D1F79C0197FF03C0309521951C
:10C010003F4FE216F3060CF47901B701F7FE02C0B8
:10C02000695F7F4F2B01A3E055944794AA95E1F7F0
:10C0300022E030E0420E531E6090660A7090670A5C
:10C040008090680A9090690A2091420130914301E2
:10C050004091440150914501C401B3010E94F59FF4
:10C0600059016A013093130A2093120A021B130B21
:10C07000C801845E9D4F68E671E00E94C09F9C01EC
:10C08000245B304080918C0190918D01009731F0BC
:10C09000019790938D0180938C011BC049E1E416B8
:10C0A000F104BCF480915D0490915E04820F931FB3
:10C0B00090935E0480935D0480913304882349F05B
:10C0C000815080933304882321F4B0926204A092BB
:10C0D000610480918C0190918D01892BF9F48091FC
:10C0E0008E019927289FB001299F700D389F700DF0
:10C0F0001124CB01B2010E94C09FCB01AA2797FD5A
:10C10000A095BA2F680E791E8A1E9B1E6092660A41
:10C110007092670A8092680A9092690A809133044B
:10C12000882369F580916104909162042091120A3C
:10C130003091130A821B930B845E9D4F68E671E079
:10C140000E94C09F9C01245B3040809179018695BC
:10C150009927289FD001299FB00D389FB00D112439
:10C160009D01B7FF02C0215F3F4FF4E03595279551
:10C17000FA95E1F7309336042093350404C0109209
:10C1800036041092350480915F04882381F0109268
:10C190006704109268041092690410926A04109265
:10C1A0006B0410926C0410926D0410926E04F09067
:10C1B0002C04FF20F1F480913B0A282F33274427D9
:10C1C00055278091A3049091A404A091A504B09157
:10C1D000A604BC01CD010E94819FDC01CB01BC0102
:10C1E000CD0128EF3AE240E050E00E94F59F29019E
:10C1F00002C044245524E0902B04EE20F1F48091F9
:10C200003B0A282F33274427552780919B04909180
:10C210009C04A0919D04B0919E04BC01CD010E949C
:10C22000819FDC01CB01BC01CD0128EF3AE240E067
:10C2300050E00E94F59F190102C02224332480910E
:10C240000F0A9091100A893C91051CF088EC90E04F
:10C2500005C088539F4F34F488E39FEF9093100AF2
:10C2600080930F0A80911A0A90911B0A893C9105CC
:10C270001CF088EC90E005C088539F4F34F488E3AD
:10C280009FEF90931B0A80931A0A80911C0A909149
:10C290001D0AAA2797FDA095BA2F2091640AA22E05
:10C2A000BB24CC24DD24BC01CD01A60195010E9454
:10C2B000819F9B01AC0180910F0A9091100AAA27DF
:10C2C00097FDA095BA2FE7E0880F991FAA1FBB1F03
:10C2D000EA95D1F7280F391F4A1F5B1F57FF04C08B
:10C2E000215C3F4F4F4F5F4F76E05595479537950F
:10C2F00027957A95D1F78201020F131F10931D0A1B
:10C3000000931C0A80910D0A90910E0AAA2797FDAE
:10C31000A095BA2FBC01CD01A60195010E94819F75
:10C320009B01AC0180911A0A90911B0AAA2797FDE4
:10C33000A095BA2F67E0880F991FAA1FBB1F6A95A7
:10C34000D1F7280F391F4A1F5B1F57FF04C0215C1C
:10C350003F4F4F4F5F4FA6E055954795379527952F
:10C36000AA95D1F74101820E931E90920E0A8092F7
:10C370000D0A80915F0A9091600A880F991FAA2781
:10C3800097FDA095BA2F2091140A332744275527EB
:10C39000BC01CD010E94819F5B016C0197FF08C029
:10C3A0002FE330E040E050E0A20EB31EC41ED51EC5
:10C3B000F6E0D594C794B794A794FA95D1F78091F5
:10C3C0002A0A282F332744275527809187049091E4
:10C3D0008804A0918904B0918A04BC01CD010E9417
:10C3E000819FDC01CB01BC01CD0120EF35E540E0B0
:10C3F00050E00E94F59FB501620F731F7093600AB1
:10C4000060935F0A0150104134F080E090E1909316
:10C410001D0A80931C0A80911C0A90911D0A80506D
:10C42000904F34F480E090EF90931D0A80931C0AA3
:10C4300051E0851650E1950634F080E090E190934C
:10C440000E0A80930D0A80910D0A90910E0A805079
:10C45000904F34F480E090EF90930E0A80930D0A91
:10C460006150704134F080E090E19093600A8093D5
:10C470005F0A80915F0A9091600A8050904F34F477
:10C4800080E090EF9093600A80935F0A809110049F
:10C4900085FD16C0809102019927209126013091D7
:10C4A000270149815A81489F8001499F100D589F5B
:10C4B000100D1124C801B9010E94AC9F7A836983D1
:10C4C000809109058150809309058F3F09F047C08D
:10C4D00080910A0590910B05892B41F480912601EA
:10C4E0009091270190930B0580930A058091260176
:10C4F0009091270120910A0530910B0528173907E3
:10C5000018F42F5F3F4F09C08091260190912701B9
:10C510008217930730F42150304030930B0520935D
:10C520000A0584E6809309058091AF08282F3327F8
:10C5300040910A0550910B054217530710F48AE009
:10C540000CC080910001280F311D2417350738F4E5
:10C5500080910704882319F081508093070480910B
:10C5600007048823D1F08091390490913A04A09176
:10C570003B04B0913C04B7FD10C08091AD0880939E
:10C58000380480EE91EBAFEFBFEF809339049093C6
:10C590003A04A0933B04B0933C0469817A81660F0E
:10C5A000771F660F771F7A8369838091560A80FD13
:10C5B00002C00C944F6DEE2011F00C944F6DFF20D3
:10C5C00011F00C944F6D8091B50599278F7790707D
:10C5D000009711F00C944F6D3C018091BB04909139
:10C5E000BC04892B09F044C080911C0190911D016D
:10C5F0008959934058F087B58A3F20F480913503DC
:10C60000815011C081E0809317055EC080911C01AC
:10C6100090911D018436910530F587B58630F8F08C
:10C62000809135038F5F8093350395E089029001F7
:10C6300011248091EC07821B87BD87B5809588BD4A
:10C640008CE291E090931E0380931D038EE591E0B0
:10C650009093BC048093BB040E94EA1E35C081E025
:10C660008093160531C0F0921605F09217052CC084
:10C67000709234036092330380910804882321F080
:10C6800081E00E94E89817C080914304909144048F
:10C69000A0914504B091460454E0880F991FAA1F49
:10C6A000BB1F5A95D1F78093360390933703A0931D
:10C6B0003803B09339038091BB049091BC04019777
:10C6C0009093BC048093BB048091560A2091260469
:10C6D00081FF3CC0223348F58091950181508093C1
:10C6E00095018F3F09F052C08091AC01882339F445
:10C6F00080916004882319F088E28093AC01109245
:10C7000060048091430490914404A0914504B09149
:10C71000460480933F0490934004A0934104B09357
:10C72000420481E08093950131C0273478F18091F3
:10C73000AC01882339F480916004882319F487E2DE
:10C740008093AC0188EC809395011DC080914601D7
:10C7500090914701820F911D209152083327829FAB
:10C76000D001839FB00D929FB00D1124CD01AA2757
:10C7700097FDA095BA2F80933F0490934004A09317
:10C780004104B093420481E0809360048091A3044B
:10C790009091A404A091A504B091A604E090420158
:10C7A000F09043010091440110914501BC01CD017D
:10C7B000A80197010E94F59F59016A0180919B048D
:10C7C00090919C04A0919D04B0919E04BC01CD0168
:10C7D000A80197010E94F59FB901C5010E94A19D82
:10C7E0009093270A8093260ACC9734F08CE390E04C
:10C7F0009093270A8093260A8091260A9091270A0F
:10C800000E94F7799093270A8093260A80E280930A
:10C81000410110923E0410923D04809160048823EF
:10C8200009F4A1C78091100499279C0120713070F0
:10C8300084FD99C780910F04826080930F047091EA
:10C84000390A872F992741E0842E912C882299223A
:10C8500080FD04C08091560A81FD10C0E980FA80F5
:10C8600030930D0520930C0530933E0420933D0436
:10C8700080911004806C8093100410C38091100488
:10C8800081FFDFC20091820110918301C8010F96E0
:10C89000E0915304F0915404FF8BEE8B8E179F07A9
:10C8A0000CF09AC080911605882309F095C08091FC
:10C8B000100487FF15C0809110048F7780931004B7
:10C8C0008091290390912A03A0912B03B0912C030E
:10C8D00080933F0490934004A0934104B09342049A
:10C8E000E090190AEE20D9F180913F049091400424
:10C8F000A0914104B0914204BC01CD0124E630E096
:10C9000040E050E00E94F59FAE2CBB24CC24DD24F7
:10C91000A216B306C406D50614F590923E04809282
:10C920003D048091AC018823C1F48091430490912F
:10C930004404A0914504B0914604BC01CD012FE50B
:10C9400030E040E050E00E94F59FA216B306C40616
:10C95000D5061CF48AE18093AC018DE338C0809148
:10C960000E0590910F05459784F0809129039091D1
:10C970002A03A0912B03B0912C0380933F04909342
:10C980004004A0934104B093420480911004806459
:10C99000809310042E893F89201B310B2F5030408B
:10C9A00037FF03C0309521953F4F30933E042093CD
:10C9B0003D0480910704882349F0C90163E070E0D9
:10C9C0000E94C09F70933E0460933D048BE280936D
:10C9D00041011092370437C1C8010F97EE88FF88D4
:10C9E000E816F906CCF5209117052223A9F58091C8
:10C9F000100486FF15C0809110048F7B8093100473
:10CA00008091290390912A03A0912B03B0912C03CC
:10CA100080933F0490934004A0934104B093420458
:10CA2000809110048068809310048E899F89801BF8
:10CA3000910B0F9697FF03C0909581959F4F90950E
:10CA400081959F4F90933E0480933D048DE28093A7
:10CA5000410120933704F7C08DE380934101609139
:10CA60003804662371F12091390430913A044091E1
:10CA70003B0450913C0480913F0490914004A0916C
:10CA80004104B091420482179307A407B507CCF480
:10CA900080911004806480931004862F99279093CE
:10CAA0003E0480933D048AE0809337048EE58093B2
:10CAB00041018091100487FFC6C0809110048F77D8
:10CAC00033C0662309F443C02091390430913A04FD
:10CAD00040913B0450913C0480913F04909140046C
:10CAE000A0914104B0914204281739074A075B0717
:10CAF00074F580911004806880931004862F992724
:10CB0000909581959F4F90933E0480933D0486EFCE
:10CB10008093370486E7809341018091100486FF5B
:10CB200092C0809110048F7B809310048091290320
:10CB300090912A03A0912B03B0912C0380933F0482
:10CB400090934004A0934104B09342047CC0809130
:10CB50001004807C09F477C080913704882309F0A1
:10CB60004CC08091290390912A03A0912B03B0918E
:10CB70002C03885C9040A040B04020913F0430914D
:10CB80004004409141045091420482179307A40746
:10CB9000B5076CF08091290390912A03A0912B0393
:10CBA000B0912C03885C9040A040B0401DC08091A3
:10CBB000290390912A03A0912B03B0912C03885351
:10CBC0009F4FAF4FBF4F281739074A075B07BCF08D
:10CBD0008091290390912A03A0912B03B0912C03FB
:10CBE00088539F4FAF4FBF4F80933F0490934004B3
:10CBF000A0934104B093420402C010923704809184
:10CC000010048F738093100410920D0510920C0580
:10CC100071FF06C084EF91E090931E0380931D0383
:10CC200080914704882379F48091430490914404CF
:10CC3000A0914504B0914604C397A105B1051CF02D
:10CC400081E08093470460910C0570910D058091FF
:10CC50003D0490913E04680F791F70930D05609319
:10CC60000C05CB0177FF04C088279927861B970BFB
:10CC7000855F91400CF4CEC040913704442389F184
:10CC80008091390490913A0420913F0430914004FE
:10CC9000821B930B0996439748F480913904909135
:10CCA0003A04A0913B04B0913C0412C0242F3327D6
:10CCB00027FD3095432F532F80913F0490914004DE
:10CCC000A0914104B0914204820F931FA41FB51F8D
:10CCD00080933F0490934004A0934104B093420496
:10CCE00024C020913F043091400440914104509170
:10CCF0004204809152081616170644F463E00E941D
:10CD0000A09F280F311D411D511D07C063E00E94E7
:10CD1000A09F281B31094109510920933F043093FA
:10CD20004004409341045093420410920D05109228
:10CD30000C05E0904304F0904404009145041091E8
:10CD40004604D801C70180509440A040B0402091D3
:10CD50003F043091400440914104509142048217B5
:10CD60009307A407B5075CF4D801C70180509C4F16
:10CD7000AF4FBF4F281739074A075B0744F080932E
:10CD80003F0490934004A0934104B09342048091E7
:10CD9000390A81FF06C084E690E090931E038093D9
:10CDA0001D03809156088823A9F5809138048823B3
:10CDB00089F540912D0450912E0457FF02C04D5F1C
:10CDC0005F4F5595479555954795809126019091D0
:10CDD0002701209102013327489FB001499F700D20
:10CDE000589F700D1124CB01B9010E94C09F709310
:10CDF000830160938201663471051CF486E490E03F
:10CE000005C06739710534F086E990E0909383019D
:10CE1000809382018091BB049091BC04892BD1F155
:10CE20008091290390912A03A0912B03B0912C03A8
:10CE300080933F0490934004A0934104B093420434
:10CE400029C08091430490914404A0914504B0917D
:10CE5000460480599140A040B04080933F04909395
:10CE60004004A0934104B093420480915608882363
:10CE700011F0992702C088E790E090938301809396
:10CE8000820189819A8190932E0480932D048EE2F1
:10CE900080934101E0902D04F0902E0480912903AD
:10CEA00090912A03A0912B03B0912C0320913F0471
:10CEB00030914004409141045091420428173907B1
:10CEC0004A075B0724F08091390A80FD98C480915D
:10CED00008046091BB047091BC04882309F07CC2F3
:10CEE000672B49F0E0902D04F0902E0410920F056E
:10CEF00010920E05E1C08091290390912A03A09120
:10CF00002B03B0912C03821B930BA40BB50B8093C6
:10CF1000D9049093DA04A093DB04B093DC0482304C
:10CF2000E0E89E07EFEFAE07EFEFBE072CF481E0DD
:10CF300090E8AFEFBFEF09C08F5F9F47A040B040C0
:10CF400064F08FEF9FE7A0E0B0E08093D904909366
:10CF5000DA04A093DB04B093DC048091D9049091AF
:10CF6000DA0490930F0580930E0580917B01282FA2
:10CF70003327442755278091D9049091DA04A09152
:10CF8000DB04B091DC04BC01CD010E94819F97FFBE
:10CF900004C0615E7F4F8F4F9F4F25E09595879529
:10CFA000779567952A95D1F76093D9047093DA0441
:10CFB0008093DB049093DC0465300EEF70070FEF75
:10CFC00080070FEF90072CF484E09EEFAFEFBFEFE8
:10CFD00009C0605074408040904064F080E094E06C
:10CFE000A0E0B0E08093D9049093DA04A093DB042E
:10CFF000B093DC046090D9047090DA04209133037C
:10D000003091340337FF02C0295F3F4F03E035956D
:10D0100027950A95E1F74FEF223834071CF421E8F1
:10D020003FEF05C02038310514F020E830E0C90199
:10D03000AA2797FDA095BA2F20917C01332744277A
:10D040005527BC01CD010E94819F97FF04C06D5FF1
:10D050007F4F8F4F9F4F12E09595879577956795F6
:10D060001A95D1F79B015FEF613075071CF420E042
:10D070003FEF06C06F3F710519F014F020E031E07A
:10D0800080911004807C49F0C90137FD03969C0112
:10D0900035952795359527950DC08091390A80FFE4
:10D0A00009C0C90137FD07969C01A3E03595279576
:10D0B000AA95E1F7620E731E20917A01222309F4EA
:10D0C00054C06091630470916404809165049091F0
:10D0D000660497FF04C061587F4F8F4F9F4FF7E062
:10D0E0009595879577956795FA95D1F733274427D6
:10D0F00055270E94819F97FF04C0615E7F4F8F4F2D
:10D100009F4FE5E09595879577956795EA95D1F7D7
:10D110006093D9047093DA048093DB049093DC0469
:10D120006138AFEF7A07AFEF8A07AFEF9A072CF4B9
:10D1300080E89FEFAFEFBFEF0AC06F3F7105810539
:10D14000910569F064F080E091E0A0E0B0E08093A8
:10D15000D9049093DA04A093DB04B093DC048091AB
:10D16000D9049091DA04680E791E80917801282FF5
:10D1700033278091EA0A992787FD9095289FF0012F
:10D18000299FF00D389FF00D11249F01F7FF02C079
:10D1900021583F4F220F232F221F330BFFEF21383F
:10D1A0003F071CF420E83FEF06C02F3F310519F080
:10D1B00014F020E031E0260D371DC901AA2797FDA4
:10D1C000A095BA2F00912D0410912E0498014427A8
:10D1D00037FD4095542FBC01CD010E94819F97FFE0
:10D1E00004C061507E4F8F4F9F4F59E095958795B2
:10D1F000779567955A95D1F7E61AF70A80913D041D
:10D2000090913E04892B09F064C0101611060CF0B1
:10D2100060C020910E0530910F05C90137FF03C092
:10D22000309521953F4F2D33310540F480915B04BB
:10D2300090915C048E159F0574F526C02C533040E8
:10D2400045E0369527954A95E1F72031310510F0F4
:10D250002FE030E040915B0450915C0418161906F1
:10D26000E4F480E190E0821B930B489F9001499F7A
:10D27000300D589F300D1124B4E036952795BA959E
:10D28000E1F72E153F0520F58091800190918101F5
:10D29000E816F906F4F07C011CC0205F3F4F809136
:10D2A000800190918101829FB001839F700D929FB8
:10D2B000700D11249B01A4E036952795AA95E1F7FE
:10D2C0004E155F0514F07A0104C0E216F30608F06B
:10D2D0007901C701AA2797FDA095BA2FFDE0880F15
:10D2E000991FAA1FBB1FFA95D1F72091260A3091EA
:10D2F000270A442737FD4095542FBC01CD010E94D9
:10D30000F59F2093DD043093DE044093DF045093B7
:10D31000E004E090DD04F090DE048091100590912F
:10D3200011059C01220F331F280F391F2E0D3F1DA1
:10D3300037FF02C02D5F3F4FA90155954795559581
:10D340004795509311054093100580914E08282F62
:10D350003327220F331F220F331F241735076CF496
:10D3600080915E0A282F3327220F331F220F331F8D
:10D37000205530404217530724F030931105209375
:10D3800010058091390A80FF14C08091100590919A
:10D390001105A981BA818A179B0724F0B093110562
:10D3A000A0931005E0911005F0911105FA83E9832F
:10D3B00026C229813A81201B310B37FF02C02D5F25
:10D3C0003F4F3595279535952795E0901005F090BE
:10D3D0001105E20EF31EC1C1672B49F0E0902D0448
:10D3E000F0902E0410920F0510920E0538C1809116
:10D3F000290390912A03A0912B03B0912C03821B47
:10D40000930BA40BB50B8093D9049093DA04A093EB
:10D41000DB04B093DC04823000E890070FEFA00734
:10D420000FEFB0072CF481E090E8AFEFBFEF09C039
:10D430008F5F9F47A040B04064F08FEF9FE7A0E070
:10D44000B0E08093D9049093DA04A093DB04B09306
:10D45000DC048091D9049091DA0490930F058093B5
:10D460000E0580917B01282F332744275527809173
:10D47000D9049091DA04A091DB04B091DC04BC01E2
:10D48000CD010E94819F97FF04C0615E7F4F8F4F47
:10D490009F4F05E095958795779567950A95D1F704
:10D4A0006093D9047093DA048093DB049093DC04D6
:10D4B000653028EF72072FEF82072FEF92072CF4C9
:10D4C00084E098EFAFEFBFEF09C060507840804034
:10D4D000904064F080E098E0A0E0B0E08093D90450
:10D4E0009093DA04A093DB04B093DC046090D90439
:10D4F0007090DA0480917A01282F332780913A03C3
:10D5000090913B03829FA001839F500D929F500DED
:10D5100011249A0157FF02C021503F4F232F330F90
:10D52000330B8091330390913403820F931FAA270A
:10D5300097FDA095BA2F8093D9049093DA04A09315
:10D54000DB04B093DC048091370420913D043091DA
:10D550003E04882331F0B3E0220F331FBA95E1F780
:10D560001BC0809152089927289FB001299F700DF8
:10D57000389F700D11249B01A3E0220F331FAA9541
:10D58000E1F7260F371F37FF02C0215E3F4FF5E05E
:10D5900035952795FA95E1F730930A04209309040D
:10D5A0008091090490910A049C01442737FD40951D
:10D5B000542F8091D9049091DA04A091DB04B091AA
:10D5C000DC04821B930BA40BB50B8093D9049093BE
:10D5D000DA04A093DB04B093DC0420917C013327B0
:10D5E00044275527BC01CD010E94819F97FF04C0AD
:10D5F000615E7F4F8F4F9F4FE5E0959587957795BB
:10D600006795EA95D1F76093D9047093DA04809313
:10D61000DB049093DC046530A8EF7A07AFEF8A074C
:10D62000AFEF9A072CF484E098EFAFEFBFEF09C09B
:10D63000605078408040904064F080E098E0A0E046
:10D64000B0E08093D9049093DA04A093DB04B09304
:10D65000DC048091D9049091DA04680E791EE618F2
:10D66000F70880915B0490915C048E159F053CF453
:10D670008091800190918101E816F9060CF07C01FF
:10D68000C701AA2797FDA095BA2F5DE0880F991FC3
:10D69000AA1FBB1F5A95D1F72091260A3091270A5D
:10D6A000442737FD4095542FBC01CD010E94F59FC2
:10D6B0002093DD043093DE044093DF045093E004B4
:10D6C000E090DD04F090DE0480911005909111054A
:10D6D0009C01220F331F280F391F2E0D3F1D37FFCE
:10D6E00002C02D5F3F4FA901559547955595479528
:10D6F000509311054093100580914E08282F332731
:10D70000220F331F220F331F241735076CF480912B
:10D710005E0A282F3327220F331F220F331F205575
:10D7200030404217530724F0309311052093100521
:10D730008091390A209110053091110580FF10C0A9
:10D74000E981FA812E173F0724F0F0931105E09349
:10D750001005E0901005F0901105FA82E9824FC0A3
:10D760003A8329834CC080915608882301F5609143
:10D770002D0470912E0477FF02C06D5F7F4F759569
:10D780006795759567954091260150912701809185
:10D790000201282F3327649FC001659F900D749F5D
:10D7A000900D1124B9010E94C09FCB0101C099279F
:10D7B00090938301809382018091820190918301F3
:10D7C000873491051CF486E490E005C08639910504
:10D7D00034F086E990E0909383018093820109817F
:10D7E0001A81109311050093100580911004806C2C
:10D7F0008093100480910F048D7F80930F0480919B
:10D80000100499279C012270307081FF39C18091EA
:10D81000120590911305A0911405B091150500977C
:10D82000A105B10521F0809147048130B9F48091C0
:10D830002D0490912E04AA2797FDA095BA2F1EE0E3
:10D84000880F991FAA1FBB1F1A95D1F78093120545
:10D8500090931305A0931405B09315058091470488
:10D86000813019F482E08093470429813A8179015B
:10D870000027F7FC0095102F8091260A9091270A27
:10D880009C01442737FD4095542FC801B7010E94E1
:10D89000819FDC01CB018093DD049093DE04A09393
:10D8A000DF04B093E004B7FF04C08150904EAF4F47
:10D8B000BF4F7C018D01ADE015950795F794E79476
:10D8C000AA95D1F7E092DD04F092DE040093DF0424
:10D8D0001093E00460911104709112043FE0603AEB
:10D8E000730750F58091120590911305A0911405CE
:10D8F000B09115059C01AD01FAE056954795379515
:10D900002795FA95D1F7821B930BA40BB50BA801B1
:10D910009701E4E0220F331F441F551FEA95D1F70A
:10D92000820F931FA41FB51F8093120590931305B8
:10D93000A0931405B093150560547F4118F58091AC
:10D94000120590911305A0911405B09115059C0145
:10D95000AD016CE056954795379527956A95D1F7B7
:10D96000821B930BA40BB50BA8019701F2E0220FC9
:10D97000331F441F551FFA95D1F7820F931FA41F21
:10D98000B51F41C0809133039091340380913303DC
:10D990009091340397FF03C0909581959F4F8436F3
:10D9A0009105CCF58091290390912A03A0912B0336
:10D9B000B0912C039C0180913F0490914004281B5E
:10D9C000390B37FF03C0309521953F4F2F3F31056D
:10D9D00009F00CF58091120590911305A0911405A2
:10D9E000B09115059C01AD01EEE056954795379530
:10D9F0002795EA95D1F7821B930BA40BB50B8E0DDF
:10DA00009F1DA01FB11F8093120590931305A09333
:10DA10001405B09315058091120590911305A091FE
:10DA20001405B09115057EE0B695A7959795879555
:10DA30007A95D1F790932E0480932D044091540849
:10DA4000442399F055279C01BA010E94C09FC90147
:10DA5000861B970B90935C0480935B04260F371F03
:10DA600030938101209380011FC010925C041092BA
:10DA70005B048FEF93E0909381018093800114C049
:10DA8000109247041092120510921305109214057B
:10DA90001092150530932E0420932D0405C080911B
:10DAA0001004806C809310048091260581FF37C09C
:10DAB00089819A8197FD0396959587959595879588
:10DAC00020910D0430910E042817390760F48091DD
:10DAD0002D0490912E04892B31F0220F331F220F39
:10DAE000331F3A8329838091290390912A03A091BF
:10DAF0002B03B0912C0380933F0490934004A09398
:10DB00004104B093420488E99AE390931E03809302
:10DB10001D0380E09EE090930C0180930B01209107
:10DB2000210A822F9927880F991F880F991F88969D
:10DB300069817A818617970714F09A838983709197
:10DB40005E0A7D8B872F9927880F991F880F991F51
:10DB500080559040A981BA818A179B0714F49A8353
:10DB6000898380916B03882341F48091F10A8F3F70
:10DB700021F480912A05882321F18091110490914C
:10DB800012040297C097E8F4E981FA811E161F0675
:10DB9000C4F481E090E09093120480931104E22E8B
:10DBA000FF24EE0CFF1CEE0CFF1C8701085D1F4FCD
:10DBB0001A8309838091F10A883218F489E08093EE
:10DBC000AC0129813A813093AA072093A90780915B
:10DBD000D5049091D604A091D704B091D80412E056
:10DBE000880F991FAA1FBB1F1A95D1F700915F0AD2
:10DBF0001091600A081B190B213A31058CF0C901FC
:10DC000037FD019695958795801791070CF48C0147
:10DC1000909581959F4F081719076CF48C010BC0E4
:10DC20000135110514F000E510E03FEF003B13074C
:10DC300014F400EB1FEF4D89242F3327220F331FDD
:10DC4000220F331FC90169817A81861B970B8017C8
:10DC500091070CF48C0189819A81821B930B081720
:10DC600019070CF48C0180911C0A90911D0A609197
:10DC7000590470915A04861B970B90932C0A809339
:10DC80002B0AD0903B0A20916B0430916C04409198
:10DC90006D0450916E04DD2041F0461A570AC2010E
:10DCA000AA2797FDA095BA2F04C0AA2797FDA09593
:10DCB000BA2F280F391F4A1F5B1F20936B04309324
:10DCC0006C0440936D0450936E0480916B049091AA
:10DCD0006C04A0916D04B0916E0481509A4FA040E5
:10DCE000B04064F080E09AEFA0E0B0E080936B0475
:10DCF00090936C04A0936D04B0936E0480916B04B8
:10DD000090916C04A0916D04B0916E048050964087
:10DD1000AF4FBF4F64F480E096E0AFEFBFEF80936A
:10DD20006B0490936C04A0936D04B0936E04C09048
:10DD3000630820912B0A30912C0A78E0E72EEC142E
:10DD400098F08C2D9927829FA001839F500D929F60
:10DD5000500D1124CA0157FD07967C0163E0F5942C
:10DD6000E7946A95E1F712C08C2D86959927829FDA
:10DD7000B001839F700D929F700D1124CB0177FD30
:10DD800003967C01F594E794F594E794A0907D01C7
:10DD9000B0907E019501442737FD4095542F809126
:10DDA0006B0490916C04A0916D04B0916E04BC0161
:10DDB000CD010E94F59FE20EF31E90906701692D40
:10DDC000772788279927980117FF04C02227332730
:10DDD000201B310B37FF02C02F5F3F4F3595279532
:10DDE000A981BA812A0F3B1F442737FD4095542F44
:10DDF0000E94819F97FF04C0615C7F4F8F4F9F4FB0
:10DE000026E095958795779567952A95D1F79B019B
:10DE10006E157F050CF47B01309521953F4FE2167E
:10DE2000F3060CF4790180910D0A90910E0A60912D
:10DE3000570470915804861B970B90930C0A80939B
:10DE40000B0A209167043091680440916904509155
:10DE50006A04DD2041F0261A370AC101AA2797FD7E
:10DE6000A095BA2F04C0AA2797FDA095BA2F280F16
:10DE7000391F4A1F5B1F2093670430936804409347
:10DE8000690450936A048091670490916804A0919A
:10DE90006904B0916A0481509A4FA040B04064F088
:10DEA00080E09AEFA0E0B0E080936704909368046C
:10DEB000A0936904B0936A04809167049091680408
:10DEC000A0916904B0916A0480509640AF4FBF4F53
:10DED00064F480E096E0AFEFBFEF80936704909327
:10DEE0006804A0936904B0936A0420910B0A3091EE
:10DEF0000C0A48E04C1598F08C2D9927829FB001B0
:10DF0000839F700D929F700D1124CB0177FD0796B2
:10DF10006C0193E0D594C7949A95E1F712C0C6942A
:10DF20008C2D9927829FD001839FB00D929FB00DB9
:10DF30001124CD01B7FD03966C01D594C794D594F7
:10DF4000C7949501442737FD4095542F809167046D
:10DF500090916804A0916904B0916A04BC01CD015C
:10DF60000E94F59FC20ED31E692D77278827992717
:10DF7000980117FF04C022273327201B310B37FFDE
:10DF800002C02F5F3F4F35952795E981FA812E0F0B
:10DF90003F1F442737FD4095542F0E94819F97FFD4
:10DFA00004C0615C7F4F8F4F9F4FA6E0959587958A
:10DFB00077956795AA95D1F79B016C157D050CF4B3
:10DFC0006B01309521953F4FC216D3060CF46901C1
:10DFD0008091210A282E33245090A508F7E1AF2E16
:10DFE000F9E0BF2EEEEC8E2EE8E09E2E7BE0472E71
:10DFF0006CE3662E6AE0762ED4012C9112160CF09A
:10E0000030C1203429F4E981FA81FF8BEE8B1FC0E7
:10E0100049815A81CA01AA2797FDA095BA2F3327B3
:10E0200027FD3095432F532FBC01CD010E94819FC6
:10E0300097FF04C0615C7F4F8F4F9F4F56E09595CF
:10E040008795779567955A95D1F77F8B6E8BF401FD
:10E050002181203439F42E893F892E0D3F1D3F8BBD
:10E060002E8B2AC0203C39F44E895F894E195F09F6
:10E070005F8B4E8B21C0C701AA2797FDA095BA2FB1
:10E08000332727FD3095432F532FBC01CD010E942C
:10E09000819F97FF04C0615C7F4F8F4F9F4F46E089
:10E0A00095958795779567954A95D1F7AE89BF89FC
:10E0B000A60FB71FBF8BAE8BF4012281203439F439
:10E0C0002E893F892C0D3D1D3F8B2E8B2AC0203C75
:10E0D00039F44E895F894C195D095F8B4E8B21C0E5
:10E0E000C601AA2797FDA095BA2F332727FD3095A3
:10E0F000432F532FBC01CD010E94819F97FF04C085
:10E10000615C7F4F8F4F9F4F36E095958795779550
:10E1100067953A95D1F7AE89BF89A60FB71FBF8B18
:10E12000AE8BF4012381203439F42E893F89200FEE
:10E13000311F3F8B2E8B2AC0203C39F44E895F89DA
:10E14000401B510B5F8B4E8B21C0C801AA2797FD46
:10E15000A095BA2F332727FD3095432F532FBC01AD
:10E16000CD010E94819F97FF04C0615C7F4F8F4F5C
:10E170009F4F26E095958795779567952A95D1F7D6
:10E18000AE89BF89A60FB71FBF8BAE8BF50180810B
:10E1900081FD08C0D3018D919C91EE89FF898E1776
:10E1A0009F0774F4D3018D919C91EE89FF898E0FA6
:10E1B0009F1F97FD0196959587959F8B8E8B1EC00F
:10E1C000552049F42E893F89220F331F281B390B14
:10E1D0003F8B2E8B13C031E0351580F4252D33276E
:10E1E0004E895F89841B950BB9010E94C09FCB01AA
:10E1F0006E897F89680F791F7F8B6E8BC101880FB5
:10E20000991F880F991FAE89BF898A179B0764F4ED
:10E21000BD898B2F9927880F991F880F991FEE8929
:10E22000FF89E817F90714F09F8B8E8B8E899F89E1
:10E2300097FD03969595879595958795F50181832B
:10E24000880F991F880F991F2E893F89281B390B2A
:10E25000C901880F8283EE89FF89D301ED93FC9376
:10E2600003C0F501118212824A9422E030E0620E6E
:10E27000731E44E050E0840E951E68E070E0A60E28
:10E28000B71E47FEB9CEE2E1C95E0C942CA084B162
:10E29000806A84B93D9A82E58CBD1DBC459A81E0B7
:10E2A0008093700A8AEA8093810A83E88093820AC5
:10E2B0008AE08093830A1092850A1092840A109251
:10E2C000870A1092860A1092E90A1092A50A089508
:10E2D0003091700A332309F070C00DB407FE6DC091
:10E2E00083E080931C03459A2EB580912D059927D4
:10E2F0008130910589F0823091051CF4892B21F041
:10E300003EC00297B9F03BC03093A40A20932E057B
:10E310002138A9F581E008C0253549F480912E0502
:10E32000820F80932E0582E080932D0528C03093C4
:10E330002D0525C08091A40AE82FFF27EA53F54F49
:10E3400020838F5F8093A40A90912E058032A0F0E5
:10E35000291769F480E2A6ECBAE0E6EAFAE00D904B
:10E3600001928A95E1F781E08093A50A02C030937B
:10E37000A50A10922D0503C0920F90932E052091AF
:10E38000800A2232A0F4459800000000000000003E
:10E39000E091790AF0917A0AE20FF11D80818EBD39
:10E3A0008091A20A9081890F8093A20A03C081E024
:10E3B0008093700A2F5F2093800A0895EF92FF9256
:10E3C0000F931F9380915C089927880F991F880FDE
:10E3D000991F7C010027F7FC0095102F8091A30462
:10E3E0009091A404A091A504B091A604BC01CD0114
:10E3F000A80197010E94F59F3093850A2093840A13
:10E4000080919B0490919C04A0919D04B0919E04E6
:10E41000BC01CD01A80197010E94F59F3093870AA6
:10E420002093860A2091660A3091670A4091680A13
:10E430005091690ADA01C90173E0880F991FAA1F78
:10E44000BB1F7A95D1F7820F931FA41FB51F820FB0
:10E45000931FA41FB51F20914201309143014091A9
:10E46000440150914501BC01CD010E94F59F3093BC
:10E470008D0A20938C0A8091B5049091B604209166
:10E48000400330914103821B930B9093930A809336
:10E49000920AE091AB04F091AC048091320A909121
:10E4A000330ABF010E94C09FCB019B01220F331F83
:10E4B000220F331F280F391F280F391F37FF02C0C3
:10E4C0002D5F3F4F35952795359527953093890AD0
:10E4D0002093880A8091620A9091630ABF010E948A
:10E4E000C09F9B01220F331F220F331F260F371FA0
:10E4F000260F371F37FF02C02D5F3F4F35952795F9
:10E500003595279530938B0A20938A0A1092AC0494
:10E510001092AB041092330A1092320A1092630ADE
:10E520001092620A8091830A9927AA27BB27FC01CF
:10E530003A97E830F10508F030C2EF57FF4F0C94DE
:10E5400047A0809125048093960A809124048093AB
:10E55000970A809123048093980A809122048093E3
:10E56000990A8091210480939A0A809120048093D3
:10E570009B0A80911F0480939C0A80911E048093C3
:10E580009D0A8091100480939E0A80911004837FDD
:10E59000809310048091010180939F0A809126014D
:10E5A000909127018093A00A80910F048093A10A83
:10E5B0004299F3C180910F04877F80930F04EDC1CE
:10E5C0008091EB0A9091EC0A9093970A8093960AB7
:10E5D0008091EF0A9091F00A9093990A8093980A9B
:10E5E000809191080E94734880939A0A809141011A
:10E5F00080939B0A90912F0590939C0AE92FFF2707
:10E6000013E0EE0FFF1F1A95E1F7E95EF64F8081E8
:10E6100080939D0A868180939E0A838180939F0ABE
:10E6200087818093A00A85818093A10A9F5F909340
:10E630002F05E92FFF27EE0FFF1FEE0FFF1FEF53F0
:10E64000F74F8585882309F0A8C1992309F4A5C14E
:10E65000892F992701966CE070E00E94C09F9C0171
:10E66000982FE82FFF27EE0FFF1FEE0FFF1FEF532E
:10E67000F74F8585882311F4222351F720932F0526
:10E680008CC1809102018093960A809192088093B8
:10E69000970A809193088093980A809194088093B8
:10E6A000990A8091950880939A0A8091990880939D
:10E6B0009B0A80919A0880939C0A80919B08809382
:10E6C0009D0A80919E0880939E0A80919C08809369
:10E6D0009F0A80919D088093A00A80919F085BC14A
:10E6E000809190088093960A80916708863081F027
:10E6F0008091E802823451F00E94DE7EE82FFF27ED
:10E70000ED51FE4E84918093E80202C00E94DE7EAD
:10E71000809153058093970A8091AD088093980A61
:10E720008091A6088093990A38C1F8948091430893
:10E73000E82FFF27EE0FFF1FE858F64F0190F081FA
:10E74000E02DE038F1051CF0EFE7F0E006C02FEF18
:10E75000E138F20714F4E1E8FFEFE093960A8091C4
:10E760004408E82FFF27EE0FFF1FE858F64F0190EF
:10E77000F081E02DE038F1051CF0EFE7F0E006C095
:10E780007FEFE138F70714F4E1E8FFEFE093970A31
:10E7900080914208E82FFF27EE0FFF1FE858F64F41
:10E7A0000190F081E02DE038F1051CF0EFE7F0E09A
:10E7B00006C08FEFE138F80714F4E1E8FFEFE093CB
:10E7C000980A80914108E82FFF27EE0FFF1FE858B5
:10E7D000F64F0190F081E02DE038F1051CF0EFE7F5
:10E7E000F0E006C02FEFE138F20714F4E1E8FFEFA4
:10E7F0007894E093990A80914A0480939A0A8091D0
:10E800004B0480939B0A80914C0480939C0A8091D6
:10E810004D0480939D0A80914E0480939E0A8091BE
:10E820004F0480939F0A809150048093A00A8091A6
:10E830005104B1C08091D005863018F01092D005F7
:10E8400085E08093960A8091A0088093970A809132
:10E85000430490914404A0914504B0914604BC0146
:10E86000CD0125E030E040E050E00E94F59F30937C
:10E87000990A2093980A80913F0490914004A091B6
:10E880004104B0914204BC01CD0125E030E040E0FC
:10E8900050E00E94F59F30939B0A20939A0A809142
:10E8A000960880939C0A8091970880939D0A809196
:10E8B000980880939E0A8091490480939F0A8091D2
:10E8C00030058093A00A8091A9079091AA0797FD2F
:10E8D000039695958795959587955DC082E0809381
:10E8E000960A8093970A1092980A89E38093990A6E
:10E8F0008091030180939A0A8091B50580939B0AC9
:10E900009091B60590939C0A8F778093B50590718E
:10E910009093B6058091AE0880939D0A8091560A27
:10E9200080939E0A8091390A80939F0A8091A20861
:10E930008093A00A8091B3082EC0809175088093BF
:10E94000960A8091B1088093970A80916F01809315
:10E95000980A80916E088093990A80916F0880933D
:10E960009A0A8091700880939B0A80916E0180932F
:10E970009C0A8091720880939D0A8091730880930D
:10E980009E0A8091740880939F0A8091F10A809377
:10E99000A00A8091D3078093A10A8091A50A8823B9
:10E9A00009F479C16091A60A8091A601681719F04F
:10E9B0008AEF8093A4016093A60181E080938F0188
:10E9C0004091A70A5091A80ACA0181509E4F8F5FBB
:10E9D0009340B0F42091A90A3091AA0AC90181504C
:10E9E0009E4F8F5F934060F480914D0885FF08C073
:10E9F00050931C0540931B0530931A05209319056D
:10EA00008091AD0A9091AE0A21E08936920724F4F4
:10EA100090939101809390012091B70A3091B80AA8
:10EA200080911D0390911E038217930740F48091FB
:10EA3000F002882321F430931E0320931D03862FB8
:10EA400099278936910509F4A5C08A36910544F4C1
:10EA50008736910571F08836910509F462C023C1AB
:10EA60008A36910509F414C18B36910509F4E2C088
:10EA70001AC18091B90A8093E60A8091BA0A8093FC
:10EA8000E80A8091BB0A8093E70A8091BC0A8093D0
:10EA90008E018091BD0A8093EA0A8091BE0A80931C
:10EAA000A5018091BF0A80932C058091C00A8093B4
:10EAB000180580911D048823F9F02091C10A309136
:10EAC000C20A37FD19C0309362042093610490910B
:10EAD0007708992389F08FE0989FC0011124281BA3
:10EAE000390BC90188599E4F68E671E00E94C09FAA
:10EAF0009093620480936104209123053091240552
:10EB00008091C30A9091C40A280F391F37FF02C0B1
:10EB10002F5F3F4F3595279530932405209323058C
:10EB2000C2C08091B90A80937B0A8091BA0A80930F
:10EB30007C0A8091BB0A80937D0A8091BC0A8093F5
:10EB40007E0A8091BD0A80937F0A809199079091F7
:10EB5000BE0A892B8093990790919A0793708091B0
:10EB6000BF0A8C70982B90939A078091C00A80936B
:10EB70002A058091C10A809396018091C20A8093F0
:10EB8000E90A8091C30A809326058091C40A809384
:10EB9000250589C08091B90A8093710A8091BA0ACB
:10EBA0008093720A8091BB0A8093730A8091BC0A99
:10EBB0008093740A8091BD0A9091BE0A9093760A60
:10EBC0008093750A8091BF0A9091C00A9093780A49
:10EBD0008093770A8091C10A992787FD9095909339
:10EBE000B3098093B2098091C20A8093380480915E
:10EBF000C30A9091C40A9C01442737FD4095542FC5
:10EC0000DA01C90163E0880F991FAA1FBB1F6A952B
:10EC1000D1F7820F931FA41FB51F820F931FA41F4C
:10EC2000B51F8093390490933A04A0933B04B093AA
:10EC30003C0439C08091B90A809329058091BA0AB1
:10EC4000809328058091BB0A809327059091BC0A88
:10EC5000992349F08091AC01882319F081518330C8
:10EC600010F49093AC018091BD0A80935B05809174
:10EC7000BE0A80935A058091BF0A9091C00A909372
:10EC80005805809357058091C10A809359050BC0A0
:10EC90000E94457F08C010921C0510921B0510921F
:10ECA0001A05109219051F910F91FF90EF9008958A
:10ECB0008091700A882319F480E090E008954598C7
:10ECC00081E89AE090937A0A8093790A90912B05D3
:10ECD000E92FFF27E956FE4F9F5F90932B05808118
:10ECE0008093830A9D3010F010922B051092700AC9
:10ECF0000E94DE7181E08093800A8091810A809376
:10ED0000A20A8EBD81E090E0089587B18C6087B93A
:10ED1000429843981092320580E88093A80110929F
:10ED200031058093A70108958091B2099091B309AC
:10ED300081589F4F39F08091B2099091B309815861
:10ED400080933C05809137058150809337058F3F34
:10ED500009F052C180918A088093380580918C080F
:10ED60008093390589E080933705809110049927B5
:10ED700080739070892B21F48091B60580FF1DC0AF
:10ED800080918E08882351F080913A05882319F4E8
:10ED900084E08093320581E080933A0580918F086A
:10EDA000882379F080913B05882319F484E08093CF
:10EDB000310581E080933B0504C010923A05109222
:10EDC0003B0580913A05882309F082C08091B00804
:10EDD000282F332724FF07C080914804882319F483
:10EDE00025FD8FC090C090918B08983F48F080918E
:10EDF000340A8D3D28F08091380588236CF00AC0D4
:10EE0000983F78F08091340A853059F48091380524
:10EE100087FF02C0429A01C0429881E08093A80116
:10EE200054C0809132058150809332058F3F09F0A4
:10EE30006BC08091B30885FF2FC090913C05892F4E
:10EE4000869580933205992361F4909330058091E3
:10EE5000380587FF02C0429A01C042981092A8016B
:10EE600053C081E0809330058091A80190913805CE
:10EE7000882349F480933C0580E48093A80199237A
:10EE80000CF43FC040C0982311F0429A01C0429850
:10EE900086958093A80138C08091340A8695809326
:10EEA00032058091A801813021F410923C0580E464
:10EEB00001C086958093A8018091A80190913805A2
:10EEC000892311F0429A01C04298109230051CC06B
:10EED000809132058150809332058F3FA9F489E0FB
:10EEE000809332058091A801813011F480E801C03F
:10EEF00086958093A8018091A80190918E0889231E
:10EF000011F0429A01C0429880913B05882309F094
:10EF100043C09091B00897FF07C0809148048823B0
:10EF200019F496FD52C053C090918D08983F48F057
:10EF300080915D0A8D3D28F08091390588236CF021
:10EF40000AC0983F78F080915D0A853059F480912D
:10EF5000390587FF02C0439A01C0439881E080933E
:10EF6000A70136C0809131058150809331058F3FD4
:10EF700079F580915D0A8695809331058091A7018E
:10EF8000813011F480E401C086958093A7018091BF
:10EF9000A7019091390517C0809131058150809368
:10EFA00031058F3FA9F489E0809331058091A70155
:10EFB000813011F480E801C086958093A70180918B
:10EFC000A70190918F08892311F0439A01C04398BB
:10EFD000429B05C080910F04886080930F04439B7F
:10EFE00006C080910F04806180930F040895809182
:10EFF0000F048F7E80930F0408954FB724E130E013
:10F00000F8948091C9008F778093C9008091C900DE
:10F010008F7B8093C9008091C9008F7D8093C90048
:10F02000832F99278093CD002093CC008091C80036
:10F0300082608093C80080E18093C9008091CA00FB
:10F040008F778093CA008091CA008F7B8093CA001B
:10F050008091CA008F7D8093CA008091CA008F7E04
:10F060008093CA008091CA00877F8093CA008091F4
:10F07000C9008B7F8093C9008091CA00846080930F
:10F08000CA008091CA0082608093CA008091C80043
:10F0900087FF03C08091CE00F9CF8091C9008068BE
:10F0A0008093C9004FBF0895EF92FF920F931F9373
:10F0B000CF93DF93482F00E010E08091A9018130C9
:10F0C00061F41092A90184E480933D0510923F05FC
:10F0D00010923E051092400539C180913D0588236C
:10F0E00019F421E030E001C0980190913E05992388
:10F0F00071F4232B11F081E010C084E480933D056E
:10F1000090933F0590933E059093400508C1913040
:10F1100069F4232B09F0F9C082E080933E058091C9
:10F120003F058F5F80933F0583E0F7C09230D1F4B5
:10F13000232B09F0EAC083E080933D05409340050E
:10F1400090913F05923039F41092410547FF03C07A
:10F1500081E08093410583E080933E059F5F90931B
:10F160003F05DDC0933009F0D0C0232B09F0CDC09E
:10F1700090933D0582E080933E0580913F058F5F2F
:10F1800080933F0520914005822F9927782F66278D
:10F19000842F9927682B792B80916708813049F457
:10F1A0007370CB018050924063E070E00E94C09F7A
:10F1B00017C0823061F47770CB018050944066E0D4
:10F1C00070E00E94C09F2695269526950BC073700F
:10F1D00068567140CB0177FD0196BC017595679526
:10F1E00026952695022F11270F7010700F5F1F4F65
:10F1F0000D30110508F082C07801E00EF11EF70114
:10F20000E858F64F808191819B01281B390BC90179
:10F2100037FF03C0909581959F4F069704F5E091C5
:10F22000A908EE2351F0FF27EE0FFF1FE858F64F15
:10F23000808191818436910594F480914904883CC1
:10F2400030F480914904865F8093490408C088ECBB
:10F250008093490480916F008F7D80936F00F70148
:10F26000E858F64F808191819C01220F331F280FAF
:10F27000391F260F371F37FF02C02D5F3F4FE901AF
:10F28000D595C795D595C795CB0101968C179D0748
:10F2900014F4219706C061507040C617D7070CF4CC
:10F2A000219680914904843BD0F0F701E858F64F4D
:10F2B00080819181FE01E81BF90BCF0163E070E0D2
:10F2C0000E94C09FCB01880F991F860F971F2EEBBE
:10F2D00039E0E20EF31EF7019183808307C02EEB25
:10F2E00039E0E20EF31EF70111821082000F111FA8
:10F2F0000858164FF801D183C08311C0023111059F
:10F3000070F081E08093A9010AC081E08093A90197
:10F3100010923F051092410584E480933D05809151
:10F320003F05803198F080914105882331F4809128
:10F33000A901882311F48093400110923F05109297
:10F34000410510923E0584E480933D05E6E0CDB78B
:10F35000DEB70C9438A0CF93FC0197FF05C0CFEF28
:10F36000F095E195FF4F01C0C1E028E631E0CF0103
:10F37000B9010E94C09FFC018B35910554F08B555B
:10F3800090408A35910538F484EB90E08E1B9F0BFA
:10F39000FC0141E00DC0CF01855B90408A359105AD
:10F3A00018F4E45BF04003C02E1B3F0BF9014FEF54
:10F3B000EE0FFF1FED5CF64F259134918C2F9927AE
:10F3C00087FD9095289FB001299F700D389F700D83
:10F3D0001124842F992787FD9095689FA001699F2C
:10F3E000500D789F500D1124CA01CF9108952AE540
:10F3F00030E0281B390BC9010E94AB790895CF93E7
:10F40000DF9380E00E94B2918091260190912701C4
:10F410006AE070E00E94C09F9F938F9380912601C5
:10F42000909127016AE070E00E94C09F7F936F93E4
:10F4300087E09AE09F938F93C5EAD1E9DF93CF935A
:10F44000E0919C05F0919D0509952DB73EB7285F89
:10F450003F4F2DBF8091A401882361F186E00E9477
:10F46000B2918091960199279F938F938091750A0D
:10F470009091760A6AE070E00E94AC9F7F936F9350
:10F480008FED90E09F938F938091120A9091130AD1
:10F490009F938F9380E19AE09F938F93DF93CF9315
:10F4A000E0919C05F0919D0509958DB79EB70C964E
:10F4B0008DBF12C086E00E94B2918EE19AE09F93C8
:10F4C0008F93DF93CF93E0919C05F0919D05099573
:10F4D0000F900F900F900F9080912A05882309F4C8
:10F4E00052C080914205909143050E94721A882370
:10F4F00091F08091AA01882319F01092AA0103C00B
:10F5000081E08093AA018CED95E00E94691A9093A6
:10F510004305809342058091AA018823E1F080E0B1
:10F520000E94B2911F921F9290912A0581E1989FAB
:10F53000C0011124825B944F9F938F93DF93CF93ED
:10F54000E0919C05F0919D0509952DB73EB72A5F86
:10F550003F4F2DBF3BC086E00E94B29180912A05AB
:10F5600099279F938F9385E29AE09F938F93DF93E0
:10F57000CF93E0919C05F0919D0509958DB79EB7BD
:10F5800006968DBF23C0809152058823F9F00E9412
:10F59000B89180E10E94B29184EB98E09F938F93A1
:10F5A0008091010199279F938F9381E39AE09F9324
:10F5B0008F93DF93CF93E0919C05F0919D05099582
:10F5C0002DB73EB7285F3F4F2DBF5CC080E10E9442
:10F5D000B2918091EA029091EB026CE370E00E949C
:10F5E000AC9F9F938F938091EA029091EB026CE322
:10F5F00070E00E94AC9F7F936F938091EF0A90918F
:10F60000F00A9F938F938CE39AE09F938F93C5EAC0
:10F61000D1E9DF93CF93E0919C05F0919D05099589
:10F620008091560A2DB73EB7265F3F4F2DBF80FF12
:10F6300029C08AE10E94B2918091410199279F934C
:10F640008F938091430490914404A0914504B0911C
:10F650004604BC01CD0124E630E040E050E00E94C9
:10F66000F59F3F932F9389E49AE09F938F93DF93C5
:10F67000CF93E0919C05F0919D0509958DB79EB7BC
:10F6800008968DBFDF91CF910895CF93DF9380E0EF
:10F690000E94B29180913609992787FD90959F939A
:10F6A0008F9380912E09992787FD90959F938F9333
:10F6B00080912609992787FD90959F938F9380913C
:10F6C0001E09992787FD90959F938F9380E59AE077
:10F6D0009F938F93C5EAD1E9DF93CF93E0919C0587
:10F6E000F0919D05099580E10E94B2912DB73EB73A
:10F6F000245F3F4F2DBF80915609992787FD909534
:10F700009F938F9380914E09992787FD90959F93A2
:10F710008F9380914609992787FD90959F938F93AA
:10F7200080913E09992787FD90959F938F9380E65E
:10F730009AE09F938F93DF93CF93E0919C05F09194
:10F740009D05099580913F082DB73EB7245F3F4F37
:10F750002DBF853098F480E10E94B29180E79AE055
:10F760009F938F93DF93CF93E0919C05F0919D053C
:10F7700009950F900F900F900F9018C08730B0F43C
:10F7800088E10E94B2918FED90E09F938F9381E882
:10F790009AE09F938F93DF93CF93E0919C05F09134
:10F7A0009D0509958DB79EB706968DBFDF91CF91C8
:10F7B00008950F931F9380E00E94B2912AE030E0F9
:10F7C0008091EB0A9091EC0AB9010E94AC9F9F9343
:10F7D0008F938091EB0A9091EC0AB9010E94AC9F43
:10F7E0007F936F938091260190912701B9010E9428
:10F7F000C09F9F938F938091260190912701B9011B
:10F800000E94C09F7F936F938AE89AE09F938F93A3
:10F8100005EA11E91F930F93E0919C05F0919D0576
:10F82000099580E10E94B2918DB79EB70C968DBF6D
:10F830008091EF0A9091F00A9F938F938091ED0A47
:10F840009091EE0A9F938F938CE99AE09F938F9308
:10F850001F930F93E0919C05F0919D0509958DB73D
:10F860009EB708968DBF1F910F910895EF92FF925A
:10F870000F931F9380E00E94B2918FEDE82EF12C40
:10F88000FF92EF9280919001909191019F938F93BD
:10F890008091290599279F938F9388EA9AE09F93F7
:10F8A0008F9305EA11E91F930F93E0919C05F09166
:10F8B0009D05099580E10E94B2918DB79EB70A9689
:10F8C0008DBF8091270599279F938F93FF92EF9289
:10F8D0008091280599279F938F938BEB9AE09F93B4
:10F8E0008F931F930F93E0919C05F0919D050995CF
:10F8F0008DB79EB70A968DBF1F910F91FF90EF9025
:10F9000008950F931F93CF93DF938091A401C5EACD
:10F91000D1E9882309F47DC080E00E94B2918091F2
:10F92000720A99279F938F938091740A99279F93C6
:10F930008F938EEC9AE09F938F938E01DF93CF93FA
:10F94000E0919C05F0919D0509958DB79EB70896AD
:10F950008DBF8091730A833031F48CE00E94B291A4
:10F960008DED9AE005C08CE00E94B29182EE9AE0A3
:10F970009F938F93DF93CF93E0919C05F0919D052A
:10F9800009950F900F900F900F908091710A81FF51
:10F9900012C08CE00E94B29187EE9AE09F938F9301
:10F9A0001F930F93E0919C05F0919D0509950F9091
:10F9B0000F900F900F9080E10E94B291809196017C
:10F9C00099279F938F938FED90E09F938F938091D2
:10F9D000770A9091780A9F938F938091750A9091FE
:10F9E000760A6AE070E00E94AC9F7F936F938CEE82
:10F9F0009AE09F938F9385EA91E99F938F93E0918B
:10FA00009C05F0919D0509958DB79EB70C968DBF0D
:10FA100012C082E00E94B2918FEF9AE09F938F9381
:10FA2000DF93CF93E0919C05F0919D0509950F9090
:10FA30000F900F900F90DF91CF911F910F9108952C
:10FA4000CF93C82F209144052093450599278F32E5
:10FA50009105E1F0803391051CF44F9779F027C0B0
:10FA60008F349105D9F08F38910509F586E0289FEC
:10FA7000F0011124E751F64F849117C086E0289FCA
:10FA8000F0011124E651F64F84910FC086E0289FC3
:10FA9000F0011124E551F64F849107C086E0289FBC
:10FAA000F0011124E451F64F849180934405909124
:10FAB0004405809145059813C0E08091AB01282F43
:10FAC00033278F5F8093AB0120FF0FC00E94B89156
:10FAD0009091440586E0989FF0011124E351F64F80
:10FAE000259134918C2FF901099580E090E0CF9118
:10FAF00008951092EC0A1092EB0A1092F00A1092FC
:10FB0000EF0A1092EE0A1092ED0A1092F10A82E3C7
:10FB100090E00E94691A90934705809346050895E6
:10FB2000E82FFF2783E0EE0FFF1F8A95E1F7E95EDC
:10FB3000F64F9581993C18F4892F99270895808173
:10FB400082FF07C08AE0989FC00111248850974027
:10FB50000895892F99270895A0E0B0E0E2EBFDE732
:10FB60000C9419A080914605909147050E94721A45
:10FB7000882309F4C0C08091460590914705C2963C
:10FB80009093470580934605C0E0D0E07E01BB24FA
:10FB90007FEFC72EDB2C07E119E0F801838187FF97
:10FBA00014C0B3948581893C30F08D2D0E94907DE6
:10FBB000C80FD91F02C0C80FD11DF8018181E80EFE
:10FBC000F11C86818C1508F4C82ED394085F1F4F52
:10FBD000FBE0FD1510F7C092F10AEF2841F52091E6
:10FBE0004C0530914D0540914E0550914F05BB2776
:10FBF000A52F942F832F90934B0580934A05AA2716
:10FC0000BB27281B390B4A0B5B0BCE01AA27BB274E
:10FC1000280F391F4A1F5B1F20934C0530934D0559
:10FC200040934E0550934F05C5E0D0E013C080913E
:10FC30004A0590914B058C179D0718F4C81BD90BEA
:10FC400002C0C0E0D0E08B2D9927880F991FC80F04
:10FC5000D91F2596D093EC0AC093EB0ACF3FD1056C
:10FC600078F480912601909127018C9F90018D9FBF
:10FC7000300D9C9F300D1124C90164E670E013C063
:10FC8000CE0196958795969587952091260130917E
:10FC90002701289FA001299F500D389F500D112446
:10FCA000CA0169E170E00E94AC9F7093EE0A609314
:10FCB000ED0A80914805909149058C0F9D1F909306
:10FCC00049058093480552E0813D9507A0F02091B9
:10FCD000EF0A3091F00A2F5F3F4F805D9240E2E0E3
:10FCE000813D9E07C0F79093490580934805309366
:10FCF000F00A2093EF0AE9E0CDB7DEB70C9435A007
:10FD000030915C05E32FFF2783E0EE0FFF1F8A95FC
:10FD1000E1F7E95EF64F2781422F552747FD5095C1
:10FD200080915D059927841795072CF420935D0534
:10FD300030935F050AC0222341F080915E05992728
:10FD40004817590714F420935E05832F8F5F809323
:10FD50005C058C30D0F010925C0580915E058F3F81
:10FD600019F08093550502C01092550580915D05EC
:10FD70008093560580915F05809354058FEF8093A3
:10FD80005E0510925D0510925F05089595E1899FCB
:10FD9000802D11240E947E9788EC9DE09F938F9385
:10FDA00080E597E99F938F93E0919C05F0919D05E5
:10FDB00009950F900F900F900F900895CF93C0E08A
:10FDC0004091AC01409353058091100485FF0CC015
:10FDD00080910704882331F080916708863011F400
:10FDE000CEE029C0C0E127C080912A058823D1F048
:10FDF000282F3327C90101968197A4F480914804E4
:10FE0000882341F4F901E20FF31FE35FF44F84917B
:10FE1000882341F4220F331F245F344FF901C4912A
:10FE2000CC2349F48091B30886FD03C01092AC0145
:10FE300004C0C42F02C0C0935305809160058C1785
:10FE400071F480916105909162050E94721A882375
:10FE500019F480E090E017C080EA9FE002C080EDD6
:10FE600097E00E94691A9093620580936105CC2304
:10FE700031F08091AC01C81711F41092AC01C0931D
:10FE800060058C2F9927CF91089520E030E050E055
:10FE90008091C40A992789389105B9F08A3891056B
:10FEA00034F481309105F1F00297F9F021C08D38DA
:10FEB0009105A1F08E38910524F48A38910541F01E
:10FEC00017C08E38910539F013C02AE43BE008C012
:10FED00022E23CE005C022EF3AE002C02EE13BE026
:10FEE0005CE206C025EC32E002C028ED32E054E0CE
:10FEF0009091B90A40E08091BA0A481770F49517BA
:10FF000060F4D901A90FB11DE42FFF27EA55F54F81
:10FF100085898C939F5F4F5FEECF089520E335E78F
:10FF2000809141018B3211F08D32F9F480915208A9
:10FF3000282F332780913D0490913E04829FA00199
:10FF4000839F500D929F500D1124CA0163E070E011
:10FF50000E94C09FCB019B01205D3A48C196C1978A
:10FF600008F03FC02EEF34E73CC0803229F5809185
:10FF7000100481FF36C02091500530915105205D5D
:10FF80003A4855E72133350748F085E724393807E3
:10FF900018F420E335E702C02456304045E720330B
:10FFA0003407F8F454E72D3C350718F020E335E723
:10FFB00018C02C593F4F15C08E3549F49091380424
:10FFC0008AE0989F90011124205D3A480AC0863744
:10FFD00041F4909138048AE0989FC0011124281BB5
:10FFE000390BC90108951F9399278A38910509F49F
:10FFF000A5C18B38910524F48938910551F05EC371
:020000021000EC
:100000008D38910509F491C28E38910509F4EAC141
:1000100055C30E94DE7E182F8093240C80914304E8
:1000200090914404A0914504B0914604BC01CD01D7
:1000300024E630E040E050E00E94F59FDA01C9017B
:100040008C509E4F9093500B80934F0B112319F4BB
:100050000E948E7F02C080E395E79093560B8093B9
:10006000550B8091550B9091560B9093580B8093A4
:10007000570B90935A0B8093590B20914F0B309153
:10008000500B8091530B9091540B2817390724F48F
:100090003093540B2093530B8091510B9091520B42
:1000A0008217930724F43093520B2093510B109234
:1000B0004C0B8AE49BE090937405809373058091C8
:1000C00041018093700B80910F0480FF02C083E494
:1000D00001C080E28093710B20912A05222311F147
:1000E000822F6AE00E94A09F805D80935B0B822F2D
:1000F0000E94A09F892F805D80935C0B8AE3809390
:100100005D0B81E1289FF0011124AEE5BBE0E25BCD
:10011000F44F9FE084918D939150319697FFFACFE1
:1001200080E241C080910704882361F0ABE5BBE029
:10013000E6E8FDE094E184918D939150319697FF2C
:10014000FACFB9C28091100485FF0CC0ABE5BBE0CB
:10015000ECE9FDE094E184918D939150319697FF05
:10016000FACFA9C280915205882301F1ABE5BBE02B
:10017000EFE7FDE096E084918D939150319697FFE3
:10018000FACF80910101805D80935F0BA2E6BBE016
:10019000E4EBF8E09BE081918D93915097FFFBCFCA
:1001A00080E280936D0B80936E0BB9C030915A053D
:1001B000332309F499C087E580935B0B80E5809336
:1001C0005C0B40E240935D0B20915B05822F6AE05F
:1001D0000E94A09F805D80935E0B822F0E94A09F53
:1001E000892F805D80935F0B8FE28093600B832F5C
:1001F0000E94A09F805D8093610B832F0E94A09F2F
:10020000892F805D8093620B4093630B209157058B
:100210003091580583E0293E380780F0C90168EE27
:1002200073E00E94AC9FCB01805D8093640BC90199
:1002300068EE73E00E94AC9F9C0102C04093640B87
:100240002536310580F0C90164E670E00E94AC9F5C
:10025000CB01805D8093650BC90164E670E00E946C
:10026000AC9F9C0103C080E28093650BC9016AE0EA
:1002700070E00E94AC9FCB01805D8093660BC9014A
:100280006AE070E00E94AC9F805D8093670B8DE612
:100290008093680B80E28093690B20915905253685
:1002A00060F0822F64E60E94A09F805D80936A0BBD
:1002B000822F0E94A09F292F02C080936A0B822F59
:1002C0006AE00E94A09F805D80936B0B822F0E944A
:1002D000A09F892F805D80936C0B83E780936D0BCB
:1002E00080E280936E0BE7C1809134048823D1F4BF
:1002F000ABE5BBE0E4EBFDE090E184918D939150A0
:10030000319697FFFACF92E390936B0B8EE2809336
:100310006C0B80E380936D0B90936E0B81E6809362
:100320006F0BC9C1ABE5BBE0E2EBFDE094E184916A
:100330008D939150319697FFFACFBDC180914304C0
:1003400090914404A0914504B0914604BC01CD01B4
:1003500024E630E040E050E00E94F59FDA01C90158
:100360008C509E4F9093380C8093370C8091240CC6
:10037000882319F40E948E7F02C080E395E7909352
:100380003A0C8093390C88E780933B0C8091720A79
:1003900080933C0C8091710A81FF02C084E407C005
:1003A0008091730A833011F480E201C081E280936E
:1003B0003D0C82E29CE090937405809373058091DC
:1003C00096018093490C80913D0C80934B0C809159
:1003D000770A9091780A97FD019695958795809375
:1003E0003E0C69C10E94807E809143049091440438
:1003F000A0914504B0914604BC01CD0124E630E053
:1004000040E050E00E94F59FDA01C9018C509E4FF8
:1004100090930D0B80930C0B8091260190912701F6
:100420009093070B8093060B8091260190912701F2
:100430009093090B8093080B8091120A9091130AF4
:1004400097FD0196959587958093F80A8093FF0A0A
:100450002091770A3091780A37FF02C02F5F3F4F13
:10046000359527952093FD0A8091750A9091760A1B
:1004700064E170E00E94AC9F6093FE0A2093040B3D
:100480006093050B8091240C882319F40E948E7FC1
:1004900002C080E395E79093150B8093140B88E7D7
:1004A0008093160B80912601909127019093110B58
:1004B0008093100B809155058C5E80930A0B809180
:1004C00056058C5E80930B0B8091EF0A9091F00A99
:1004D0006AE070E00E94AC9F7093130B6093120B64
:1004E0008091240C8093F40A8091EB0A9091EC0A9D
:1004F00090930F0B80930E0B82EF9AE0909374050C
:10050000809373052091EA023091EB02C9016CE3FC
:1005100070E00E94AC9F6093190BC9016CE370E01E
:100520000E94AC9F80931A0BC6C00E94807E80916F
:10053000750A9091760A64E670E00E94AC9F709311
:10054000340B6093330B8091120A9091130A97FD3C
:100550000196959587958093240B809190019091B9
:10056000910197FD0196959587958093250B809134
:10057000D3078093280B8091770A9091780A97FD92
:100580000196959587958093290B80910201482FBC
:1005900055279A012E5F3F4F8091260190912701A8
:1005A0002817390784F48091260190912701841B34
:1005B000950B9C01220F331F280F391F822F865065
:1005C0008093300B02C01092300B8091300B853637
:1005D00018F084E68093300B80912A059927909338
:1005E000320B8093310B8091430490914404A0918D
:1005F0004504B0914604BC01CD0124E630E040E062
:1006000050E00E94F59FDA01C9018C509E4F9093F3
:10061000360B8093350B80912601909127019093A2
:100620002B0B80932A0B80912601909127019093A8
:100630002D0B80932C0B8091240C882319F40E949D
:100640008E7F02C080E395E79093380B8093370B41
:100650008091240C88588093390B809126019091C9
:10066000270190933D0B80933C0B809155058C5E48
:1006700080932E0B809156058C5E80932F0B80917A
:10068000EF0A9091F00A6AE070E00E94AC9F7093CC
:100690003F0B60933E0B1092200B8091EB0A9091E0
:1006A000EC0A90933B0B80933A0B8EE19BE0909386
:1006B0007405809373052CE230E002C020E030E046
:1006C000C9011F910895EF92FF920F931F93CF934B
:1006D000DF9380915005909151059C0153E0220FCA
:1006E000331F5A95E1F7281B390B80913303909102
:1006F0003403280F391F37FF02C0295F3F4F43E003
:10070000359527954A95E1F730935105209350058B
:1007100090916405992309F026C380916305282FE1
:100720003327442755278F5F80936305F9012131D3
:10073000310508F015C3E757FF4F0C9447A080918F
:10074000100485FF2AC080E00E947E9780912601D8
:10075000909127016AE070E00E94C09F9F938F9361
:1007600080912601909127016AE070E00E94C09F6D
:100770007F936F938EED9DE09F938F9381E797E931
:100780009F938F93E0919C05F0919D0509952DB75E
:100790003EB7285F3F4F2DBF28C080E00E947E9764
:1007A00080912601909127016AE070E00E94C09F2D
:1007B0009F938F9380912601909127016AE070E0CA
:1007C0000E94C09F7F936F938BEE9DE09F938F93CA
:1007D00080E597E99F938F93E0919C05F0919D05AB
:1007E00009958DB79EB708968DBF8091560A80FFF8
:1007F0003FC0809160048823E9F08AE00E947E97E0
:100800008091410199279F938F9380914304909108
:100810004404A0914504B0914604BC01CD0124E6F6
:1008200030E040E050E00E94F59F3F932F9388EF27
:100830009DE0C8C68AE00E947E9780914304909113
:100840004404A0914504B0914604BC01CD0124E6C6
:1008500030E040E050E00E94F59F3F932F9384E00A
:100860009EE09F938F9380E597E99F938F93D1C7E5
:100870008AE00E947E978FE09EE09F938F9380E5B1
:1008800097E90C94348D8091100485FF2AC085E18E
:100890000E947E978091EA029091EB026CE370E0F7
:1008A0000E94AC9F9F938F938091EA029091EB02FC
:1008B0006CE370E00E94AC9F7F936F9389E19EE0B0
:1008C0009F938F9381E797E99F938F93E0919C0586
:1008D000F0919D0509952DB73EB7285F3F4F2DBF7D
:1008E00028C085E10E947E978091EA029091EB02F8
:1008F0006CE370E00E94AC9F9F938F938091EA021B
:100900009091EB026CE370E00E94AC9F7F936F9339
:1009100086E29EE09F938F9380E597E99F938F9364
:10092000E0919C05F0919D0509958DB79EB70896BD
:100930008DBF8FE10E947E9780E690E09F938F931A
:100940008091120A9091130A9F938F9383E39EE004
:100950009F938F93C0E5D7E9DF93CF93E0919C05F8
:10096000F0919D05099580910F042DB73EB7285F42
:100970003F4F2DBF80FF06C089E20E947E978EE325
:100980009EE06FC389E20E947E9780E49EE0E2C60B
:100990008091100485FF1BC08AE20E947E9780919F
:1009A000EF0A9091F00A9F938F9382E49EE09F93C9
:1009B0008F9381E797E99F938F93E0919C05F09146
:1009C0009D0509958DB79EB706968DBF1BC08AE21F
:1009D0000E947E978091EF0A9091F00A9F938F93E7
:1009E0008AE49EE09F938F9380E597E99F938F938E
:1009F000E0919C05F0919D0509952DB73EB72A5FC2
:100A00003F4F2DBF86E30E947E978091EB0A909125
:100A1000EC0A6AE070E00E94AC9F9F938F938091F4
:100A2000EB0A9091EC0A6AE070E00E94AC9F7F9321
:100A30006F9382E59EE09F938F9380E597E99F9364
:100A40008F93E0919C05F0919D0509958DB79EB718
:100A50000896E7C689E00E947E978EE59EE09F9308
:100A60008F9300E517E91F930F93E0919C05F09198
:100A70009D0509958EE10E947E970F900F900F9033
:100A80000F9080E69EE09F938F931F930F93E091CA
:100A90009C05F0919D05099583E30E947E970F9038
:100AA0000F900F900F9082E69EE09F938F931F937D
:100AB0000F93E0919C05F0919D0509958FE30E94AD
:100AC0007E970F900F900F900F9084E69EE09F937B
:100AD0008F931F930F93E0919C05F0919D050995CD
:100AE0008EE70E947E970F900F900F900F908AE7ED
:100AF0009EE09F938F931F930F93B8C78091A4019B
:100B0000882309F462C08DE50E947E9780E99EE00B
:100B10009F938F93C0E5D7E9DF93CF93E0919C0536
:100B2000F0919D05099584E50E947E970F900F90A6
:100B30000F900F908091720A99279F938F9382E96B
:100B40009EE09F938F93DF93CF93E0919C05F0916C
:100B50009D0509958EE50E947E972DB73EB72A5FC9
:100B60003F4F2DBF8091750A9091760A6AE070E040
:100B70000E94AC9F7F936F938BE99EE09F938F932E
:100B8000DF93CF93E0919C05F0919D0509958DB77A
:100B90009EB706968DBF8091730A833081F4809151
:100BA000710A81FF06C08BE50E947E9785EA9EE070
:100BB000D1C58BE50E947E9788EA9EE0CBC58BE588
:100BC0000E947E978BEA9EE04BC784E0FCC3809135
:100BD000A401882309F47AC08091660520E5E22EFD
:100BE00027E9F22E882309F44BC089E60E947E97FC
:100BF0008091290599279F938F938EEA9EE09F937A
:100C00008F93FF92EF92E0919C05F0919D050995DD
:100C100085E70E947E972DB73EB72A5F3F4F2DBFD5
:100C20008091960199279F938F9300E610E01F9380
:100C30000F938091770A9091780A9F938F9389EB15
:100C40009EE09F938F93FF92EF92E0919C05F0912D
:100C50009D05099582E70E947E978DB79EB70A96FB
:100C60008DBF8091270599279F938F931F930F9393
:100C70008091280599279F938F9385EC9EE091C6DC
:100C800089E60E947E978091960199279F938F9382
:100C900080E690E09F938F938091770A9091780AF5
:100CA0009F938F938091740A99279F938F9385EDDB
:100CB0009EE09F938F93FF92EF92E0919C05F091BD
:100CC0009D0509958DB79EB70C96ABC585E07BC396
:100CD00090912A059923D1F080917005882381F0A5
:100CE000913270F487E00E94C67E83E90E947E976D
:100CF00080912A0599279F938F938EEE9EE0CDC316
:100D000083E90E947E9789EF9EE0DCC38091100406
:100D100090E5E92E97E9F92E85FF06C084E90E9447
:100D20007E978FEF9EE003C483E90E947E9782E165
:100D30009FE0FDC38091870C863059F48091660551
:100D4000882319F010926605B8C681E08093660585
:100D5000B4C6883009F0B1C60E94839781E004C40C
:100D600090936305B2C6913009F009C48091630580
:100D7000282F3327442755278F5F80936305F90178
:100D80002131310508F09CC6E656FF4F0C9447A070
:100D90008091100485FF43C080E00E947E9780917F
:100DA000EF0A9091F00A9F938F9380912601909182
:100DB00027016AE070E00E94C09F9F938F9380910B
:100DC0002601909127016AE070E00E94C09F7F9306
:100DD0006F938091EA029091EB026CE370E00E94C5
:100DE000AC9F9F938F938091EA029091EB026CE30A
:100DF00070E00E94AC9F7F936F9388E29FE09F9387
:100E00008F9381E797E99F938F93E0919C05F091F1
:100E10009D0509952DB73EB7225F3F4FCFC580E0B6
:100E20000E947E978091EF0A9091F00A9F938F9392
:100E300080912601909127016AE070E00E94C09F96
:100E40009F938F9380912601909127016AE070E033
:100E50000E94C09F7F936F938091EA029091EB0272
:100E60006CE370E00E94AC9F9F938F938091EA02A5
:100E70009091EB026CE370E00E94AC9F7F936F93C4
:100E800083E49FE0EBC285E10E947E9780E690E0DC
:100E90009F938F9380919001909191019F938F9355
:100EA0008EE59FE09F938F93C0E5D7E9DF93CF93C3
:100EB000E0919C05F0919D0509958091560A2DB70A
:100EC0003EB7285F3F4F2DBF80FF51C08091600427
:100ED000882339F18FE10E947E978091430490919D
:100EE0004404A0914504B0914604BC01CD0124E620
:100EF00030E040E050E00E94F59F3F932F9388E65A
:100F00009FE09F938F9380E697E99F938F93E09163
:100F10009C05F0919D0509958DB79EB706968DBFEE
:100F200038C08FE10E947E978091430490914404E1
:100F3000A0914504B0914604BC01CD0124E630E007
:100F400040E050E00E94F59F3F932F9381E79FE0A0
:100F50009F938F93DF93CF93E0919C05F0919D0534
:100F600009952DB73EB72A5F3F4F2DBF12C08FE1C5
:100F70000E947E978AE79FE09F938F93DF93CF93A2
:100F8000E0919C05F0919D0509950F900F900F90B1
:100F90000F9089E20E947E978091410199279F934B
:100FA0008F9384E89FE031C48091A4018823F9F0F5
:100FB0008BE20E947E978091960199279F938F9351
:100FC0008091750A9091760A6AE070E00E94AC9F69
:100FD0007F936F9380E690E09F938F938091770A41
:100FE0009091780A9F938F9387E89FE068C182E091
:100FF000EAC18FE30E947E978091ED0A9091EE0AFC
:101000009F938F938091EB0A9091EC0A6AE070E0D5
:101010000E94AC9F9F938F938091EB0A9091EC0A72
:101020006AE070E00E94AC9F7F936F938EE99FE02F
:101030009F938F93C0E5D7E9DF93CF93E0919C0511
:10104000F0919D05099580910F042DB73EB7265F5D
:101050003F4F2DBF80FF0AC082E50E947E9782EB42
:101060009FE09F938F9380E697E9FEC482E50E94FC
:101070007E9785EB9FE06EC38091A40100E5E02E92
:1010800007E9F02E882309F449C084E50E947E9781
:101090008091720A99279F938F938091740A992760
:1010A0009F938F9388EB9FE09F938F93E701FF922D
:1010B000EF92E0919C05F0919D0509958DB79EB743
:1010C00008968DBF8091730A833051F484E60E94A4
:1010D0007E978BEC9FE09F938F93FF92EF920BC0D4
:1010E00084E60E947E9781ED9FE09F938F9381E736
:1010F00097E99F938F93E0919C05F0919D05099549
:101100000F900F900F900F908091710A81FFDDC4B6
:1011100084E60E947E9787ED9FE01CC384E50E94D1
:101120007E978DED9FE003C28091650510E5E12E6D
:1011300017E9F12E882309F45BC089E60E947E97A7
:1011400083E00E94907D6AE070E00E94AC9F9F93D4
:101150008F9383E00E94907D6AE070E00E94AC9FD4
:101160007F936F9382E00E94907D6AE070E00E941E
:10117000AC9F9F938F9382E00E94907D6AE070E025
:101180000E94AC9F7F936F9381E00E94907D6AE004
:1011900070E00E94AC9F9F938F9381E00E94907DAE
:1011A0006AE070E00E94AC9F7F936F9380E00E94A2
:1011B000907D6AE070E00E94AC9F9F938F9380E0E7
:1011C0000E94907D6AE070E00E94AC9F7F936F93D5
:1011D00083EF9FE09F938F93FF92EF92E0919C05A6
:1011E000F0919D0509952DB73EB72C5E3F4FE6C3A4
:1011F00089E60E947E9780E690E09F938F9380918E
:101200003609992787FD90959F938F9380912E099A
:10121000992787FD90959F938F9380912609992711
:1012200087FD90959F938F9380911E09992787FD45
:1012300090959F938F9380E190E19F938F93FF927E
:10124000EF92E0919C05F0919D0509958DB79EB7B1
:101250000E96E7C28091650590913F08882309F4B6
:10126000AFC0943009F4AEC09630C9F58EE70E9445
:101270007E9785E00E94907D6AE070E00E94AC9FBE
:101280009F938F9385E00E94907D6AE070E00E94BA
:10129000AC9F7F936F9384E00E94907D6AE070E042
:1012A0000E94AC9F9F938F9384E00E94907D6AE0A0
:1012B00070E00E94AC9F7F936F9383E290E19F93D5
:1012C0008F9380E597E99F938F93E0919C05F09130
:1012D0009D0509952DB73EB7245F3F4F6FC39730EB
:1012E00008F4F3C38EE70E947E9788E00E94907D09
:1012F0006AE070E00E94AC9F9F938F9388E00E9409
:10130000907D6AE070E00E94AC9F7F936F9387E0CE
:101310000E94907D6AE070E00E94AC9F9F938F9343
:1013200087E00E94907D6AE070E00E94AC9F7F930E
:101330006F9386E00E94907D6AE070E00E94AC9F0F
:101340009F938F9386E00E94907D6AE070E00E94F8
:10135000AC9F7F936F9385E00E94907D6AE070E080
:101360000E94AC9F9F938F9385E00E94907D6AE0DE
:1013700070E00E94AC9F7F936F9384E00E94907D09
:101380006AE070E00E94AC9F9F938F9384E00E947C
:10139000907D6AE070E00E94AC9F7F936F9382E340
:1013A00090E19F938F9380E597E99F938F93E091CE
:1013B0009C05F0919D0509958DB79EB7489631C261
:1013C000943021F486E00E94C67E7FC39630F1F40B
:1013D0008EE70E947E9780E690E09F938F938091A6
:1013E0004609992787FD90959F938F9380913E0999
:1013F000992787FD90959F938F938FE490E19F931A
:101400008F9380E597E99F938F93CFC2973008F42D
:101410005CC38EE70E947E9780E690E09F938F9357
:1014200080915609992787FD90959F938F9380917E
:101430004E09992787FD90959F938F938091460938
:10144000992787FD90959F938F9380913E099927C7
:1014500087FD90959F938F9382E690E19F938F9362
:1014600080E597E99F938F93ECCE90912A0599237D
:1014700009F44AC0809170058823F9F09132E8F4AC
:1014800087E00E94C67E83E90E947E9780912A05AC
:1014900099279F938F9385E790E19F938F9380E6A1
:1014A00097E99F938F93E0919C05F0919D05099595
:1014B0002DB73EB72A5F3F4F81C283E90E947E97D6
:1014C00080E890E19F938F9300E517E91F930F93B6
:1014D000E0919C05F0919D0509951F921F929091B6
:1014E0002A0581E1989FC0011124825B944F9F934C
:1014F0008F931F930F93E0919C05F0919D050995A3
:101500008DB79EB70A968DC180911004C0E5EC2E70
:10151000C7E9FC2E85FF06C084E90E947E9786E815
:1015200090E105C083E90E947E9789E990E19F934D
:101530008F93FF92EF929AC28091870C863079F454
:1015400080916505882319F01092650503C081E03C
:101550008093650585E00E94C67E86E0A3C2883040
:1015600031F40E94839782E080936405A4C28130A5
:1015700009F0A3C20E948397109264059CC2923026
:1015800009F0A1C280916305282F332744275527EE
:101590008F5F80936305F9012131310508F090C216
:1015A000E555FF4F0C9447A080E00E947E9784EBA6
:1015B00098E09F938F938091010199279F938F9338
:1015C0008FEA90E19F938F9380E697E99F938F93A3
:1015D000E0919C05F0919D0509952DB73EB7285FD8
:1015E0003F4FECC185E10E947E9782EC98E09F938B
:1015F0008F93809102016AE00E94A09F892F992712
:101600009F938F93809102010E94A09F99279F939F
:101610008F938EEB90E19F938F9380E597E99F9353
:101620008F93E0919C05F0919D05099569CF8AE221
:101630000E947E978FEC90E19F938F93C0E5D7E94E
:10164000DF93CF93E0919C05F0919D0509958091E2
:10165000560A0F900F900F900F9080FF41C080911D
:101660004D089091260481FD0BC0892F99279F93E7
:101670008F9384ED90E19F938F93DF93CF9313CF5C
:10168000E0919C05F0919D05933318F08EED90E16B
:1016900002C085EE90E19F938F93DF93CF930995DE
:1016A0000F900F900F900F908091390AE0919C0558
:1016B000F0919D059091260480FF0BC0892F9927FA
:1016C0009F938F938CEE90E19F938F93DF93CF93B3
:1016D000A4C0892F99279F938F9382EF90E1C4C074
:1016E00088EF90E137C08FE30E947E9781E091E11F
:1016F0009F938F93C0E5D7E9DF93CF93E0919C054B
:10170000F0919D0509950F900F900F900F9080918B
:10171000A308882319F485E091E11CC080911D0481
:10172000E0919C05F0919D05882319F08EE091E1F0
:1017300002C085E191E19F938F93DF93CF93099549
:101740000F900F900F900F908091B20886FFBDC14F
:101750008CE191E19F938F93DF93CF9387C184E5D1
:101760000E947E9783E291E19F938F93C0E5D7E932
:10177000DF93CF93E0919C05F0919D0509958091B1
:10178000560A0F900F900F900F9085FD03C088E2CE
:1017900091E108C0809191080E947348823358F407
:1017A00081E391E19F938F93DF93CF93E0919C0529
:1017B000F0919D0516C0843B18F088E391E1F2CFCB
:1017C0008091B208E0919C05F0919D0585FF03C0D2
:1017D0008FE391E102C086E491E19F938F93DF93C1
:1017E000CF9309950F900F900F900F908091A708BD
:1017F000882309F46AC18EE50E947E978091A7082C
:1018000099279F938F938DE491E19F938F93DF931B
:10181000CF93E0919C05F0919D0509958DB79EB7FA
:1018200006968DBF52C189E60E947E9788E591E1B8
:101830009F938F93C0E5D7E9DF93CF93E0919C0509
:10184000F0919D0509950F900F900F900F9080914A
:10185000A608E0919C05F0919D05882351F09927F9
:101860009F938F9382E691E19F938F93DF93CF9322
:101870001ECE86E691E19F938F93DF93CF93FAC0BC
:1018800080916705B0E5EB2EB7E9FB2E882309F0C0
:1018900053C08EE70E947E9780916F0199279F9396
:1018A0008F9380914208E82FFF27EE0FFF1FE85823
:1018B000F64F808191819F938F9380914108E82F0B
:1018C000FF27EE0FFF1FE858F64F808191819F930D
:1018D0008F938CE691E19F938F93FF92EF92E0912B
:1018E0009C05F0919D05099583E90E947E978DB72F
:1018F0009EB70A968DBF80914408E82FFF27EE0F10
:10190000FF1FE858F64F808191819F938F938091BC
:101910004308E82FFF27EE0FFF1FE858F64F80819E
:10192000918181589F4F9F938F9380E891E19F937E
:101930008F93FF92EF924CCE8EE70E947E9780911C
:101940004C0499279F938F9380914B0499279F93E1
:101950008F9380914A0499279F938F938FE891E109
:101960009F938F93FF92EF92E0919C05F0919D05DC
:10197000099583E90E947E978DB79EB70A968DBF21
:1019800080914F0499279F938F9380914E049927BC
:101990009F938F9380914D0499279F938F9383EA10
:1019A00091E19F938F93FF92EF92E0919C05F091CC
:1019B0009D0509952DB73EB7265F3F4F2DBF85C0CA
:1019C00080917005882309F480C08EE70E947E977D
:1019D0008091560A86FD11C087EB91E19F938F930A
:1019E00081E797E99F938F93E0919C05F0919D0586
:1019F00009950F900F900F900F908091B008992744
:101A00008F709070892B89F086EC91E19F938F9372
:101A100081E797E99F938F93E0919C05F0919D0555
:101A200009950F900F900F900F908091560A82FFAA
:101A300011C080ED91E19F938F9381E797E99F9388
:101A40008F93E0919C05F0919D0509950F900F9063
:101A50000F900F908091560A83FD37C085ED91E17C
:101A60009F938F9381E797E99F938F93E0919C05D4
:101A7000F0919D0509950F900F900F900F9025C044
:101A80000091870C063089F480916705882319F04E
:101A90001092670503C081E08093670586E00E948D
:101AA000C67E87E00E94C67E08C0013031F40E94E5
:101AB000839700936405109263051092870C05C00C
:101AC0001092630502C010926405E6E0CDB7DEB760
:101AD0000C9438A04FB728E130E0F8948091C90009
:101AE0008F778093C9008091C9008F7B8093C90054
:101AF0008091C9008F7D8093C900832F992780939F
:101B0000CD002093CC008091C80082608093C800F3
:101B100080E18093C9008091CA008F778093CA00CA
:101B20008091CA008F7B8093CA008091CA00809107
:101B3000CA008F7E8093CA008091CA00886080931B
:101B4000CA008091C9008B7F8093C9008091CA0030
:101B500084608093CA008091CA0082608093CA002A
:101B60008091C80087FF03C08091CE00F9CF80919B
:101B7000C90080688093C9008091650C846080935F
:101B8000650C4FBF089590913D05992341F48F3026
:101B900031F49093690580E580933D050895E091C7
:101BA0006905EF5FE0936905E83121F481E08093F6
:101BB00068050895E93120F089E180936905089569
:101BC000FF27E25BF34F80830895A0E0B0E0EBEEE7
:101BD000FDE80C9418A091E0D92E82E0A82EBD2C2F
:101BE000E12C01E0F02E8091650C82FDB5C0809162
:101BF0006F008F7D80936F00E091A908EE2351F074
:101C0000FF27EE0FFF1FE858F64F80819181843641
